:100000000C94BC2B0D94B6240D948B240D94602479
:100010000D9435240D940A240D94DF230D94B423FC
:100020000D9489230C94ED2B0C94ED2B0C94ED2B5B
:100030000C94ED2B0C943B830C94ED2B0C94ED2B3A
:100040000C94ED2B0C94EB850C94ED2B0C94ED2B78
:100050000C94ED2B0C94ED2B0C94DA830D94E1248D
:100060000C94ED2B0C94BC8C0C94ED2B0C94ED2B80
:100070000C94ED2B0C94ED2B0C94ED2B0C94ED2BA0
:100080000C94ED2B0C94ED2B0C94ED2B0C94ED2B90
:100090000C94ED2B0C94ED2B0C94ED2B0C94ED2B80
:1000A0000C94ED2B0C94ED2B0C94ED2B0C94ED2B70
:1000B0000C94ED2B0C94ED2B0C94ED2B0C94ED2B60
:1000C0000C94ED2B0C94ED2B0C94ED2B0C94ED2B50
:1000D0000C94ED2B0C94ED2B0C94ED2B0C94ED2B40
:1000E0000C94ED2B246724672B672B672B673267F3
:1000F000326732673F6739673967396779847D844A
:10010000A684AA848C8497846684F08CF68C078DF0
:10011000128D1A8D2F8D1E8D2F8D228D268D2F8D58
:100120002C8D07C70CC711C71BC725C79EC72FC774
:1001300037C73FC749C753C75DC76CC776C79EC798
:1001400080C78AC794C7EF000B01ED000D01DF00E7
:100150001901F100E1001301FB00DB00FD00F700D5
:1001600009011901E900DD00E500084AD73B3BCE53
:10017000016E84BCBFFDC12F3D6C74319ABD5683A6
:100180003DDA3D00C77F11BED9E4BB4C3E916BAA5E
:10019000AABE000000803F05A84CCDB2D44EB938AD
:1001A00036A9020C50B9918688083CA6AAAA2ABE94
:1001B000000000803F000D94D6160D94EE160D94AD
:1001C000B9160D94C8160D942B250D94F2160D94A6
:1001D0006C090D94EA160D94A1160D94AF160D94AA
:1001E000BD160D94C4160D942D210D94CE070D94BB
:1001F000E0160D94991D0D94D2160D94DC160D94F5
:10020000A3160D94961B0D945F160D9471160D9404
:1002100063160D94E4160D94C0160D94B3160D9448
:100220004B0B0D9460160D94CE160D9437160D944D
:100230006A230D94F71647322F47332062616420FA
:10024000706172616D65746572730A00536C6565E7
:10025000702E2E2E00205A3A200020593A200042BB
:10026000656420583A20004C756C7A426F742054B3
:10027000415A20362072656164792E00526573758B
:100280006D696E67207072696E7400436C69636B90
:1002900020746F20726573756D652E2E2E004E6F63
:1002A000206D6F76652E004D313235002569730063
:1002B00025696D20256973002569682025696D20F1
:1002C00025697300256964202569682025696D20EA
:1002D00025697300256979202569642025696820CE
:1002E00025696D20256973005072696E74207469E8
:1002F0006D653A2000000125301D0C1824311C0BBF
:1003000017232F1B0A1E16040306080202222B1AAB
:100310004142212A193F40033809FF3607FF372899
:10032000294527444350726F746563746564205097
:10033000696E0A00457874727564657220256920BB
:100340002573004C756C7A426F742054415A2036E4
:100350002072656164792E0042656420646F6E6569
:100360002E0020573A004265642068656174696E0A
:10037000672E0042656420636F6F6C696E672E00A4
:100380004C756C7A426F742054415A2036204F6667
:10039000662E004361703A454D455247454E4359DC
:1003A0005F5041525345523A310A004361703A431B
:1003B0004153455F4C494748545F4252494748546E
:1003C0004E4553533A300A004361703A544F474701
:1003D0004C455F4C49474854533A300A00436170DA
:1003E0003A534F4654574152455F504F5745523A42
:1003F000300A004361703A4C4556454C494E475FC0
:10040000444154413A310A004361703A5A5F5052B4
:100410004F42453A310A004361703A4155544F4CBE
:100420004556454C3A310A004361703A5052494EA4
:10043000545F4A4F423A310A004361703A50524F7A
:1004400047524553533A300A004361703A4155547C
:100450004F5245504F52545F54454D503A310A0067
:100460004361703A454550524F4D3A310A00464972
:10047000524D574152455F4E414D453A4D61726C68
:10048000696E20204649524D574152455F564552AC
:1004900053494F4E3A312E312E352E3434204558A3
:1004A0005452554445525F545950453A4475616C15
:1004B000457874727564657220763220534F5552B8
:1004C00043455F434F44455F55524C3A68747470DE
:1004D000733A2F2F636F64652E616C6570686F626D
:1004E0006A656374732E636F6D2F646966667573D6
:1004F000696F6E2F4D41524C494E2050524F544F10
:10050000434F4C5F56455253494F4E3A312E30209F
:100510004D414348494E455F545950453A4C756CDE
:100520007A426F742054415A20362045585452550F
:100530004445525F434F554E543A32205555494435
:100540003A38343566303033632D616562642D345A
:100550006535332D613662392D376430393834666C
:1005600064653630390A004D31343520533C696EAC
:100570006465783E206F7574206F662072616E67C7
:10058000652028302D31290A00205A0020590058B2
:100590000020204D61783A2000205A002059005850
:1005A0000020204D696E3A20004F6E20004F666695
:1005B00000536F667420656E6473746F70733A20B5
:1005C00000486F74656E64206F6666736574733A75
:1005D0000020643A0020693A0020703A0020643A12
:1005E0000020693A0020703A0043290A0061626CD9
:1005F000656420286D696E2074656D702000436FFE
:100600006C6420657874727564657320617265200E
:10061000004B64200023646566696E6520204445B4
:100620004641554C545F004B692000236465666960
:100630006E65202044454641554C545F004B702068
:100640000023646566696E65202044454641554C2B
:10065000545F00504944204175746F74756E652075
:1006600066696E69736865642120507574207468CA
:1006700065206C617374204B702C204B6920616E77
:1006800064204B6420636F6E7374616E74732066B4
:10069000726F6D2062656C6F7720696E746F204396
:1006A0006F6E66696775726174696F6E2E680A0095
:1006B000504944204175746F74756E652066616998
:1006C0006C6564212074696D656F75740A0050490A
:1006D00044204175746F74756E65206661696C6540
:1006E00064212054656D7065726174757265207443
:1006F0006F6F20686967680A00204B643A20002009
:100700004B693A2000204B703A20000A20436C616C
:100710007373696320504944200A002054753A20BD
:1007200000204B753A2000206D61783A2000206D42
:10073000696E3A200020643A200020626961733AB1
:100740002000426564204C6576656C696E67200008
:100750004661696C656420746F20656E61626C65CA
:1007600020426564204C6576656C696E670A0042BC
:100770006564204C6576656C20436F7272656374A6
:10078000696F6E204D61747269783A000000B0C1E3
:1007900000809743000000004F6666736574732005
:1007A0006170706C696564004572723A20546F6FB5
:1007B000206661722100546F6F206661722066723C
:1007C0006F6D207265666572656E636520706F6916
:1007D0006E740A004E6F2063617365206C696768F0
:1007E000740A004163746976652045787472756493
:1007F00065723A2000556E6B6E6F776E20636F6D79
:100800006D616E643A202200434F4D4D554E494371
:100810004154494F4E0044525952554E0045525290
:100820004F525300494E464F004543484F00100079
:10083000C90210012C014001220170011801B00110
:100840000E01F00104015002FA00B002F000300382
:10085000E600D003DC009004D2007005C800A006BA
:10086000BE000008B400B009AA00D00BA000600EC2
:10087000960060118C000015820020197800C01DC0
:100880006E00A0226400B0275A00902C5000003166
:100890004600E0343C0010383200903A2800603CBA
:1008A0001E00A03D1400803E0A00203F00002F2FB4
:1008B0002000290824081D08160808086F6666002D
:1008C00044454255473A0020706F736974696F6EF2
:1008D000206F7574206F662072616E67652E0A0046
:1008E0003F50726F626520001000AD0330016A0155
:1008F00050022B0170030A019004F500B005E500D9
:10090000D006D800F007CE001009C500300ABE009E
:10091000500BB700700CB100900DAB00B00EA600EC
:10092000D00FA200F0109D00101299003013950016
:100930005014920070158E0090168B00B01787002F
:10094000D0188400F0198100101B7E00301C7B0041
:10095000501D7900701E7600901F7300B02070004B
:10096000D0216E00F0226B00102469003025660053
:10097000502663007027610090285E00B0295C005B
:10098000D02A5900F02B5600102D5400302E510063
:10099000502F4E0070304B0090314800B03245006F
:1009A000D0334200F0343E0010363B003037370081
:1009B0005038330070392E00903A2900B03B2300A4
:1009C000D03C1B00F03D1100103F0100F03F000043
:1009D00053442063617264206F6B0A006F70656E10
:1009E000526F6F74206661696C65640A00766F6C83
:1009F000756D652E696E6974206661696C65640A3F
:100A000000534420696E6974206661696C0A007C39
:100A10003C3E5E2B3D3F2F5B5D3B2C2A225C0065FC
:100A20006E7175657565696E672022004572726F1B
:100A3000722077726974696E6720746F2045455023
:100A4000524F4D210A00486F6D652025732573258F
:100A500073206669727374002066697273740A0089
:100A60005A0059005800486F6D652000577269742C
:100A7000696E6720746F2066696C653A20006F703C
:100A8000656E206661696C65642C2046696C653A08
:100A900020006F70656E206661696C65642C20466D
:100AA000696C653A200046696C652073656C656306
:100AB0007465640A002053697A653A200046696CBF
:100AC00065206F70656E65643A20006F70656E20FA
:100AD0006661696C65642C2046696C653A2000206B
:100AE00066696C653A20004E6F7720002220706F97
:100AF00073002220706172656E743A220053554271
:100B0000524F5554494E452043414C4C207461721C
:100B10006765743A22004B494C4C45442E200074C2
:100B20007279696E6720746F2063616C6C207375D5
:100B3000622D67636F64652066696C6573207769F1
:100B4000746820746F6F206D616E79206C657665B6
:100B50006C732E204D4158206C6576656C2069734E
:100B60003A00004D3234004D363030204230004DD6
:100B70003234004D3233202573006175746F25695E
:100B80002E670043616E6E6F7420656E746572200F
:100B90007375626469723A2000022E2E004D6169FD
:100BA0006E000A003B20454550524F4D20496E646F
:100BB00065783A20005570646174696E67207A6FB9
:100BC000666673657420696E20454550524F4D3AF4
:100BD00020000600060006000600060006000600CB
:100BE000060006003FC01F800F00060006000F0031
:100BF0001F803FC006000600060006000600060033
:100C000006000600060007F8000C0C001002002089
:100C100001006001804000804003E04001C04000CE
:100C20008040000040000060000020000010000034
:100C30000C0C0007F80001FE00030300040080080C
:100C400000401800601000207C00203800201000B8
:100C50002000002000002000006000004000008014
:100C600003030001FE00FFFFFF7F80FFC0FFC0FF06
:100C7000C07F807F80FFC0FFC0FFC03F001E000C10
:100C8000005A204F6666736574004D6F7665205874
:100C9000004D6F76652059004D6F7665205A0045EE
:100CA0007874727564657232004578747275646523
:100CB000723100506C6561736520726573657400F4
:100CC0005052494E5445522048414C5445440050DE
:100CD00072696E7465722068616C7465642E206B35
:100CE000696C6C28292063616C6C6564210A006260
:100CF00065640A002C2073797374656D2073746FBA
:100D00007070656421204865617465725F49443A7A
:100D10002000544845524D414C2052554E415741B8
:100D2000592042454400546865726D616C205275CB
:100D30006E6177617900544845524D414C205255BF
:100D40004E4157415920453100544845524D414C80
:100D50002052554E41574159204530004865617435
:100D6000696E67206661696C65642042454400488D
:100D7000656174696E67206661696C6564004865C9
:100D80006174696E67206661696C656400486561BD
:100D900074696E67206661696C656420453100483E
:100DA000656174696E67206661696C6564204530B1
:100DB0000000002100240027002A002D003000330D
:100DC0000001010000040107010A010102102020B6
:100DD000080810204010204080020102010804028F
:100DE0000101020408102040808040201008040205
:100DF000018004020180402010080402010804025E
:100E00000101020408102040800102040810204063
:100E10008005050505070508080808020202020A00
:100E20000A0808040404040101010101010101038D
:100E300003030303030303040707070C0C0C0C0C48
:100E40000C0C0C0202020206060606060606060B3B
:100E50000B0B0B0B0B0B0B1FFFFFFFFFFFFF6000CC
:100E600000000001FF400000000000FF80000000C3
:100E700000007F83CF00000C303F87FF80000C30E4
:100E80001F867980000C000F8C30C7838C30E78C74
:100E900030CFC7CC31F38C30DCECEC33B98C30D8AC
:100EA0006C6C33198C30D06C0C33198C30D86C0CC2
:100EB00033198C30DC6C0E3B198C30CF7C079F19BA
:100EC0008C30C77C038F19400000000000026000D6
:100ED00000000000061FFFFFFFFFFFF82020506CFE
:100EE000616E6E657242756666657242797465738D
:100EF0003A20002046726565204D656D6F72793A23
:100F00002000436F6D70696C65643A204E6F7620E7
:100F1000323120323031370A00207C20417574682C
:100F20006F723A2028416C657068204F626A656371
:100F3000747320496E632E2C204C756C7A426F744A
:100F400020476974205265706F7369746F727929D4
:100F50000A004E6F76203231203230313731333A49
:100F600033373A353600204C617374205570646114
:100F70007465643A2000312E312E350A004D6172BD
:100F80006C696E0020536F667477617265205265DC
:100F90007365740A00205761746368646F67205238
:100FA000657365740A002042726F776E206F7574E6
:100FB0002052657365740A002045787465726E610D
:100FC0006C2052657365740A00506F7765725570B6
:100FD0000A0073746172740A006572726F7220770E
:100FE000726974696E6720746F2066696C650A00A7
:100FF0004572726F723A00456E6473746F7073203D
:1010000025632025632025632025630020503A00B6
:10101000205A3A0020593A0020583A00656E64730D
:10102000746F7073206869743A20006563686F3A62
:1010300000446F6E6520736176696E672066696C27
:10104000652E0A004D3239004B494C4C45442E2048
:101050000024F4D43050C38E20C2A24017828B707B
:1010600011127A910D816CD90AA861E108C75866FE
:1010700007615143061E4B5D05C145A7041A411186
:1010800004093D9803713931034036DB0265339121
:1010900002D4305402802E1D02632CEE01752AC545
:1010A00001B028A001102781018F2564012B244B5A
:1010B00001E0223401AC211F018D200D01801FFCB5
:1010C00000841EED00971DDF00B81CD200E61BC691
:1010D00000201BBC00641AB200B219A8000A19A0B3
:1010E000006A189900D117910040178B00B516843B
:1010F0000031167E00B31579003A157300C7146FDE
:101100000058146A00EE1366008813630025135E0E
:1011100000C7125B006C12570015125400C1115128
:101120000070114F0021114B00D61049008D10475F
:10113000004610440002104200C00F4000800F3EE5
:1011400000420F3C00060F3B00CB0E3800930E37D9
:10115000005C0E3500270E3400F30D3200C10D3156
:1011600000900D3000600D2E00320D2D00050D2C6D
:1011700000D90C2B00AE0C2900850C29005C0C2733
:1011800000350C27000E0C2600E80B2400C40B24AD
:1011900000A00B23007D0B23005A0B2100390B21EB
:1011A00000180B2000F80A1F00D90A1E00BB0A1EF7
:1011B000009D0A1D00800A1D00630A1C00470A1BCF
:1011C000002C0A1B00110A1A00F7091A00DD091980
:1011D00000C4091900AB091900920917007B09180E
:1011E00000630917004C091600360916002009167D
:1011F000000A091500F5081500E0081400CC0814D1
:1012000000B8081400A4081400900813007D081208
:10121000006B081300580812004608120034081129
:1012200000230811001208110001081100F0071036
:1012300000E0071000D0071000C0071000B0070F33
:1012400000A107100091070E0083070F0074070F1D
:101250000065070E0057070E0049070E003B070DFB
:10126000002E070E0020070D0013070D0006070DC6
:1012700000F9060C00ED060D00E0060C00D4060C8B
:1012800000C8060C00BC060C00B0060C00A4060B3F
:101290000099060C008D060B0082060B0077060BEA
:1012A000006C060B0061060A0057060B004C060A8C
:1012B0000042060A0038060A002E060A0024060A22
:1012C000001A060A001006090007060A00FD0509B3
:1012D00000F4050900EB050900E2050900D905093C
:1012E00000D0050900C7050900BE050900B50508BD
:1012F00000AD050800A50509009C05080094050837
:10130000008C050800840508007C050800740508A9
:10131000006C050700650508005D05070056050817
:10132000004E05070047050700400508003805077F
:1013300000310507002A050700230507001C0506E4
:1013400000160507000F050700080506000205073F
:1013500000FB040600F5040700EE040600E804069E
:1013600000E2040700DB040600D5040600CF0406F3
:1013700000C9040600C3040600BD040600B7040645
:1013800000B1040500AC040600A6040600A0040594
:10139000009B04060095040500900406008A0405DD
:1013A0000085040500800406007A04050075040524
:1013B00000700405006B0405006604050061040567
:1013C000005C04050057040500520405004D0405A7
:1013D0000048040500430405003E0404003A0405E7
:1013E0000035040500300404002C04050027040423
:1013F00000230405001E0404001A0404001604055A
:1014000000110404000D0404000904050004040490
:101410000000040400FC030400F8030400F40304C7
:1014200000F0030400EC030400E8030400E40304F8
:1014300000E0030400DC030400D8030400D4030428
:1014400000D0030400CC030400C8030300C5030359
:101450000024F404D9201BC40C5C0E9804C4095F5A
:101460000265077101F405F900FB04B30048048725
:1014700000C10369005803550003034500BE023A4A
:10148000008402310053022A0029022500040220B0
:1014900000E4011C00C8011900AF011700980114F5
:1014A0000084011300710110006101100051010E50
:1014B0000043010D0036010B002B010B0020010B36
:1014C00000150109000C01090003010800FB0008D8
:1014D00000F3000800EB000700E4000600DE000651
:1014E00000D8000600D2000600CC000500C70005A9
:1014F00000C2000500BD000400B9000400B50004EE
:1015000000B1000400AD000400A9000400A5000320
:1015100000A20003009F0004009B0003009800034A
:10152000009500020093000300900003008D00026C
:10153000008B000300880002008600020084000384
:1015400000810002007F0002007D0002007B00029B
:1015500000790002007700010076000200740002AA
:101560000072000100710002006F0002006D0001B6
:10157000006C0002006A00010069000200670001BF
:1015800000660001006500010064000200620001C5
:101590000061000100600001005F0002005D0001C9
:1015A000005C0001005B0001005A000100590001CD
:1015B00000580001005700010056000100550001CD
:1015C00000540001005300000053000100520001CC
:1015D0000051000100500001004F0001004E0000CA
:1015E000004E0001004D0001004C0001004B0000C6
:1015F000004B0001004A00010049000100480000C2
:1016000000480001004700010046000000460001BC
:1016100000450000004500010044000100430000B7
:1016200000430001004200000042000100410000B0
:101630000041000100400001003F0000003F0001A8
:10164000003E0000003E0001003D0000003D0001A2
:10165000003C0000003C0000003C0001003B00009A
:10166000003B0001003A0000003A00010039000090
:101670000039000100380000003800000038000187
:10168000003700000037000100360000003600007F
:101690000036000100350000003500000035000173
:1016A000003400000034000000340001003300006A
:1016B000003300000033000100320000003200005F
:1016C0000032000100310000003100000031000153
:1016D000003000000030000000300001002F00004A
:1016E000002F0000002F0000002F0001002E00003E
:1016F000002E0000002E0001002D0000002D000033
:10170000002D0000002D0001002C0000002C000026
:10171000002C0000002C0001002B0000002B00001A
:10172000002B0000002B0001002A0000002A00000E
:10173000002A0000002A0001002900000029000002
:1017400000290000002900000029000100280000F5
:1017500000280000002800000028000000280001E8
:1017600000270000002700000027000000270000DD
:1017700000270001002600000026000000260000CF
:1017800000260000002600010025000000250000C2
:1017900000250000002500000025000000250001B4
:1017A00000240000002400000024000000240000A9
:1017B000002400010023000000230000002300009B
:1017C000002300000023000000230000002300018C
:1017D0000022000000220000002200000022000081
:1017E0000022000000220001002100000021000072
:1017F0000021000000210000002100000021000065
:101800000021000100200000002000000020000056
:101810000020000000200000002000000020000048
:1018200000200001001F0000001F0000001F00003A
:10183000001F0000001F0000001F0000001F00012B
:10184000001E0000001E0000001E0000001E000020
:10185000004D383420582059205A204500457272D6
:101860003A204D494E54454D5020424544004D4983
:101870004E54454D50207472696767657265640007
:101880004572723A204D494E54454D502045310025
:101890004572723A204D494E54454D502045300016
:1018A0004572723A204D415854454D5020424544AE
:1018B000004D415854454D502074726967676572F8
:1018C0006564004572723A204D415854454D502090
:1018D0004531004572723A204D415854454D5020D3
:1018E000453000024D6F7665206178697300446968
:1018F0007361626C65207374657070657273004DFE
:10190000383400426564204C6576656C696E67000A
:101910004732382058590A4D313039205331373544
:101920000A473238205A0A4D313039205231343585
:101930000A4731320A4732390A4D313034205330A8
:10194000004175746F20686F6D6500473238004D37
:1019500061696E005072696E7420706175736564A0
:10196000004D3132350025753A253032750025306D
:1019700032753A2530327500257564202530327570
:101980003A253032750000060900FE000000000014
:1019900001090008FE000005080806000040F0C824
:1019A0008888987810050808060000C0F88888889C
:1019B0008888F80505050600012030F83020050864
:1019C000080600002070F820202020E00509090604
:1019D00000FF2070A8A8B8888870200509090600B3
:1019E000FFE080C0B0A8283028280509090600FFBC
:1019F000F8A88888888888A8F8050A0A0600FE20C2
:101A00005050505088A8A888700303030600034074
:101A1000A04000060900FE070192032120FFFF08F5
:101A2000FF07FF0000000600000107070602008014
:101A3000808080800080030202060105A0A00507C7
:101A4000070600005050F850F850500507070600F0
:101A5000002078A07028F020050707060000C0C805
:101A600010204098180507070600006090A040A8C5
:101A70009068020303060104C040800307070601C3
:101A8000002040808080402003070706010080403E
:101A9000202020408005050506000120A870A82010
:101AA0000505050600012020F82020020303060298
:101AB000FFC04080050101060003F8020202060291
:101AC00000C0C0050505060001081020408005077C
:101AD0000706000070888888888870030707060159
:101AE0000040C040404040E0050707060000708805
:101AF00008708080F8050707060000F8102010081D
:101B000008F005070706000010305090F810100587
:101B10000707060000F880F0080888700507070628
:101B20000000708080F0888870050707060000F8C4
:101B30000810202020200507070600007088887004
:101B40008888700507070600007088887808087084
:101B5000020505060200C0C000C0C002060606025B
:101B6000FFC0C000C04080040707060000102040EE
:101B700080402010050303060002F800F804070760
:101B80000601008040201020408005070706000065
:101B900070880810200020050707060000708808DC
:101BA00068A8A870050707060000708888F888886C
:101BB00088050707060000F08888F08888F0050788
:101BC000070600007088808080887005070706007F
:101BD00000F08888888888F0050707060000F880EC
:101BE00080F08080F8050707060000F88080F0800C
:101BF0008080050707060000708880B88888700517
:101C00000707060000888888F88888880107070683
:101C100002008080808080808005070706000038F1
:101C20001010101090600507070600008890A0C0F3
:101C3000A09088050707060000808080808080F8DB
:101C400005070706000088D8A88888888805070740
:101C50000600008888C8A89888880507070600003D
:101C600070888888888870050707060000F08888D3
:101C7000F080808005070706000070888888A8909B
:101C800068050707060000F08888F0A0908805071F
:101C900007060000788080700808F0050707060036
:101CA00000F8202020202020050707060000888853
:101CB00088888888700507070600008888888888D3
:101CC00050200507070600008888888888A85005E6
:101CD00007070600008888502050888805070706F7
:101CE000000088888850202020050707060000F89B
:101CF0000810204080F8030707060100E08080807C
:101D00008080E005050506000180402010080307DB
:101D100007060100E02020202020E0050303060044
:101D200004205088050101060000F80202020602A4
:101D300005804005050506000070087888780507CD
:101D4000070600008080B0C88888F00505050600F9
:101D500000708080887005070706000008086898F2
:101D60008888780505050600007088F880700507EA
:101D7000070600003048E0404040400506060600E7
:101D8000FF7088887808700507070600008080B01B
:101D9000C88888880107070602008000808080804C
:101DA000800308080601FF200020202020A0400416
:101DB0000707060000808090A0C0A09003070706D8
:101DC0000100C04040404040E0050505060000D04D
:101DD000A8A8A8A8050505060000B0C88888880539
:101DE000050506000070888888700506060600FF55
:101DF000F08888F080800506060600FF78888878DD
:101E00000808050505060000B0C8808080050505A6
:101E100006000070807008F00407070600004040CC
:101E2000E040404030050505060000888888986835
:101E30000505050600008888885020050505060070
:101E4000008888A8A8500505050600008850205085
:101E5000880506060600FF8888887808700505054D
:101E6000060000F8102040F8030707060100204094
:101E7000408040402001070706020080808080806B
:101E80008080030707060100804040204040800515
:101E90000202060002689000000006000000000038
:101EA0000600000000000600000000000600000020
:101EB0000000060000000000060000000000060010
:101EC0000000000006000000000006000000000006
:101ED00006000000000006000000000006000000F0
:101EE00000000600000000000600000000000600E0
:101EF00000000000060000000000060000000000D6
:101F000006000000000006000000000006000000BF
:101F100000000600000000000600000000000600AF
:101F200000000000060000000000060000000000A5
:101F3000060000000000060000000000060000008F
:101F4000000006000000000006000000000006007F
:101F50000000000006000000000006000000000075
:101F60000600000107070602008000808080808054
:101F70000507070600002070A8A0A8702005070725
:101F8000060000304040E04050A80505050600006E
:101F90008870507088050707060000885020F820D8
:101FA000F8200107070602008080800080808005FD
:101FB00008080600003048205050209060030101BE
:101FC000060107A0050707060000F888B8B8B8881A
:101FD000F8050707060001700878887800F80505FD
:101FE000050600012850A05028050303060001F84B
:101FF00008080202020602064080050707060000E4
:10200000F888A88898A8F8050101060006F80404D5
:10201000040600036090906005070706000020207A
:10202000F8202000F804050506000360902040F029
:10203000030505060003E020E020E002020206029C
:102040000640800508080600FF8888888898E88090
:10205000800507070600007898987818181802027B
:1020600002060202C0C00202020602FF408003050F
:102070000506000340C04040E00507070600017068
:102080008888887000F8050505060001A0502850D2
:10209000A00507070600008890A858B8080805079B
:1020A000070600008890B848982038050808060000
:1020B00000C040C048D838080805070706000020BF
:1020C000002040808870050808060000402000704D
:1020D00088F888880508080600001020007088F835
:1020E00088880508080600002050007088F8888855
:1020F0000508080600006890007088F888880508C0
:10210000080600005000708888F8888805080806CE
:1021100000002050207088F8888805070706000016
:102120003860A0B8E0A0B80508080600FF708880F5
:102130008088702060050808060000402000F880B4
:10214000F080F8050808060000081000F880F0800C
:10215000F8050808060000205000F880F080F80517
:1021600007070600005000F880F080F80308080612
:102170000100804000E0404040E003080806010004
:10218000204000E0404040E003080806010040A075
:1021900000E0404040E0030707060100A000E040E7
:1021A0004040E0050707060000704848E8484870CE
:1021B00005080806000068900088C8A898880508E7
:1021C0000806000040207088888888700508080686
:1021D00000001020708888888870050808060000B4
:1021E00020500070888888700508080600006890F4
:1021F0000070888888700508080600005000708804
:1022000088888870050505060001885020508805DB
:1022100008080600FF1070A8A8A8A87040050808C4
:102220000600004020888888888870050808060015
:10223000001020888888888870050808060000201B
:1022400050008888888870050808060000500088BB
:1022500088888888700508080600001020885020AB
:102260002020200509090600FFC040704848704042
:1022700040E00408080601FF609090A09090E08084
:1022800005080806000040200070087888780508D6
:1022900008060000102000700878887805080806F5
:1022A00000002050007008788878050808060000B3
:1022B00068900070087888780507070600005000CD
:1022C00070087888780508080600002050207008FB
:1022D000788878050606060000D02878A0A8500562
:1022E00006060600FF70808870206005080806005A
:1022F000004020007088F880700508080600001073
:1023000020007088F8807005080806000020500042
:102310007088F8807005070706000050007088F884
:10232000807003080806010080400040C04040E083
:1023300003080806010020400040C04040E00308B8
:102340000806010040A00040C04040E00307070627
:102350000100A00040C04040E0050707060000A0C3
:1023600040A010788870050808060000689000B04A
:10237000C888888805080806000040200070888802
:102380008870050808060000102000708888887092
:10239000050808060000205000708888887005082D
:1023A0000806000068900070888888700507070696
:1023B000000050007088888870050505060001201F
:1023C00000F800200507070600FF1070A8A8A870F5
:1023D00040050808060000402000888888986805A5
:1023E00008080600001020008888889868050808FA
:1023F00006000020500088888898680507070600B6
:1024000000500088888898680509090600FF102098
:1024100000888888F808700407070601FFC040603C
:10242000506040E00508080600FF50008888887862
:1024300008705A00590058000920000000000000F0
:10244000000000000000007FFFE00000000000002E
:102450000000000000007000E0000000000000002C
:10246000000000000061F8600000000000000000B3
:102470000000000041F82000000000000000000003
:1024800000000040F02000000000000000000000FC
:10249000000040602000000000000000000000007C
:1024A000005801A07F80003FC000000000410400F0
:1024B0005C63A0FBC00079E0000000002082005EA9
:1024C000F7A0F3C00076E0000000002082005EF775
:1024D000A0EBC0007EE0000000004104005C63A0AF
:1024E0007B80003DC0000000008208005801A07BF6
:1024F00080003BC000000001041000406020FBC0D1
:102500000077E00000000104100040F020FBC00054
:1025100070E00000000082080041F820FFC0007F4A
:10252000E00000000041040061F8603F00001F80EF
:10253000000000000000007000E01E00000F00001E
:10254000000001FFFF807FFFE00C0000060000009C
:102550000001FFFF800000000000000000000000FC
:10256000000000007FFFE00000000000000000000D
:102570000000007000E0000000000000000000000B
:102580000000630C6000000000000000000000007C
:1025900000470E20000000000000000000000000C6
:1025A0004F0F200000000000000000000000005F4E
:1025B0000FA00000000000000000000000005E0707
:1025C000A07F80003FC00000000041040040602068
:1025D000FBC00079E00000000020820040F020F302
:1025E000C00076E00000000020820040F020EBC038
:1025F000007EE0000000004104004060207B80007D
:102600003DC0000000008208005E07A07B80003B08
:10261000C0000000010410005F0FA0FBC00077E0C5
:10262000000000010410004F0F20FBC00070E0000C
:10263000000000820800470E20FFC0007FE000007D
:102640000000410400630C603F00001F8000000098
:10265000000000007000E01E00000F0000000001FC
:10266000FFFF807FFFE00C0000060000000001FF7C
:10267000FF8000000043616E6E6F74206F70656EA6
:10268000207375626469722000456E642066696C0F
:1026900065206C6973740A00426567696E2066691B
:1026A0006C65206C6973740A0046696C652064650A
:1026B0006C657465643A0044656C6574696F6E207E
:1026C0006661696C65642C2046696C653A20006F10
:1026D00070656E206661696C65642C2046696C6566
:1026E0003A200001050800FF060121023520FFFF06
:1026F00007FF06FF09005022165680808080008068
:10270000153353A0A0A00257575050F850F850501E
:102710000257572070A07028702013355580A040B4
:10272000A02002475740A0A040A0A05025135380EE
:10273000808012265640808080804012265680403D
:10274000404040800245559060F060900255552011
:1027500020F82020113353604080044151F01133A0
:102760005340E040024656101020408080123656FA
:1027700040A0A0A0A04012365640C0404040E00219
:1027800046566090106080F0024656F0206010902F
:10279000600246562060A0F02020024656F080E0FD
:1027A0001090600246566080E0909060024656F0BD
:1027B0001020204040024656609060909060024693
:1027C00056609090701060122555C0C000C0C011B6
:1027D000365660600060408012365620408080404F
:1027E00020034353F000F0123656804020204080F2
:1027F00012365640A020400040015858304898A852
:10280000A8904030024656609090F0909002465654
:10281000E090E09090E002465660908080906002E8
:102820004656E090909090E0024656F080E080801E
:10283000F0024656F080E08080800246566090802C
:10284000B090600246569090F0909090123656E00C
:1028500040404040E002465670202020A040024602
:102860005690A0C0A0A0900246568080808080F044
:1028700002465690F0F090909002465690D0F0B0FC
:10288000B090024656609090909060024656E0905C
:1028900090E08080014757609090D0B06010024671
:1028A00056E09090E09090024656609040209060F4
:1028B000123656E04040404040024656909090907C
:1028C00090600246569090909060600246569090BC
:1028D00090F0F090024656909060609090025656AC
:1028E000888850202020024656F010204080F012A8
:1028F0003656E080808080E002465680804020107E
:1029000010123656E020202020E016325240A0015E
:102910004151F0162252804002445470909070024F
:1029200046568080E09090E01234546080806002CF
:10293000465610107090907002445460B0C060020F
:102940004656205040E04040014555609070106070
:102950000246568080E09090901236564000C0406B
:1029600040E01137572000202020A040024656802A
:102970008090E09090123656C040404040E00254B3
:1029800054D0A8A8A8024454E09090900244546007
:10299000909060014555E090E08080014555709031
:1029A000701010024454A0D0808012345460C020B3
:1029B000C00246564040E04050200244549090905F
:1029C00070123454A0A0A04002545488A8A8500209
:1029D000445490606090014555909070906002441E
:1029E00054F02040F0024757304020C020403022B1
:1029F0001656808080808080024757C0204030403B
:102A000020C006425250A0FFFFFFFFFFFFFFFFFF65
:102A1000FFFFFFFFFFFFFFFFFFFFFFFFFFFFFFFFC6
:102A2000FFFFFFFFFFFFFFFF090050221656800047
:102A3000808080800146562070A0A07020024656FB
:102A40002050E04050A002555588705070880256C2
:102A5000568850F820F82022175780808000808008
:102A6000800247577080E0907010E0173151A0024B
:102A7000565670A8C8C8A87014355560A06000E00C
:102A800003435350A050123353E02020143151E03F
:102A900002565670E8D8E8D870173151E015335314
:102AA00040A04012355540E04000E014355540A0AC
:102AB0002040E0143555C020C020C016225240806E
:102AC000014555909090E08002565678E8E86828D5
:102AD0002824115180112252408014355540C040A5
:102AE00040E014355540A04000E0034353A050A0FF
:102AF000024757808080A060F0200247578080A066
:102B0000D010207002475780408060A0F02012361D
:102B10005640004080A04002475740206090F0900F
:102B20009002475720406090F09090024757609085
:102B30006090F0909002475750A06090F090900203
:102B4000475790006090F0909002475760906090D7
:102B5000F0909002465670A0A0F0A0B001475760D8
:102B60009080809060400247574020F080E080F0E5
:102B70000247572040F080E080F00247576090F015
:102B800080E080F00247579000F080E080F012373C
:102B9000578040E0404040E01237572040E040403E
:102BA00040E012375740A0E0404040E0123757A0C5
:102BB00000E0404040E00256567048E84848700245
:102BC000475750A090D0B090900247574020609057
:102BD0009090600247572040609090906002475765
:102BE0006090609090906002475750A060909090E5
:102BF0006002475790006090909060123353A0405D
:102C0000A002465670B0B0D0D0E0024757402090A6
:102C100090909060024757204090909090600247BB
:102C200057609090909090600247579000909090DD
:102C3000906002575710208850202020024656806E
:102C4000E09090E0800246566090A0A090A00247DD
:102C500057402000709090700247572040007090BD
:102C60009070024757205000709090700247575064
:102C7000A0007090907002465650007090907002C4
:102C8000475760906070909070025454F068B0782C
:102C9000113555608080604002475740200060B089
:102CA000C06002475720400060B0C06002475760D4
:102CB000900060B0C060024656500060B0C0601224
:102CC0003757804000C04040E0123757204000C0D6
:102CD0004040E012375740A000C04040E012365656
:102CE000A000C04040E0024757A040A01070906094
:102CF00002475750A000E0909090024757402000B4
:102D000060909060024757204000609090600247BA
:102D1000576090006090906002475750A00060900C
:102D200090600246569000609090601235554000C9
:102D3000E0004002445470B0D0E002475740200009
:102D400090909070024757204000909090700247FA
:102D5000576090009090907002465690009090902E
:102D60007001485820400090907090600147578053
:102D700080E090E0808001475790009090709060D4
:102D800001050700FE0500FB01F220FFFE05FE0520
:102D9000FE0200400215258080800080053242A09E
:102DA000A002556550F850F8500146562070C030CA
:102DB000E02002556590102040480255656080680B
:102DC0009068051222808002253540808080400274
:102DD00025358040404080043343A040A003334366
:102DE00040E0400122324080043141E00211218064
:102DF0000255650810204080024555609090906013
:102E0000022535C040404040024555E0106080F04A
:102E1000024555E0106010E00245552060A0F0200A
:102E2000024555F080E010E00245556080E090607A
:102E3000024555F01020404002455560906090607A
:102E400002455560907010600313238000800214C7
:102E50002480008080023545204080402003334399
:102E6000E000E00235458040204080024555E010FA
:102E70006000400255657088B8A8700245556090A2
:102E800090F090024555E090E090E002354560807A
:102E9000808060024555E0909090E0023545E080EA
:102EA000E080E0023545E080E0808002455570809A
:102EB000B090700245559090F09090023545E040FA
:102EC0004040E0024555301010906002455590A0FA
:102ED000C0A09002354580808080E002556588D88A
:102EE000A8888802455590D0B090900245556090D2
:102EF000909060024555E09090E0800146566090C9
:102F000090906010024555E09090E0900245557019
:102F1000806010E0023545E0404040400245559059
:102F2000909090600245559090A0A0400255658811
:102F3000A8A8A850024555909060909002455590E1
:102F400090701060023545E0204080E0022535C0D9
:102F5000808080C00255658040201008022535C061
:102F6000404040C005324240A0024151F0052232AB
:102F700080400244547090907002455580E09090DB
:102F8000E00234446080806002455510709090707B
:102F900002445460B0C0600235452040E04040002B
:102FA000465670909070106002455580E090909069
:102FB0000215258000808080002737400040404077
:102FC00040800245558090A0E090021525808080C9
:102FD0008080025464F0A8A8A8024454E090909025
:102FE00002445460909060004656E09090E08080EB
:102FF000004656709090701010023444A0C080803B
:1030000002445470C030E002354540E040402002A8
:103010004454909090700244549090A040025464A4
:10302000A8A85050023444A04040A00046569090BA
:1030300090701060024454F02040F002354560402A
:103040008040600215258080808080023545C04028
:103050002040C005425250A0FFFFFFFFFFFFFFFFCF
:10306000FFFFFFFFFFFFFFFFFFFFFFFFFFFFFFFF70
:10307000FFFFFFFFFFFFFFFFFF020040FFFFFFFF1B
:10308000FFFFFFFFFFFFFFFFFFFFFFFFFFFFFFFF50
:10309000FFFFFFFFFFFFFFFFFFFFFFFFFFFFFFFF40
:1030A000FFFFFFFFFFFFFFFFFFFFFFFFFFFFFFFF30
:1030B000FFFFFFFFFFFFFFFFFFFFFFFFFFFFFFFF20
:1030C000FFFFFFFFFFFFFFFFFFFFFFFFFFFFFFFF10
:1030D000FFFFFFFFFFFFFFFFFFFFFF01060D00FEE9
:1030E00009016602D620FFFE0BFE0AFE0D006022DB
:1030F0001969808080808080800080183363A0A060
:10310000A00357675050F850F85050025969207882
:10311000A0A0702828F02002596948A8501020402B
:1031200050A89002586840A0A040A098906828132A
:1031300063808080113B6B20404080808080804095
:103140004020113B6B8040402020202020404080C8
:1031500006556520A870A8200455652020F8202079
:10316000113363604080065161F811336340E040E1
:1031700002596908081010204040808002596920D7
:1031800050888888888850200259692060A02020B3
:10319000202020F80259697088880810204080F8A3
:1031A000025969F8081020700808887002596910DF
:1031B0001030505090F81010025969F88080B0C853
:1031C0000808887002596970888080F08888887043
:1031D000025969F8081010202040404002596970D7
:1031E000888888708888887002596970888888788B
:1031F0000808887011386840E040000040E0401145
:10320000386840E0400000604080025969081020A2
:10321000408040201008045464F80000F802596906
:10322000804020100810204080025969708888086A
:10323000102020002002596970888898A8A8B080C2
:10324000780259692050888888F8888888025969E6
:10325000F048484870484848F002596970888080B2
:103260008080808870025969F0484848484848483A
:10327000F0025969F8808080F0808080F8025969F6
:10328000F8808080F080808080025969708880801A
:10329000809888887002596988888888F888888822
:1032A00088123969E040404040404040E00259699E
:1032B000381010101010109060025969888890A082
:1032C000C0A090888802596980808080808080803A
:1032D000F80259698888D8A8A88888888802596916
:1032E00088C8C8A8A898988888025969708888886A
:1032F0008888888870025969F0888888F080808082
:1033000080015A6A70888888888888A8700802595D
:1033100069F0888888F0A090888802596970888050
:10332000807008088870025969F820202020202029
:10333000202002596988888888888888887002597E
:103340006988888888505050202002596988888868
:1033500088A8A8A8A85002596988885050205050C1
:1033600088880259698888505020202020200259DE
:1033700069F808101020404080F8113B6BE0808015
:1033800080808080808080E0025969808040402079
:1033900010100808113B6BE0202020202020202066
:1033A00020E0085363205088015161F82A2262808E
:1033B0004002566670087888986802596980808053
:1033C000F088888888F0025666708880808870024D
:1033D000596908080878888888887802566670884D
:1033E000F880887002596930484040F040404040C1
:1033F00000586870888888780888700259698080C9
:1034000080B0C8888888881238684000C040404032
:1034100040E0004A6A1000301010101090906002D6
:10342000596980808090A0C0A09088123969C040FE
:10343000404040404040E0025666D0A8A8A8A88876
:10344000025666B0C8888888880256667088888860
:103450008870005868F0888888F0808080005868FC
:103460007888888878080808025666B0C880808006
:10347000800256667088601088700258684040F07C
:1034800040404048300256668888888898680256CE
:10349000668888885050200256668888A8A8A85058
:1034A000025666885020205088005868888888987E
:1034B00068088870025666F810204080F8015B6B3F
:1034C0001820202020C02020202018221969808068
:1034D00080808080808080015B6BC020202020184D
:1034E00020202020C008536348A890FFFFFFFFFF63
:1034F000FFFFFFFFFFFFFFFFFFFFFFFFFFFFFFFFDC
:10350000FFFFFFFFFFFFFFFFFFFFFFFF0D00602238
:1035100019698000808080808080800358682070D6
:10352000A8A0A0A8702002596930484040E040405F
:1035300048B0035666887050507088025969888870
:103540005050F820F8202022196980808080008067
:10355000808080124A6A60908060909060109060D5
:103560001A3262A0A00359697088A8D8C8D8A88860
:1035700070045767700878887800F80356662850FA
:10358000A0A05028045363F80808163161E00359DD
:10359000697088E8D8D8E8D888700A5161F817446B
:1035A00064609090600357672020F8202000F8079F
:1035B000356540A02040E007356540A04020C02A86
:1035C000226240800058688888888898E880800255
:1035D000596978E8E8E8E868282828262161C020A9
:1035E0002262408007356540C04040E00457677064
:1035F0008888887000F8035666A050282850A002DA
:103600005A6A40C04040E00818283808025A6A4008
:10361000C04040E01028081038025A6A40A04020FC
:10362000A0481828380802596920002020408088C6
:103630008870025A6A40200020508888F8888802E2
:103640005A6A10200020508888F88888025A6A3008
:10365000480020508888F88888025A6A285000203C
:10366000508888F88888025A6A505000205088880C
:10367000F88888025A6A20502020508888F8888864
:1036800002596958A0A0A0B0E0A0A0B8005B6B7080
:1036900088808080808088702040025A6A402000A4
:1036A000F88080F08080F8025A6A102000F880804C
:1036B000F08080F8025A6A304800F88080F08080FC
:1036C000F8025A6A505000F88080F08080F8123A70
:1036D0006A804000E04040404040E0123A6A2040AA
:1036E00000E04040404040E0124A6A609000E04004
:1036F00040404040E0123A6AA0A000E04040404014
:1037000040E0025969F0484848E8484848F0025A01
:103710006A2850008888C8A8988888025A6A402079
:103720000070888888888870025A6A102000708823
:103730008888888870025A6A30480070888888882B
:103740008870025A6A2850007088888888887002B9
:103750005A6A505000708888888888700355658838
:1037600050205088015B6B08709898A8A8A8C8C81A
:103770007080025A6A402000888888888888700291
:103780005A6A10200088888888888870025A6A30AF
:10379000480088888888888870025A6A5050008853
:1037A000888888888870025A6A102000888850208B
:1037B00020202002596980F0888888F0808080026B
:1037C0005969609090A0A0908888B0025969402003
:1037D000007008788898680259691020007008788D
:1037E000889868025969304800700878889868029B
:1037F00059692850007008788898680259695050B3
:1038000000700878889868025A6A3048300070085A
:1038100078889868025666702870A0A8500058688A
:10382000708880808870204002596940200070882C
:10383000F88088700259691020007088F8808870BC
:103840000259693048007088F880887002596950C0
:1038500050007088F8808870123969804000C0403C
:10386000404040E0123969204000C040404040E004
:10387000124969609000C040404040E0123969A0A0
:10388000A000C040404040E0025A6A5020601070E2
:103890008888888870025969285000B0C88888884C
:1038A00088025969402000708888888870025969A8
:1038B000102000708888888870025969304800702C
:1038C000888888887002596928500070888888889C
:1038D0007002596950500070888888887003576753
:1038E000202000F8002020015868087098A8A8C877
:1038F0007080025969402000888888889868025939
:1039000069102000888888889868025969304800C2
:103910008888888898680259695050008888888803
:103920009868005B6B102000888888986808887009
:10393000005A6A8080B0C88888C8B08080005B6BFD
:10394000505000888888986808887000000000003F
:103950000000000000000000000000000000000067
:1039600000000000000000000000000000000C004B
:103970000000000000000C00000000000000120029
:1039800000000000000023000000000000002100F3
:103990000000000000004C800000000000005E807D
:1039A0000000000000009240000000000000A14064
:1039B00000000000000121200000000000027F90B4
:1039C0000000000000020010000000000007FFF8E7
:1039D00000000000000400080000000000080004CF
:1039E00000000000000800060000000000100002B7
:1039F0000000000000301E010000000000207F8158
:103A0000000000000041FFE0800000000043FCF0E7
:103A10008000000000873B7840000000018EDBFC46
:103A200060000000010FEBCC20000000021FEDB68B
:103A300010000000021FDEB6100000000439CD7F28
:103A4000080000000436E0FF08000000087EC0BB4C
:103A500084000000187F005D86000000107FC0ED2C
:103A600082000000203CC07301000000203B337F37
:103A700001000000701BE77E03800000C81DEEDE21
:103A800004C00000880FDEDC04400001240FDF3C8E
:103A9000092000012607DBF8192000027203E7F075
:103AA000139000025101FFE02290000489007F8002
:103AB0002448000904801E004824000BFE4000003A
:103AC000DFF40010004000008002001FFFFFFFFF36
:103AD000FFFE0000000000000000000000000000E9
:103AE00000000000000000000000001022103C3C1C
:103AF0000E1F0010221004221104001022100822B0
:103B0000110400102210083C110400102210102291
:103B100011040010221020221104001E1C1E3C3C27
:103B20000E04000000000000000000000000000083
:103B30000000000000000000000000000000000085
:103B40000000000000000000000000000000000075
:103B50000000000000000000000000000000000065
:103B60000000000000000000000000000000000055
:103B70000000000000000000000000000000000045
:103B80000000000000000000002040002042403AF9
:103B90000020403A006F6B004D6F766520302E316B
:103BA0006D6D004D6F766520316D6D004D6F7665E2
:103BB0002031306D6D004D6F76652061786973003E
:103BC0004578747275646572004D6F7665205A0091
:103BD0004D6F76652059004D6F7665205800746FE3
:103BE00020726573756D65005761697420666F7228
:103BF000207072696E74005052494E5420504155E5
:103C00005345440045787472756465206D6F726524
:103C100000526573756D65207072696E740052454F
:103C200053554D45204F5054494F4E533A00202094
:103C30004E6F7A7A6C653A20002000506C65617393
:103C40006520776169742E2E2E0048656174696E57
:103C500067206E6F7A7A6C65005052494E5420503E
:103C600041555345440020204E6F7A7A6C653A20C6
:103C700000200068656174206E6F7A7A6C652E0092
:103C8000507265737320627574746F6E20746F0068
:103C90005052494E54205041555345440020204E27
:103CA0006F7A7A6C653A2000200066696C616D65F8
:103CB0006E7420657874727564650057616974204C
:103CC000666F72005052494E54205041555345443E
:103CD0000020204E6F7A7A6C653A200020006669D9
:103CE0006C616D656E74206C6F61640057616974FE
:103CF00020666F72005052494E5420504155534532
:103D0000440020204E6F7A7A6C653A2000746F2050
:103D1000636F6E74696E75652E2E2E00616E642061
:103D2000707265737320627574746F6E00496E7380
:103D30006572742066696C616D656E7400505249DD
:103D40004E54205041555345440020204E6F7A7AFE
:103D50006C653A2000200066696C616D656E7420A8
:103D6000756E6C6F6164005761697420666F7200D4
:103D70005052494E54205041555345440020204E46
:103D80006F7A7A6C653A20006368616E6765006FD0
:103D900066207468652066696C616D656E74005795
:103DA00061697420666F722073746172740050527E
:103DB000494E54205041555345440020204E6F7ABF
:103DC0007A6C653A200020004261636B004D696E99
:103DD000696D756D2054656D7020697320313230C6
:103DE0002E0048656174696E67206661696C656460
:103DF000005265776970696E670050726F62696E14
:103E000067206661696C65640050726F62696E67F5
:103E1000206661696C65640050524F4245204641FE
:103E2000494C20434C45414E204E4F5A5A4C450A6E
:103E3000005265776970696E670A0052657769702C
:103E4000696E670050726F62696E67206661696CA7
:103E500065640050726F62696E67206661696C65A7
:103E6000640050524F4245204641494C20434C4546
:103E7000414E204E4F5A5A4C450A005265776970A0
:103E8000696E670A0050726F62696E6720666169C9
:103E90006C65640A0050726F62696E6720666169C2
:103EA0006C656400205A3A200020593A200042658F
:103EB0006420583A20000A0A426564204C65766501
:103EC0006C20436F7272656374696F6E204D61740C
:103ED0007269783A00202B000A436F72726563742E
:103EE000656420426564204865696768742076735C
:103EF0002E2042656420546F706F6C6F67793A0AA8
:103F000000202B000A4265642048656967687420B8
:103F1000546F706F6772617068793A0A2020202BA5
:103F20002D2D2D204241434B202D2D2B0A202020CA
:103F30007C20202020202020202020207C0A204CB3
:103F4000207C20202020282B29202020207C20526B
:103F50000A2045207C2020202020202020202020F6
:103F60007C20490A2046207C20282D29204E20280C
:103F70002B29207C20470A2054207C202020202030
:103F80002020202020207C20480A2020207C202067
:103F90002020282D29202020207C20540A20202089
:103FA0007C20202020202020202020207C0A20206F
:103FB000204F2D2D2046524F4E54202D2D2B0A20C0
:103FC00028302C30290A004D65616E206F66207301
:103FD000616D706C656420706F696E74733A200057
:103FE00020643A200020623A200045716E20636F01
:103FF000656666696369656E74733A20613A20008C
:1040000052756E6E696E6720696E204452592D524A
:10401000554E206D6F64650A004732392041757432
:104020006F20426564204C6576656C696E670A0096
:1040300028422961636B00284629726F6E7400283C
:1040400052296967687400284C29656674003F4EE0
:10405000756D626572206F662070726F6265207088
:104060006F696E747320697320696D706C6175730C
:1040700069626C65202832206D696E696D756D29E5
:104080002E0A003F2856296572626F7365206C65A1
:1040900076656C20697320696D706C6175736962F7
:1040A0006C652028302D34292E0A0043617264206B
:1040B00072656D6F766564004361726420696E732A
:1040C00065727465640048617264636F646564203E
:1040D00044656661756C742053657474696E6773AA
:1040E000204C6F616465640A0028230000282300C7
:1040F00000640000001027000000009643000096B6
:1041000043000040400000C8410000C9420000C90F
:10411000420000C84400804F4400804F4420286380
:10412000616C63756C6174656429210A0020213D0E
:104130002000454550524F4D20435243206D697336
:104140006D61746368202D202873746F7265642913
:104150002000290A002062797465733B2063726332
:1041600020002073746F7265642073657474696EC7
:104170006773207265747269657665642028002013
:104180004D61726C696E3D563430290A00284545F0
:1041900050524F4D3D00454550524F4D207665726F
:1041A00073696F6E206D69736D61746368200000C0
:1041B000060900FE06018902FE20FFFE07FE06FE3C
:1041C00000000006000701060606020080808080CD
:1041D0000080030303060103A0A0A0050707060053
:1041E000FF5050F850F850500509090600FE2070A5
:1041F000A8A07028A870200608080600FF40A8485C
:1042000010204854080507070600FF60909060984A
:1042100090680103030602038080800207070602FC
:10422000FF408080808080400207070602FF8040B8
:1042300040404040800505050600008850F8508841
:104240000505050600002020F820200204040602CF
:10425000FEC0404080050101060002F8020202068D
:104260000200C0C004060606010010102040808035
:104270000406060601006090909090600306060612
:10428000010040C0404040E0040606060100609086
:10429000102040F0040606060100F020601010E037
:1042A00005060606000010305090F81004060606B9
:1042B0000100F080E01010E00406060601006080B6
:1042C000E0909060040606060100F01010204040C7
:1042D00004060606010060906090906004060606E1
:1042E0000100609090701060020505060200C0C0D9
:1042F00000C0C00207070602FEC0C000C0404080E8
:104300000505050600001860806018050303060017
:1043100001F800F8050505060000C0300830C004AB
:104320000707060100609010604000400506060681
:1043300000007090A8B080700506060600002050AE
:1043400088F88888050606060000F088F08888F05E
:104350000406060601006090808090600406060650
:104360000100E090909090E0040606060100F080C5
:10437000E08080F0040606060100F080E080808086
:10438000040606060100609080B0906004060606F0
:1043900001009090F0909090030606060100E04026
:1043A000404040E0050606060000381010109060FE
:1043B00004060606010090A0C0A090900406060620
:1043C00001008080808080F005060606000088D805
:1043D000A8A8888804060606010090D0B0909090A6
:1043E00005060606000070888888887004060606A0
:1043F0000100E09090E080800407070601FF6090D4
:1044000090D0B06010040606060100E09090E090A5
:1044100090040606060100609040209060050606A4
:10442000060000F820202020200406060601009047
:104430009090909060040606060100909090F060C5
:10444000600506060600008888A8A8D88805060624
:1044500006000088502020508805060606000088C7
:104460008850202020040606060100F0102040801D
:10447000F0030606060100E080808080E004060666
:10448000060100808040201010030606060100E0AF
:1044900020202020E00503030600032050880501AA
:1044A000010600FEF8020202060204804004040431
:1044B000060100709090700406060601008080E0FE
:1044C0009090E004040406010070808070040606E9
:1044D0000601001010709090700404040601006042
:1044E000B0C070040606060100205040E0404004C1
:1044F00006060601FE609090701060040606060134
:10450000008080E09090900306060601004000C005
:104510004040E00308080601FE200060202020A0A3
:10452000400406060601008080A0C0A09003060695
:10453000060100C040404040E0050404060000D0F1
:10454000A8A888040404060100E0909090040404E4
:10455000060100609090600406060601FEE090905F
:10456000E080800406060601FE7090907010100432
:104570000404060100A0D080800404040601007039
:10458000C030E00406060601004040E04050200430
:104590000404060100909090700404040601009049
:1045A00090606005040406000088A8A85004040474
:1045B000060100906060900406060601FE9090904F
:1045C000709060040404060100F02040F003070727
:1045D000060100204040804040200107070602FFFE
:1045E0008080808080808003070706010080404033
:1045F0002040408004020206010350A0FFFFFFFF9D
:10460000FFFFFFFFFFFFFFFFFFFFFFFFFFFFFFFFBA
:10461000FFFFFFFFFFFFFFFFFFFFFFFFFF000000A7
:1046200006000701060606020080008080808004E4
:1046300006060601FF2070A0A070200507070600EF
:10464000FF304840F04040F8050505060000A8503E
:104650008850A80506060600008850F820F82001BA
:1046600007070602FF80808000808080040707061D
:1046700001FF708060906010E0030101060105A059
:10468000060707060000788494A49484780305053F
:1046900006010160A06000E0050505060000285045
:1046A000A05028040303060100F0101004010106C5
:1046B0000102F00607070600007884B4A4A48478F9
:1046C000040101060105F004030306010260906085
:1046D0000507070600FF2020F8202000F803050545
:1046E00006010140A02040E0030505060101C020AD
:1046F0004020C002020206020440800405050601B3
:10470000FF9090B0D08005060606000078E8E868C3
:104710002828010101060202800202020602FE4070
:104720008003050506010140C04040E00305050681
:10473000010140A04000E0050505060000A050284A
:1047400050A00508080600FF40C0405070307810A7
:104750000508080600FF40C04050680810380508EA
:10476000080600FFC0204030F0307810040707062C
:1047700001002000206080906005070706000040CF
:104780002020507088880507070600001020205060
:104790007088880507070600002050205070888820
:1047A0000507070600002850205070888805070775
:1047B000060000500020507088880507070600009A
:1047C0002050205070888805060606000078A0F06A
:1047D000A0A0B80408080601FE60908080906020C8
:1047E000400407070601004020F080E080F0040745
:1047F000070601002040F080E080F0040707060172
:10480000002050F080E080F004070706010050000F
:10481000F080E080F00307070601008040E04040A0
:1048200040E00307070601002040E0404040E0036D
:10483000070706010040A0E0404040E003070706EC
:104840000100A000E0404040E005060606000070C0
:1048500048E848487004070706010050A090D0B00F
:10486000909004070706010040206090909060043B
:10487000070706010020406090909060040707063B
:1048800001002050609090906004070706010050DE
:10489000A0609090906004070706010050006090AF
:1048A0009090600505050600008850205088040897
:1048B000080601FF1070B0B0D0D0E08004070706F2
:1048C00001004020909090906004070706010020AE
:1048D000409090909060040707060100205090904F
:1048E000909060040707060100500090909090603F
:1048F0000507070600001020885020202004060627
:1049000006010080E09090E0800406060601006049
:1049100090A0A090A004070706010040200070901E
:10492000907004070706010020400070909070040A
:1049300007070601002050007090907004070706DA
:10494000010050A00070909070040606060100500F
:1049500000709090700407070601002050207090AE
:10496000907005040406000070A8B07804060606DE
:1049700001FE70808070204004070706010040207F
:104980000060B0C07004070706010020400060B05E
:10499000C07004070706010020500060B0C070041A
:1049A0000606060100500060B0C07003070706014C
:1049B00000804000C04040E003070706010020409F
:1049C00000C04040E003070706010040A000C040CF
:1049D00040E0030606060100A000C04040E00407D6
:1049E0000706010030601070909060040707060110
:1049F0000050A000E09090900407070601004020BE
:104A0000006090906004070706010020400060905D
:104A10009060040707060100205000609090600439
:104A2000070706010050A00060909060040606068B
:104A30000100500060909060050505060000200010
:104A4000F8002004040406010070B0D0E004070759
:104A500006010040200090909070040707060100B6
:104A6000204000909090700407070601002050003D
:104A7000909090700406060601005000909090708F
:104A80000409090601FE2040009090907090600497
:104A900008080601FE8080E09090E080800408080D
:104AA0000601FE500090909070906000002200255A
:104AB0000028002B002E0031003400020100000508
:104AC0000108010B0100000A0B02090C0D0E08077A
:104AD00003040100000000000000000000000000CE
:104AE00000000000000000000000000000000000C6
:104AF0000012111000000000000000000000000083
:104B00000000000000000000000000290A002062F0
:104B1000797465733B206372632000536574746914
:104B20006E67732053746F7265642028007A5F701B
:104B3000726F62653A20007A5F6D61783A20007A80
:104B40005F6D696E3A2000795F6D61783A20007977
:104B50005F6D696E3A2000785F6D61783A20007869
:104B60005F6D696E3A20005265706F7274696E678E
:104B700020656E6473746F70207374617475730A4A
:104B8000005344207072696E74696E672062797494
:104B90006520004E6F74205344207072696E7469F2
:104BA0006E670A0020496E76616C696420657874CE
:104BB00072756465722000202F0053657474696EED
:104BC000672054726176656C20416363656C657221
:104BD0006174696F6E3A200053657474696E672062
:104BE0005265747261637420416363656C657261C0
:104BF00074696F6E3A200053657474696E67205053
:104C000072696E7420416363656C65726174696F6B
:104C10006E3A200053657474696E67205072696E35
:104C20007420616E642054726176656C2041636308
:104C3000656C65726174696F6E3A200020204D3892
:104C40003531205A005A2D50726F6265204F6666CA
:104C500073657420286D6D293A0A002044002049AC
:104C60000020204D333034205000204400204900E3
:104C700020204D33303120500020440020490020B6
:104C8000500020204D3330312045005049442073DE
:104C9000657474696E67733A0A002046002042000A
:104CA00020480020204D3134352053004D6174657B
:104CB0007269616C206865617475702070617261E1
:104CC0006D65746572733A0A0020204D34323020CD
:104CD00053004175746F20426564204C6576656CA5
:104CE000696E673A0A0020590020580020204D3292
:104CF0003138205400486F74656E64206F666673A7
:104D00006574733A0A00205A0020590020204D3261
:104D10003036205800486F6D65206F666673657485
:104D20003A0A00204500205A00205900205800204F
:104D3000420020540020204D323035205300416481
:104D400076616E6365643A20533C6D696E5F66659B
:104D50006564726174653E20543C6D696E5F747267
:104D60006176656C5F66656564726174653E20425C
:104D70003C6D696E5F7365676D656E745F74696DB8
:104D8000655F6D733E20583C6D61785F78795F6A2E
:104D900065726B3E205A3C6D61785F7A5F6A65721E
:104DA0006B3E20453C6D61785F655F6A65726B3E66
:104DB0000A0020540020520020204D323034205070
:104DC00000416363656C65726174696F6E2028755C
:104DD0006E6974732F7332293A20503C7072696E79
:104DE000745F616363656C3E20523C7265747261EE
:104DF00063745F616363656C3E20543C74726176DA
:104E0000656C5F616363656C3E0A0020450020208D
:104E10004D323031205400205A0020590020204DBE
:104E20003230312058004D6178696D756D204163D5
:104E300063656C65726174696F6E2028756E697444
:104E4000732F7332293A0A0020450020204D32305A
:104E500033205400205A0020590020204D32303396
:104E60002058004D6178696D756D206665656472C6
:104E7000617465732028756E6974732F73293A0AFB
:104E80000020450020204D3932205400205A0020B7
:104E9000590020204D39322058005374657073201A
:104EA00070657220756E69743A0A0020204D3230A8
:104EB000302044300A0020204D3230302054312040
:104EC000440020204D32303020440020446973617A
:104ED000626C65640A0046696C616D656E7420736E
:104EE000657474696E67733A0020204D313439203F
:104EF00043203B20556E69747320696E2043656CB6
:104F0000736975730A002020473231202020203B2E
:104F100020556E69747320696E206D6D0A005761AB
:104F2000726E696E673A20486F6D696E67204275D0
:104F30006D702044697669736F72203C20310A00DD
:104F40000202040000A0400000A040000000400059
:104F5000009B430080A143000087430000484200BB
:104F60000048420000404000000000FF01FF5A20BE
:104F700070726F6265206F75742E206265640A001E
:104F80005A2070726F6265206F75742E206265649E
:104F900000486F6D652058592066697273740A0065
:104FA000486F6D65205859206669727374004F66AA
:104FB00066004F6E2000456E6473746F70206162EE
:104FC0006F72740053746570732F6D6D004A657253
:104FD0006B00416363656C65726174696F6E005646
:104FE000656C6F63697479005A204F6666736574E7
:104FF00000416476616E6365642053657474696E04
:1050000067730020746F6F206C6F6E672065787413
:10501000727573696F6E2070726576656E74656403
:105020000A0020636F6C6420657874727573696F11
:105030006E2070726576656E7465640A0020746F08
:105040006F206C6F6E6720657874727573696F6E10
:105050002070726576656E7465640A0020636F6CFB
:105060006420657874727573696F6E2070726576EE
:10507000656E7465640A00526573746F72652066AC
:1050800061696C73616665004D3530320A4D3530AB
:1050900030004C6F61642073657474696E677300CF
:1050A00053746F72652073657474696E6773004121
:1050B0006476616E6365642053657474696E6773AA
:1050C000004D61696E005072696E742061626F728A
:1050D0007465640041626F7574204669726D776112
:1050E0007265004E6F2053442063617264005072F9
:1050F000696E742066726F6D2053440053746F7034
:10510000207072696E7400526573756D65207072DF
:10511000696E74005061757365207072696E7400F9
:10512000436F6E66696775726174696F6E0054656E
:105130006D7065726174757265004D6F76656D6531
:105140006E74004368616E67652066696C616D65A9
:105150006E740054756E6500496E666F20736372DD
:1051600065656E003A20007A5F6D696E3A20202DE9
:1051700032207A5F6D61783A202035005A204F66E0
:1051800066736574200045787472756465723200C8
:105190004578747275646572004D6F7665205A00AB
:1051A0004D6F76652059004D6F76652058004D6F24
:1051B00076656D656E740045313A200045303A20C1
:1051C000005A3A2000593A2000583A20004D5331F5
:1051D0002C4D53322050696E730A0020420020503B
:1051E000006F6B00526573656E643A2000205A3A76
:1051F0000020593A0020436F756E7420583A002001
:10520000453A00205A3A0020593A00583A0056547C
:10521000726176206D696E005654726176206D69F8
:105220006E005654726176206D696E00566D696E1F
:1052300000566D696E00566D696E00566D6178207E
:10524000453200566D617820453200566D617820F8
:10525000453200566D617820453100566D617820E9
:10526000453100566D617820453100566D617820DA
:105270005A00566D6178205A00566D6178205A00A8
:10528000566D6178205900566D6178205900566D31
:105290006178205900566D6178205800566D61780C
:1052A000205800566D61782058004D6F74696F6EFC
:1052B00000453273746570732F6D6D0045327374E1
:1052C0006570732F6D6D00453173746570732F6D4C
:1052D0006D00453173746570732F6D6D005A737472
:1052E0006570732F6D6D005A73746570732F6D6DDB
:1052F000005973746570732F6D6D00597374657008
:10530000732F6D6D005873746570732F6D6D005839
:1053100073746570732F6D6D004D6F74696F6E00DF
:1053200056652D6A65726B0056652D6A65726B0055
:1053300056652D6A65726B00567A2D6A65726B0030
:10534000567A2D6A65726B0056792D6A65726B000C
:1053500056792D6A65726B0056792D6A65726B00FD
:1053600056782D6A65726B0056782D6A65726B00EF
:1053700056782D6A65726B004D6F74696F6E004DC3
:1053800036303020486F74656E6420746F6F206310
:105390006F6C6420746F206368616E676520666956
:1053A0006C616D656E740A004E6F204C696E6520ED
:1053B0004E756D62657220776974682063686563F5
:1053C0006B73756D2C204C617374204C696E653A5B
:1053D000200053544F505045442E20005072696EA7
:1053E0007465722073746F707065642064756520D5
:1053F000746F206572726F72732E20466978207404
:105400006865206572726F7220616E6420757365C5
:10541000204D39393920746F20726573746172744C
:105420002E202854656D70657261747572652069EF
:10543000732072657365742E20536574206974201F
:1054400061667465722072657374617274696E67E7
:10545000290A004E6F20436865636B73756D207772
:10546000697468206C696E65206E756D6265722C5A
:10547000204C617374204C696E653A200063686546
:10548000636B73756D206D69736D617463682C2037
:105490004C617374204C696E653A20004C696E65EE
:1054A000204E756D626572206973206E6F74204C9A
:1054B000617374204C696E65204E756D6265722B48
:1054C000312C204C617374204C696E653A20004D7C
:1054D000313130004D3331004D38342058205920BF
:1054E0005A20450053442072656164206572726FD2
:1054F000720A00446F6E65207072696E74696E671F
:105500002066696C650A004B494C4C45442E2000CE
:105510004B494C4C20636175736564206279204B64
:10552000494C4C20627574746F6E2F70696E0A005E
:105530004B494C4C45442E20004B494C4C20636158
:105540007573656420627920746F6F206D75636870
:1055500020696E6163746976652074696D65202DBC
:105560002063757272656E7420636F6D6D616E6419
:105570003A2000436F6F6C696E6720646F6E652E12
:105580000048656174696E6720646F6E652E002047
:10559000573A004578747275646572202569202534
:1055A00073004C756C7A426F742054415A20362037
:1055B00072656164792E0000002000230026002916
:1055C000002C002F00320000010000030106010939
:1055D000010000B0C10000A0C10000000000009068
:1055E000430080974300008743436F6F6C646F777D
:1055F0006E0046616E2073706565642031004661FF
:105600006E207370656564203100426564004265F8
:1056100064004E6F7A7A6C652032004E6F7A7A6C35
:10562000652032004E6F7A7A6C652031004E6F7AB9
:105630007A6C652031004D61696E005A204F6666B4
:1056400073657400466C6F77203200466C6F77206C
:105650003200466C6F77203100466C6F7720310046
:1056600046616E20737065656420310046616E206E
:1056700073706565642031004265640042656400B2
:105680004E6F7A7A6C652032004E6F7A7A6C6520A4
:1056900032004E6F7A7A6C652031004E6F7A7A6CE8
:1056A0006520310053706565640053706565640062
:1056B0004D61696E00416D617820453200416D6138
:1056C0007820453200416D617820453100416D619F
:1056D0007820453100416D6178205A00416D617834
:1056E000205A00416D6178205900416D6178205940
:1056F00000416D6178205800416D6178205800416B
:105700002D74726176656C00412D74726176656CE2
:1057100000412D7265747261637400412D7265746D
:105720007261637400416363656C00416363656C1F
:10573000004D6F74696F6E004E414E494E49545989
:10574000494E46CDCCCC3D0AD7233C17B7D138774C
:10575000CC2B329595E6241FB14F0A000020410062
:1057600000C84200401C4620BCBE4CCA1B0E5AAEAC
:10577000C59D7400E300170111241FBECFEFD1E2D5
:10578000DEBFCDBF00E00CBF14E0A0E0B2E0EAEA6B
:10579000F3E602E00BBF02C007900D92AC32B107F6
:1057A000D9F725E1ACE2B4E001C01D92AB39B207F4
:1057B000E1F717E5C6E7D7E500E006C02297010943
:1057C000FE010BBF0F945531C437D10780E00807A5
:1057D000A9F70E94BA7D0D94C4310C9400002F9259
:1057E0003F924F925F926F927F928F929F92AF9271
:1057F000BF92CF92DF92EF92FF920F931F93CF93BE
:10580000DF93CDB7DEB7CB5AD1090FB6F894DEBF20
:105810000FBECDBF00919B0820E6029F800111249E
:10582000055E184F8091300580FF1AC0EBE2F0E171
:1058300084917F013FEFE31AF30A811102C07801DE
:1058400004C00E943954F701F3CFD7018D917D0137
:10585000882319F00E943954F8CF8AE00E94395405
:105860001092B0041092AF048FE380932F05109232
:105870002E0510922D0510924604109247041092A6
:10588000480410924904F80180810F5F1F4F803255
:10589000D1F38E34B1F4818190ED980F9A3020F0DD
:1058A0008D3211F08B3269F43296DF0131962C91F2
:1058B00020532A30D0F3CD01FC0101962081203203
:1058C000D9F3F0932705E09326057F01BFEFEB1A8C
:1058D000FB0A10816AE270E0C7010F9495310097CE
:1058E00039F0DC0111978C918032E1F311961C9212
:1058F0001D3429F0143519F0173409F0CAC0F70126
:105900004E2F9F2F81918032D9F380538A3008F037
:10591000C0C010932F0520912D0530912E05E42F46
:10592000F92F6AE0AF014F5F5F4F629FC001639F35
:10593000900D1124208130E020533109820F931FF4
:10594000218120532A3030F090932E0580932D052D
:105950009A0103C09C01FA01E5CFD9012F5F3F4FA7
:105960004C914032D1F31D34D1F48E31910591F038
:105970003CF48731910571F08C31910581F40AC0B6
:105980008537910564F08737910524F0803AE3E08C
:105990009E0729F4B093B004A093AF047AC010928C
:1059A000B0041092AF04D090260541E050E0FD0114
:1059B00031962C91222309F46CC02132A1F41D34BC
:1059C00091F48032910579F4F093B004E093AF0440
:1059D00063E270E0CF010F949531009709F459C04C
:1059E000DC011C9256C00FEB020F0A31A0F59F019B
:1059F000F90160812F5F3F4F6032D1F320ED260F18
:105A00002A3040F023ED260F223020F06B3211F0C7
:105A10000C94FF469F01602F70E0DB01B595A795C0
:105A2000B595A795B595A795AA5BBB4F07707A0169
:105A3000002E01C0EE0C0A94EAF7FC90FE28FC92BE
:105A40002115310511F02D1901C020E0DB01A45D05
:105A5000BB4F2C930AC02091AF043091B004232B8C
:105A600021F4B093B004A093AF04208121542A31D3
:105A700010F4DF019CCFDF0131966C9160536A30E6
:105A8000D0F39D01F9012F5F3F4F60816032D1F368
:105A9000F0CF80912F058D3409F462C7843511F45D
:105AA0000C94F944873411F00C94E24680912D0552
:105AB00090912E058A31910509F43DC6D4F48430C5
:105AC00091055CF4823091058CF597FF02C00C942F
:105AD000FC460E9403F30C94FC468430910509F4C3
:105AE000E5C50C9711F00C94FC460E94BDE50C94A2
:105AF000FC468E31910509F450C63CF48C31910579
:105B000009F435C60CF41EC637C68B35910509F469
:105B1000EDC68C35910509F4EEC68A35910511F074
:105B20000C94FC4610922C050C94FC4620916402C7
:105B3000222311F40C94FC4611E0029709F010E0C6
:105B40000F942F1982E50F941519882309F45CC16D
:105B50000F943C176B017C014090E5065090E606DF
:105B60006090E7067090E8062091E9063091EA0619
:105B70004091EB065091EC0629962CAF3DAF4EAF0D
:105B80005FAF299740914A0450914B0460914C04B7
:105B900070914D042D964CAF5DAF6EAF7FAF2D97DA
:105BA00060914E0470914F04809150049091510483
:105BB00065966CAF7DAF8EAF9FAF659720E030E00C
:105BC000A901C701B6010F942D2A882309F454C5F1
:105BD000A30192012D966CAD7DAD8EAD9FAD2D973D
:105BE0000F942D2A811111C029962CAD3DAD4EADDB
:105BF0005FAD299765966CAD7DAD8EAD9FAD659718
:105C00000F942D2A882309F437C520E030E0A9013C
:105C1000C701B6010F942D2A881F8827881F1817DF
:105C200059F080E090E0A0E8BFEBA1968CAF9DAF6B
:105C3000AEAFBFAFA1970AC020E030E040E85FE31D
:105C4000A1962CAF3DAF4EAF5FAFA197A3019201DC
:105C50002D966CAD7DAD8EAD9FAD2D970F945F2EC3
:105C600069966CAF7DAF8EAF9FAF699729962CADCB
:105C70003DAD4EAD5FAD299765966CAD7DAD8EADFA
:105C80009FAD65970F945F2E6D966CAF7DAF8EAF15
:105C90009FAF6D9769962CAD3DAD4EAD5FAD6997E9
:105CA000CA01B9010F94922A4B015C016D962CAD8B
:105CB0003DAD4EAD5FAD6D97CA01B9010F94922A0B
:105CC0009B01AC01C501B4010F94602E0F94CB3041
:105CD00061966CAF7DAF8EAF9FAF619720E030E0F3
:105CE00040E05FE30F94922A4B015C01A70196010B
:105CF000C701B6010F94922A6B017C01A5019401A2
:105D0000C501B4010F94922A9B01AC01C701B601F1
:105D10000F945F2E0F94CB309B01AC01A1966CAD1C
:105D20007DAD8EAD9FADA1970F94922A4B015C0182
:105D30002D962CAD3DAD4EAD5FAD2D97C301B2019B
:105D40000F94602E20E030E040E05FE30F94922A51
:105D50006B017C016D966CAD7DAD8EAD9FAD6D9789
:105D6000905861962CAD3DAD4EAD5FAD61970F94EF
:105D70003C2F9B01AC01C501B4010F94922A9B01F9
:105D8000AC01C701B6010F94602EA30192010F94DC
:105D90005F2E6B017C0165962CAD3DAD4EAD5FADC8
:105DA000659729966CAD7DAD8EAD9FAD29970F940B
:105DB000602E20E030E040E05FE30F94922A2B0158
:105DC0003C0161962CAD3DAD4EAD5FAD61976996DE
:105DD0006CAD7DAD8EAD9FAD69970F943C2F9B014F
:105DE000AC01C501B4010F94922A9B01AC01C3011F
:105DF000B2010F94602E29962CAD3DAD4EAD5FAD36
:105E000029970F945F2E14C089E40F9415198823E5
:105E100029F00F943C176B017C0103C0C12CD12CDD
:105E200076018AE40F9415198823F9F00F943C1732
:105E300065966CAF7DAF8EAF9FAF659720E030E089
:105E4000A901C701B6010F942D2A81111EC020E0BF
:105E500030E0A90165966CAD7DAD8EAD9FAD6597C7
:105E60000F942D2A811111C007C420E030E0A90150
:105E7000C701B6010F942D2A882309F4FDC3659646
:105E80001CAE1DAE1EAE1FAE6597B701A6017058C1
:105E900029964CAF5DAF6EAF7FAF299765966CAD1D
:105EA0007DAD8EAD9FAD659790582D966CAF7DAF53
:105EB0008EAF9FAF2D9729962CAD3DAD4EAD5FAD0A
:105EC0002997CA01B9010F94922A4B015C012D96C2
:105ED0002CAD3DAD4EAD5FAD2D97CA01B9010F940C
:105EE000922A9B01AC01C501B4010F94602E0F945E
:105EF000CB30E1966CAF7DAF8EAF9FAFE1978091D5
:105F0000E5069091E606A091E706B091E80669964D
:105F10008CAF9DAFAEAFBFAF6997A7019601BC0133
:105F2000CD010F94602EA1966CAF7DAF8EAF9FAF69
:105F3000A1972091E9063091EA064091EB06509135
:105F4000EC066D962CAF3DAF4EAF5FAF6D9765968B
:105F50002CAD3DAD4EAD5FAD65976D966CAD7DAD35
:105F60008EAD9FAD6D970F94602EA5966CAF7DAFF3
:105F70008EAF9FAFA59740914A0450914B0460911A
:105F80004C0470914D04A9964CAF5DAF6EAF7FAFDE
:105F9000A997A1962CAD3DAD4EAD5FADA197A99649
:105FA0006CAD7DAD8EAD9FADA9970F945F2E6B014B
:105FB0007C0160914E0470914F0480915004909147
:105FC0005104AD966CAF7DAF8EAF9FAFAD97A596E8
:105FD0002CAD3DAD4EAD5FADA5970F945F2E4B013F
:105FE0005C018091ED069091EE06A091EF06B091D4
:105FF000F006E9968CAF9DAFAEAFBFAFE9979C01BD
:10600000AD016091520470915304809154049091B9
:1060100055040F945F2E61966CAF7DAF8EAF9FAF2E
:1060200061972091F1063091F2064091F30650916C
:10603000F406ED962CAF3DAF4EAF5FAFED9760919C
:1060400056047091570480915804909159040F940C
:106050005F2EE5966CAF7DAF8EAF9FAFE597A70142
:10606000960129966CAD7DAD8EAD9FAD29970F94AD
:10607000922A2B013C01A50194012D966CAD7DADBA
:106080008EAD9FAD2D970F94922A9B01AC01C30159
:10609000B2010F94602E2B013C01A50194012996B9
:1060A0006CAD7DAD8EAD9FAD29970F94922A4B01BB
:1060B0005C01A70196012D966CAD7DAD8EAD9FADB7
:1060C0002D970F94922A9B01AC01C501B4010F9446
:1060D0005F2EA30192010F94D32E6B017C0120E06F
:1060E00030E0A9010F942D2A87FF0AC02BED3FE075
:1060F00049EC50E4C701B6010F94602E6B017C019E
:10610000112351F02BED3FE049EC50E4C701B601FB
:106110000F945F2E6B017C0120E030E0A901C701E4
:10612000B6010F942D2A811128C0A9962CAD3DAD42
:106130004EAD5FADA99769966CAD7DAD8EAD9FAD4F
:1061400069970F942D2A811118C0AD962CAD3DADE5
:106150004EAD5FADAD976D966CAD7DAD8EAD9FAD27
:106160006D970F942D2A811108C03BEDC32E3FE09F
:10617000D32E39ECE32E30E4F32EE1962CAD3DAD79
:106180004EAD5FADE197C701B6010F94922A9B0116
:10619000AC010F94922A4B015C0161962CAD3DAD90
:1061A0004EAD5FAD6197CA01B9010F94922A9B0170
:1061B000AC01C501B4010F94602E0F94CB304B019C
:1061C0005C012FE632E143E85AE30F942D2A87FD64
:1061D0004FC2C501B4010F94D52F0F94A92F6B9610
:1061E0007FAF6EAF6B97672B31F441E050E06B9659
:1061F0005FAF4EAF6B976B96AEADBFAD6B97BD010A
:1062000080E090E00F94312A4B015C019B01AC01CE
:10621000C701B6010F943C2F69966CAF7DAF8EAF6E
:106220009FAF6997A501940161966CAD7DAD8EAD70
:106230009FAD61970F943C2FE1966CAF7DAF8EAF11
:106240009FAFE197A5019401E5966CAD7DAD8EAD54
:106250009FADE5970F943C2FE5966CAF7DAF8EAF69
:106260009FAFE59769962CAD3DAD4EAD5FAD69979B
:10627000CA01B9010F94922A20E030E040E05FE3C8
:106280000F94922A9B01AC0160E070E080E89FE3EC
:106290000F945F2EA9966CAF7DAF8EAF9FAFA9977D
:1062A000E9962CAD3DAD4EAD5FADE99729873A87B4
:1062B0004B875C87ED964CAD5DAD6EAD7FADED97D8
:1062C0004D875E876F87788B60919C0270919D02ED
:1062D000882777FD8095982F0F94332A20916002AC
:1062E0003091610240916202509163020F94922AB0
:1062F0002AE037ED43E25CE30F94922AAD966CAF4F
:106300007DAF8EAF9FAFAD970F94481B68537F4F03
:106310008F4F9F4F61966CAF7DAF8EAF9FAF6197F0
:1063200026964FAC269727965FAC279728966FAC9A
:10633000289729967FAC299722242394312C29E190
:10634000922E6B964EAD5FAD6B972416350608F016
:106350004BC10E94EF7A0F94481B61962CAD3DAD66
:106360004EAD5FAD6197621B730B840B950B97FD70
:106370000FC00F94481B68537F4F8F4F9F4F6196FC
:106380006CAF7DAF8EAF9FAF619780E00F94DA1155
:106390009A9409F44FC0A9962CAD3DAD4EAD5FADBA
:1063A000A9972D966CAD7DAD8EAD9FAD2D970F94B9
:1063B000922A6B017C0169962CAD3DAD4EAD5FAD6F
:1063C0006997B201C3010F94922AA70196010F9415
:1063D000602E162F072FB82EA92EA9962CAD3DADF5
:1063E0004EAD5FADA997B201C3010F94922A6B0124
:1063F0007C0169962CAD3DAD4EAD5FAD69972D9694
:106400006CAD7DAD8EAD9FAD2D970F94922A9B0103
:10641000AC01C701B6010F945F2E2B013C01812F07
:10642000902FAB2DBA2D2D968CAF9DAFAEAFBFAFD9
:106430002D975BC0B10180E090E00F94312A6996FE
:106440002CAD3DAD4EAD5FAD69970F94922A4B01D7
:106450005C010F94392F6B017C01C501B4010F94CD
:10646000C1304B015C01A701960129966CAD7DAD51
:106470008EAD9FAD29970F94922A2B013C01A50167
:10648000940165966CAD7DAD8EAD9FAD65970F9413
:10649000922A9B01AC01C301B2010F94602E2B0123
:1064A0003C01A501940129966CAD7DAD8EAD9FADEB
:1064B00029970F94922A4B015C01A70196016596DA
:1064C0006CAD7DAD8EAD9FAD65970F94922A9B010B
:1064D000AC01C501B4010F945F2E2D966CAF7DAF5A
:1064E0008EAF9FAF2D9789E1982E9201A301A196BF
:1064F0006CAD7DAD8EAD9FADA1970F94602E69837D
:106500007A838B839C832D962CAD3DAD4EAD5FADD4
:106510002D97A5966CAD7DAD8EAD9FADA5970F94D3
:10652000602E6D837E838F839887E1962CAD3DAD81
:106530004EAD5FADE19769857A858B859C850F941B
:10654000602E69877A878B879C87E5962CAD3DAD59
:106550004EAD5FADE5976D857E858F8598890F94EB
:10656000602E6D877E878F87988BCE0101960F9462
:10657000FF17C090250589819A81AB81BC818DA3CD
:106580009EA3AFA3B8A78D819E81AF81B88589A74F
:106590009AA7ABA7BCA789859A85AB85BC858DA733
:1065A0009EA7AFA7B8ABAE01435D5F4FBE01675D6D
:1065B0007F4FCE0185960E9490D1AD96ECACFDAC9C
:1065C0000EAD1FADAD979E01235F3F4FAE01435D02
:1065D0005F4FBE01675D7F4FCE0185960E940FE63B
:1065E0003FEF231A330AADCEC090250580914A04AF
:1065F00090914B04A0914C04B0914D048DA39EA3A7
:10660000AFA3B8A780914E0490914F04A09150047D
:10661000B091510489A79AA7ABA7BCA78091520457
:1066200090915304A0915404B09155048DA79EA756
:10663000AFA7B8ABAE01435D5F4FBE01675D7F4F53
:10664000CE0185960E9490D1AD96ECACFDAC0EAD1E
:106650001FADAD9726E534E0AE01435D5F4FBE014F
:10666000675D7F4FCE0185960E940FE60F945E18FE
:106670000F94541B0C94FC46E0EFFFE084918F01D3
:106680000F5F1F4F882321F00E943954F801F6CF85
:10669000E6E3F2E084918F010F5F1F4F882311F42E
:1066A0000C94FC460E943954F801F4CF80E50F9415
:1066B0001519882329F00E9415554B015C0103C070
:1066C000812C912C540183E50F941519882361F0D6
:1066D0000F943C1720E030E04AE754E40F94922AEC
:1066E0000F94A92F4B015C010E9430B580910A02E2
:1066F000811105C060E08CE492E00E94E7D20F9423
:10670000541BC0905B04D0905C04E0905D04F0905A
:106710005E04C80CD91CEA1CFB1C0F94481B6C19A6
:106720007D098E099F0997FD02C00C94FC4680E00C
:106730000F94DA11F2CF81E08093640210925A0430
:106740000C94FC460E94B76581110C94FC4680E5D0
:106750000F941519882319F00F941B1701C060E0DE
:106760006983CE0101960E9437F90C94FC4680E0C3
:106770000E947DDF0C94FC4681E08093D80624982B
:106780002C9A0898109A0E948EA61092D806249AE5
:106790002C98089A10980C94FC4620E030E0A9014F
:1067A0006091E5067091E6068091E7069091E80613
:1067B0000F94602E182F88E5CB55DF4F6883C55A9C
:1067C000D040CA55DF4F7883C65AD040C955DF4FF5
:1067D0009883C75AD0400F941519CB55DF4F688165
:1067E000C55AD040CA55DF4F7881C65AD040C955E6
:1067F000DF4F9881C75AD040882321F00F943C176F
:106800009B0102C09B01812FA901BC014DA35EA386
:106810006FA378A720E030E0A9016091E9067091AC
:10682000EA068091EB069091EC060F94602E5B01D6
:106830008C0189E50F941519882321F00F943C17DA
:106840005B018C01A501B80149835A836B837C836A
:106850004090E9045090EA046090EB047090EC04DE
:106860002091E5043091E6044091E7045091E8045A
:106870006DA17EA18FA198A50F945F2E6B017C0165
:106880002CE032E040EB51EC0F94863087FF02C0E1
:106890000C94FC4621E230E040E953E4C701B60124
:1068A0000F942D2A181614F40C94FC46A30192019F
:1068B000B501C8010F945F2E6B017C012CE032E022
:1068C00040EA51EC0F94863087FF02C00C94FC46DE
:1068D00021E230E847E953E4C701B6010F942D2ABD
:1068E000181614F40C94FC460C94104781E0809325
:1068F0002C050C94FC4685E40F941519C82E8111C3
:1069000002C00E9430B500E5E02E03E0F02E05EE57
:1069100016E0B12CD12CD7018D917D010F94151962
:10692000882361F00F943C17F801608371838283A0
:106930009383F3E0DF1611F0BB24B394D3940C5F80
:106940001F4F24E0D212E7CFBB2019F00E9463BD95
:1069500003C0C1100E94BB660F9417050C94FC463F
:1069600080912D0590912E058937910509F44DC62A
:106970000CF0F6C08D34910509F42EC40CF059C00A
:106980008931910509F4B2C234F58431910509F4D5
:1069900089C27CF48131910509F478C22CF4029704
:1069A00008F4F1C10C94FC46429709F4CAC40C9453
:1069B000FC468631910509F47DC20CF477C287311B
:1069C000910509F47DC2489711F00C94FC460F9490
:1069D00050200C94FC468F31910509F4FFC294F4C9
:1069E0008B31910509F49EC20CF48EC28C31910555
:1069F00009F49CC24E9711F00C94FC460E948297B9
:106A00000C94FC468A32910509F489C32CF48097D2
:106A100009F496C20C94FC468B34910509F4D8C352
:106A20008C34910511F00C94FC460E9400670C9484
:106A3000FC468B36910509F477C40CF04CC08535C3
:106A4000910509F482C47CF58235910509F470C47E
:106A500004F58135910511F00C94FC460F94150452
:106A60000E9430B50F9474171092D6111092D51160
:106A70001092D8111092D71168EE73E080E090E088
:106A80000E94987D60E080E893E00E94E7D20C9439
:106A9000FC468335910509F44FC48435910509F40A
:106AA00050C40C94FC468836910509F499C334F41B
:106AB0008C35910509F464C40C94FC468936910523
:106AC00009F417C48A36910511F00C94FC460E9413
:106AD000A3550C94FC468337910509F4EFC4ECF4FC
:106AE0008E36910509F4DFC34CF48D36910511F013
:106AF0000C94FC460F94DA130C94FC468F369105E7
:106B000009F4D5C38237910511F00C94FC460E941C
:106B100030B50F9417050C94FC468637910509F49F
:106B20005FC574F48537910511F00C94FC4660E064
:106B30008091AF049091B0040E94D7D20C94FC468F
:106B40008737910509F450C58837910511F00C94E9
:106B5000FC4681E08093D4068093B1040C94FC46FB
:106B60008F3231E0930711F40C94293E0CF074C07D
:106B70008D3C910509F4CFC5DCF58E3B910509F4F8
:106B8000BCC3DCF48C38910509F495C34CF48D3703
:106B9000910511F00C94FC460F947F200C94FC4658
:106BA0008139910509F437C58B39910511F00C94A1
:106BB000FC460E9415560C94FC46893C910509F44C
:106BC000A2C54CF4883C910511F00C94FC460E943F
:106BD000EFDA0C94FC468B3C910509F498C58C3C8B
:106BE000910511F00C94FC460E94ADD40C94FC4627
:106BF0008D3D910509F44AC6C4F4833D910509F41D
:106C00008EC54CF48E3C910511F00C94FC460E940C
:106C1000B4BD0C94FC468A3D910509F419C68C3D1F
:106C2000910509F424C60C94FC468C3251E095077A
:106C300009F491C634F4823E910509F443C60C94DC
:106C4000FC468D3271E0970709F489C68E32914077
:106C500009F4A6C70C94FC46843FB1E09B0711F4ED
:106C60000C94CD430CF04CC08039F1E09F0711F437
:106C70000C949242E4F48E3531E0930711F40C94B5
:106C80008D4434F48033914009F40CC70C94FC46D5
:106C90008F3561E0960711F40C949044833691404F
:106CA00011F00C94FC46E0EFFFE00C94E2448239D2
:106CB000A1E09A0711F40C94994214F40C949542B3
:106CC000843AE1E09E0711F40C949D428C3A914085
:106CD00011F00C94FC4659ED852E56E0952E65EE8C
:106CE000A62E66E0B62E7DEF272E74E0372E00E04C
:106CF00010E0A22DA0952696AFAF26970C94F242F5
:106D0000883522E0920711F40C94DC43C4F4863FEA
:106D100041E0940711F40C94D34314F40C94D04341
:106D2000873F61E0960711F40C94D6438C31924072
:106D300011F00C94FC460E940C560C94FC468C38C6
:106D4000A3E09A0711F40C948A447CF48335E3E0C1
:106D50009E0711F40C94D9438B38934011F00C9496
:106D6000FC460F9411030C94FC46803A23E09207F2
:106D700009F427C1873E934011F00C94FC460F9410
:106D800091060C94FC460091AF041091B00480E58C
:106D90000F941519882369F00E9415556B017C0129
:106DA000BB24B394611571058105910531F4B12CB3
:106DB00004C0B12CC12CD12C760183E50F94151998
:106DC0008823F9F00F943C1720E030E04AE754E4C0
:106DD0000F94922A0F94A92F6B017C01B11013C05C
:106DE000611571058105910571F40115110559F0C1
:106DF000D8018C91882339F061E0C8010E94D7D274
:106E000007C0BB2091F360E08BE892E00E94E7D2DC
:106E100081E080939D080E9430B50F94541BC114EB
:106E2000D104E104F104D1F080905B0490905C0403
:106E3000A0905D04B0905E048C0C9D1CAE1CBF1C29
:106E40000F94481B681979098A099B0997FF1AC092
:106E500080919D0881110C94664714C080919D0813
:106E6000882321F080E00F94DA11F8CF8091E412AA
:106E700060E0882319F08CE792E002C087E692E098
:106E80000E94E7D210929D080C94FC4660E08EE9C7
:106E900092E00E94E7D217981698159814981398C4
:106EA0000C94FC460E94839A0C94FC460E944F5B13
:106EB0000C94FC461092E4121092E5120C94FC46DD
:106EC000E091AF04F091B0048081882329F08032F2
:106ED00009F410823196F8CF40E061E08091AF0470
:106EE0009091B0040E946A6F0C94FC461092E412D8
:106EF0000E94006787EA92E090932209809321091B
:106F00000E94ED6B0C94FC468091E512882311F4ED
:106F10000C94FC4683E50F94151981110C946B4772
:106F20000C94FC460E94F5DB0C94FC4640E060E0CB
:106F30008091AF049091B0040E946A6F0C94FC465B
:106F40008091E41281110E9430B50091AF0410913C
:106F5000B00480E50F94E718882321F00E94C955FA
:106F6000F82E01C0F12C8091E512882311F40C94C5
:106F7000FC464F2D61E0C8010E946A6F83E50F94C3
:106F80001519882381F00F941B17AB01BC014093A6
:106F90008715509388156093891570938A1586ED2F
:106FA00094E10E9451638091E512882319F081E0F9
:106FB0008093E412F1100C94FC460E9482660C94BB
:106FC000FC468091AF049091B00421E02093E3123D
:106FD00040E060E00E946A6F0C94FC460E944E669E
:106FE0001CE3C12ED12CE12CF12CA70196010F94AA
:106FF000022E162F072FCA01B901A70196010F947F
:10700000022ED62EC72ECA01B90128E130E040E099
:1070100050E00F94022EFB01C9016DE671E00F9460
:1070200028319B014D2D5C2DDE0111967D0121152E
:10703000310599F00F931F93CF92DF92FF93EF9357
:107040009F938F933F932F9384ED92E09F938F9321
:10705000FF92AF930F94C72912C00097B1F00F931E
:107060001F93CF92DF92FF93EF939F938F9384ECC4
:1070700092E09F938F93FF92AF930F94C7290FB61F
:10708000F894DEBF0FBECDBF30C0309779F00F93BC
:107090001F93CF92DF92FF93EF9388EB92E09F9341
:1070A0008F93FF92AF930F94C729E9CF452B69F0D7
:1070B0000F931F93CF92DF9280EB92E09F938F9379
:1070C000FF92AF930F94C729DACF0F931F938CEAE7
:1070D00092E09F938F93FF92AF930F94C7290F90E5
:1070E0000F900F900F900F900F9060E0C7010E94DB
:1070F000D7D2EBE2F0E184918F010F5F1F4F88231D
:1071000021F00E943954F801F6CFB70188EE92E0E1
:107110000E9442C98AE00E9439540C94FC4683E5DF
:107120000F941519882311F40C94FC460F942B1717
:10713000E82E80E50F941519811114C081E0E1104B
:1071400001C080E08093D806882331F024982C9ADF
:107150000898109A0C94FC46249A2C98089A109837
:107160000C94FC4680E50F941519882341F00F9488
:107170001B1777FF02C00C94FC468B0102C00DE088
:1071800010E0802FE5EFF2E09491891739F0319605
:1071900073E0E532F707C1F70C947C47E0EFFFE0BE
:1071A00084918F010F5F1F4F882321F00E94395473
:1071B000F801F6CFE5E2F3E084918F010F5F1F4FF6
:1071C000882311F40C94FC460E943954F801F4CF42
:1071D0000E9482660C94FC460E9487650C94FC46D3
:1071E00088E690E00E94AEDA81110C94FC46809112
:1071F000300583FF02C00C94FC4683E50F941519FB
:10720000882311F40C94FC460F943C17F090E3048F
:107210000F2D10E0000F111F045A114F0F94A42FCF
:10722000D8016D937C938F2D0E94834C0F943C1753
:1072300020E030E040E752E40F942D2A18163CF08D
:107240000E94876560E083E493E00E94E7D20F9498
:107250003C170091E30410E0F801EE0FFF1FEE0F62
:10726000FF1FE952FB4F20813181428153810F94EE
:107270008630181614F00C94FC4688EF92E09F9329
:107280008F930F5F1F4F1F930F9384E393E09F93A0
:107290008F931F920E949C650FB6F894DEBF0FBEBD
:1072A000CDBF0C94FC460F9421190C94FC460E940F
:1072B00076540C94FC468091300583FF02C00C94F8
:1072C000FC4683E50F941519882311F40C94FC46B1
:1072D0000F943C170F94A42F6739710514F066E9D9
:1072E00070E07093590E6093580E0E94394C0C94C4
:1072F000FC460E94A4960C943C4B8091300583FF81
:1073000002C00C94FC4683E50F94151962968FAF6A
:10731000629781110C94994782E50F941519811198
:107320000C9499470C94FC460E948E550C94FC4694
:1073300010922B050C94FC4681E080932B050C9455
:10734000FC460E9462FC0C94FC4683E50F94E7180F
:10735000882311F40C94FC460F943C1720E030E095
:107360004AE754E40F94922A0F94A92F60935F0484
:107370007093600480936104909362040C94FC46C3
:107380008CE590E00E94AEDA81110C94FC4660E539
:1073900073E027967FAF6EAF27973BE9A32E34E0CB
:1073A000B32E312C2796AEADBFAD27978D91279682
:1073B000BFAFAEAF27970F94E718882309F473C0C7
:1073C000B3E03B1269C00F943C176B017C0120E0D5
:1073D00030E040EA51E40F942D2A2090E30487FF27
:1073E00050C0022D10E00D5F1F4F000F111F000F46
:1073F000111FF801E556FB4FA701960160817181CD
:10740000828193810F943C2F2B013C019B01AC01A5
:1074100060919704709198048091990490919A04D6
:107420000F94922A60939704709398048093990420
:1074300090939A04F801E958FB4F4F01A301920180
:1074400060817181828193810F94922AD4016D931E
:107450007D938D939C9313970D591B4FF801608179
:107460007181828193810F94312AA30192010F943B
:10747000922A0F94A92FD8016D937D938D939C939D
:107480001397B4E02B9EF0011124E955FB4FC08205
:10749000D182E282F38207C00F943C17F50160832A
:1074A0007183828393833394F4E0AF0EB11C24E0A4
:1074B000321278CF0E9418B60C94FC46EEE6F4E047
:1074C00084918F010F5F1F4F882321F00E94395450
:1074D000F801F6CFE0E6F4E084918F010F5F1F4FD3
:1074E000882321F00E943954F801F6CFE9E4F4E052
:1074F00084918F010F5F1F4F882321F00E94395420
:10750000F801F6CFE9E3F4E084918F010F5F1F4F9C
:10751000882321F00E943954F801F6CFE8E2F4E024
:1075200084918F010F5F1F4F882321F00E943954EF
:10753000F801F6CFE7E1F4E084918F010F5F1F4F70
:10754000882321F00E943954F801F6CFE8E0F4E0F6
:1075500084918F010F5F1F4F882321F00E943954BF
:10756000F801F6CFE3EFF3E084918F010F5F1F4F37
:10757000882321F00E943954F801F6CFEDEDF3E0B5
:1075800084918F010F5F1F4F882321F00E9439548F
:10759000F801F6CFE8ECF3E084918F010F5F1F4F05
:1075A000882321F00E943954F801F6CFEBEAF3E08A
:1075B00084918F010F5F1F4F882321F00E9439545F
:1075C000F801F6CFE3E9F3E084918F010F5F1F4FDD
:1075D000882311F40C94FC460E943954F801F4CF2E
:1075E0000E94D9550C94FC4681E08093D8062498DB
:1075F0002C9A0898109A0E9463CD1092D806249A6B
:107600002C98089A10980C94FC461092D40610926C
:10761000B1040C94FC4683E50F941519882319F0E6
:107620000F941B1702C060E070E08B01112702303D
:107630001105D0F0E0EFFFE084918F010F5F1F4F45
:10764000882321F00E943954F801F6CFE7E6F5E0EF
:1076500084918F010F5F1F4F882311F40C94FC4617
:107660000E943954F801F4CF88E40F941519882347
:10767000A9F00F941B17683771053CF0633231E0B5
:1076800073072CF062E271E002C068E770E0F80175
:10769000EE0FFF1FE654FB4F7183608386E40F9467
:1076A0001519882399F00F941B176F3F710519F076
:1076B00014F06FEF70E0F801EE0FFF1FEA54FB4F7C
:1076C00077FF02C060E070E07183608382E40F9412
:1076D0001519882311F40C94FC460F941B17653080
:1076E000710534F0683871052CF067E870E002C06D
:1076F00065E070E0F801EE0FFF1FEE54FB4F718361
:1077000060830C94FC460E9485DB0C94FC460E942E
:1077100059DB0C94FC460E9425550C94FC46EBE288
:10772000F0E184918F010F5F1F4F882321F00E94A9
:107730003954F801F6CF83E50F94E718882321F038
:107740000E94C95580934D02E1EBF5E084918F01D1
:107750000F5F1F4F882321F00E943954F801F6CFA4
:1077600080914D02882319F0E9EAF5E002C0EDEAC4
:10777000F5E084918F010F5F1F4F882321F00E9455
:107780003954F801F6CFE1EAF5E084918F010F5FFB
:107790001F4F882321F00E943954F801F6CF409101
:1077A000F1045091F2046091F3047091F4048FE9B4
:1077B00095E00E9490D44091F5045091F6046091B8
:1077C000F7047091F8048CE995E00E9490D4409100
:1077D000F9045091FA046091FB047091FC0489E96A
:1077E00095E00E9490D4E1E9F5E084918F010F5F6C
:1077F0001F4F882321F00E943954F801F6CF4091A1
:1078000050025091510260915202709153028FE8E0
:1078100095E00E9490D4409154025091550260919D
:107820005602709157028CE895E00E9490D44091E6
:1078300058025091590260915A0270915B0289E896
:1078400095E00E9490D48AE00E9439540C94FC4642
:107850008AED90E00E94AEDA81110C94FC46109102
:10786000E304112311F40C94FC460C94224983E5A3
:107870000F941519882311F40C94FC460F941B17D0
:1078800070939D0260939C020C94FC468DED90E0F9
:107890000E94AEDA81110C94FC4683E50F94151911
:1078A000882311F40C94FC460091E30410E00F943B
:1078B0001B17F801EE0FFF1FE856FD4F7183608321
:1078C0000C94FC4680E50F94E718882311F40C947F
:1078D000FC460F941B17F62E062F172F83E50F94E7
:1078E0001519882321F00F941B176B0103C0CC24BA
:1078F000CA94DC2C96012F5F3F4F2330310510F0E6
:107900000C94FC4617FF02C00C94FC460E9430B554
:107910002FEFC216D20631F0CA94CD2871F000E0E4
:1079200010E00DC08F2D0F94EB1A31E020E0892B71
:1079300009F030E0032F122F02C001E010E08F2D7C
:107940000F94EB1A8017910711F40C94FC4680E019
:107950000F94DA11F4CF0E94647D0C94FC4685E408
:107960000F941519811110C080E50F94E718882332
:1079700091F00F943C176093C7047093C8048093F0
:10798000C9049093CA0407C00F942B17823060F388
:10799000E0EFFFE072C089E40F94E718882381F0DC
:1079A0000F943C172CEA35EC47E25EE30F94922AE1
:1079B0006093C3047093C4048093C5049093C60479
:1079C00084E40F94E718882381F00F943C172CEA85
:1079D00035EC47E25EE30F943C2F6093BF04709355
:1079E000C0048093C1049093C204EBE2F0E184915F
:1079F0008F010F5F1F4F882321F00E943954F80137
:107A0000F6CF4091C7045091C8046091C9047091A9
:107A1000CA0489ED95E00E9490D42CEA35EC47E247
:107A20005EE36091C3047091C4048091C504909199
:107A3000C6040F943C2FAB01BC0185ED95E00E947C
:107A40004BD52CEA35EC47E25EE36091BF047091C0
:107A5000C0048091C1049091C2040F94922AAB019A
:107A6000BC0181ED95E00E944BD58AE00E9439541B
:107A70000C94FC460E943954F80184918F010F5FE9
:107A80001F4F8111F7CF03E013E002C00E94395469
:107A9000D8018D918D018111F9CF8AE00E9439546E
:107AA0000C94FC4680E50F94E718882351F00F945E
:107AB0003C176093D3047093D4048093D5049093BF
:107AC000D60489E40F94E718882381F00F943C17BB
:107AD0002CEA35EC47E25EE30F94922A6093CF04E0
:107AE0007093D0048093D1049093D20484E40F94D3
:107AF000E718882381F00F943C172CEA35EC47E215
:107B00005EE30F943C2F6093CB047093CC0480937E
:107B1000CD049093CE04EBE2F0E184918F010F5FEE
:107B20001F4F882321F00E943954F801F6CF40916D
:107B3000D3045091D4046091D5047091D60485EE9D
:107B400095E00E9490D42CEA35EC47E25EE3609128
:107B5000CF047091D0048091D1049091D2040F94FD
:107B60003C2FAB01BC0181EE95E00E944BD52CEA85
:107B700035EC47E25EE36091CB047091CC048091D8
:107B8000CD049091CE040F94922AAB01BC018DEDEF
:107B900095E00E944BD58AE00E9439540C94FC4633
:107BA00083E50F94E718182F882371F00F943C1782
:107BB0000F94A42F70934F0260934E0221E0672B25
:107BC00009F020E02093BE0480E50F94E718882395
:107BD00071F080914E0290914F02892B19F00E9412
:107BE000C95501C081E08093BE040C94FC4611117C
:107BF0000C94FC46EBE2F0E184918F010F5F1F4F84
:107C0000882321F00E943954F801F6CF8091BE04F8
:107C1000882319F06DE074E002C068EE72E08EEF28
:107C200095E00E9442C960914E0270914F028DEE24
:107C300095E00E940CC2E9EEF5E084918F010F5FA0
:107C40001F4F882311F40C94FC460E943954F8010C
:107C5000F4CF85E40F941519882321F00F941B1796
:107C60001B0102C0212C312C83E40F9415198823A9
:107C700049F00F941B17C457DF4F79836883CC58A2
:107C8000D04008C0E5E0F0E0C457DF4FF983E88357
:107C9000CC58D04085E50F94E718882341F00E9426
:107CA000C955C257DF4F8883CE58D04005C0C25750
:107CB000DF4F1882CE58D040E12CF12C37FE03C0A4
:107CC0000CE812E402C006E113E483E50F941519F1
:107CD000882321F00F943C177B018C01F2E02F16D2
:107CE000310410F42092E3040F94481B2B013C0153
:107CF000C1010196039728F434E1C32E33E0D32E5B
:107D00000BC007E213E0D8018D918D01882309F49F
:107D1000C4CE0E943954F7CFF60181916F018823B8
:107D200019F00E943954F8CF8AE00E9439540F9418
:107D30001504FFEF2F163F0649F487E68093740E73
:107D400027E6822E912CA12CB12C0AC08FE7F101DD
:107D5000E958F14F80839FE7892E912CA12CB12CFB
:107D6000B701C8010F94A42F882777FD8095982F1D
:107D70000F94332AA6966FAFA697AA967FAFAA97BD
:107D8000E6968FAFE697EA969FAFEA9781E08093F9
:107D900080022FEF2216320629F48EEC90E0A0E04C
:107DA000B0E004C08FEF90E0A0E0B0E0AC01BD0116
:107DB0004351510961097109CB56DF4F48835983FB
:107DC0006A837B83C559D0409C01AD0124513109A0
:107DD00041095109C756DF4F288339834A835B83A2
:107DE000C959D040AC01BD01759567955795479528
:107DF000C356DF4F488359836A837B83CD59D04074
:107E00009C01AD012150310941095109CF55DF4F86
:107E1000288339834A835B83C15AD04065968CAEF0
:107E20009DAEAEAEBFAE6597CC57DF4F488259824C
:107E30006A827B82C458D040C157DF4F4882598242
:107E40006A827B82CF58D040AE961FAEAE9730E4A8
:107E5000E2963FAFE2974CE1EE964FAFEE9756E4D5
:107E6000EF965FAFEF97C158DF4F1882CF57D040E2
:107E7000C058DF4F1882C058D040CF57DF4F18820C
:107E8000C158D040CE57DF4F1882C258D040A59677
:107E90001CAE1DAE1EAE1FAEA597A1961CAE1DAEAC
:107EA0001EAE1FAEA197C12CD12C7601C857DF4F53
:107EB000188219821A821B82C858D04061E0CD57BF
:107EC000DF4F6883C358D0406B961FAE1EAE6B97D2
:107ED00010E026961FAE26972A961FAE2A9700E03E
:107EE000C1018958914FCD56DF4F99838883C3597B
:107EF000D040D101AA0FBB1FAA0FBB1FA952BB4F75
:107F00006796BFAFAEAF679780918002882309F470
:107F100002C30F94481B61966CAF7DAF8EAF9FAFCD
:107F200061978091640E882309F4A8C10E94257985
:107F3000BFEF2B163B0679F41091DF04E091E004CB
:107F40002696EFAF2697F091E1042A96FFAF2A9785
:107F50000091E20418C06796AEADBFAD67971C9163
:107F60001196BC912696BFAF26976796EEADFFADF2
:107F70006797F2812A96FFAF2A976796AEADBFAD9D
:107F8000679713960C91212F26963FAD26972A9638
:107F90004FAD2A97502FC158DF4F6881CF57D0403F
:107FA000C058DF4F7881C058D040CF57DF4F88810D
:107FB000C158D040CE57DF4F9881C258D0400F945F
:107FC0002D2A87FF1AC0C158DF4F1883CF57D040E2
:107FD0002696BFAD2697C058DF4FB883C058D04013
:107FE0002A96EFAD2A97CF57DF4FE883C158D0408C
:107FF000CE57DF4F0883C258D040212F26963FAD81
:1080000026972A964FAD2A97502FAE966FADAE9712
:10801000E2967FADE297EE968FADEE97EF969FAD2D
:10802000EF970F948630181694F4AE961FAFAE9764
:108030002696FFAD2697E296FFAFE2972A962FADE0
:108040002A97EE962FAFEE97EF960FAFEF97CD579B
:10805000DF4F3881C358D040332309F48DC0A69632
:108060002FADA697AA963FADAA97E6964FADE69795
:10807000EA965FADEA97612F26967FAD26972A96FE
:108080008FAD2A97902F0F94863018160CF0F6C0FB
:1080900061964CAD5DAD6EAD7FAD619744195509EC
:1080A00066097709C855DF4F488359836A837B8304
:1080B000C85AD040485853416109710977FDDEC064
:1080C000B501A40165968CAD9DADAEADBFAD659714
:1080D000481B590B6A0B7B0B759567955795479510
:1080E0009FEF2916390619F44093740E07C0CD5638
:1080F000DF4FA881B981C359D0404C93C855DF4F99
:10810000288139814A815B81C85AD040C857DF4FE6
:10811000288339834A835B83C858D040A6963FADF5
:10812000A697C158DF4F3883CF57D040AA964FAD9E
:10813000AA97C058DF4F4883C058D040E6965FAD3D
:10814000E697CF57DF4F5883C158D040EA966FADBE
:10815000EA97CE57DF4F6883C258D04061968CAD06
:108160009DADAEADBFAD6197CC57DF4F888399838E
:10817000AA83BB83C458D040A6962FADA697AA96D3
:108180003FADAA97E6964FADE697EA965FADEA97C0
:10819000612F26967FAD26972A968FAD2A97902F2E
:1081A0000F942D2A87FD02C00C94354B61968CAD3F
:1081B0009DADAEADBFAD6197CC57DF4F2881398102
:1081C0004A815B81C458D040821B930BA40BB50B32
:1081D000AC01BD01485853416109710977FF02C0E4
:1081E0000C94354B6B964EAD5FAD6B97452B11F0F4
:1081F0000C947F4965968CAD9DADAEADBFAD6597D6
:10820000880D991DAA1DBB1DB595A79597958795B6
:108210006FEF2616360611F00C942C4B8093740EDB
:108220006B962EAD3FAD6B972F5F3F4F6B963FAF79
:108230002EAF6B97A6963FADA697AE963FAFAE9783
:10824000AA964FADAA97E2964FAFE297E6965FAD3A
:10825000E697EE965FAFEE97EA966FADEA97EF96E8
:108260006FAFEF9761964CAC5DAC6EAC7FAC619735
:1082700071E0CD57DF4F7883C358D04020E030E025
:1082800040EA51E4A6966FADA697AA967FADAA974D
:10829000E6968FADE697EA969FADEA970F94602E2B
:1082A0009B01AC01612F26967FAD26972A968FAD54
:1082B0002A97902F0F94863018166CF4EEECF6E0A7
:1082C00084918F010F5F1F4F882309F495C50E9489
:1082D0003954F801F5CF80E398EFAFEFBFEFC15706
:1082E000DF4F288139814A815B81CF58D040821B82
:1082F000930BA40BB50B61964CAD5DAD6EAD7FAD30
:108300006197840F951FA61FB71FB7FD13C00E946A
:10831000B2958AE00E94395461966CAD7DAD8EAD08
:108320009FAD6197C157DF4F688379838A839B83B1
:10833000CF58D04061968CAD9DADAEADBFAD6197CD
:10834000880F991FAA1FBB1F84199509A609B70991
:10835000CC57DF4F288139814A815B81C458D04096
:10836000821B930BA40BB50B81389F44A241B1052E
:1083700068F0E0EBF6E084918F010F5F1F4F8823D8
:1083800009F43AC50E943954F801F5CF6B964EAD09
:108390005FAD6B97C457DF4F68817981CC58D0406F
:1083A000641775070CF0B4C0E3E5F6E084918F0123
:1083B0000F5F1F4F882321F00E943954F801F6CF38
:1083C0007FEF2716370619F40CEE12E002C00FEA11
:1083D00013E0B80181E496E00E9442C9B701A6010A
:1083E0008DE396E00E9490D48AE00E943954B8014F
:1083F0008BE296E00E9442C9A1964CAD5DAD6EAD98
:108400007FADA19787E296E00E9490D48AE00E9417
:108410003954B80185E196E00E9442C9A5964CAD59
:108420005DAD6EAD7FADA59781E196E00E9490D4E1
:108430008AE00E943954C257DF4F8881CE58D0401D
:10844000882309F4D9C42320209489F5C092D30449
:10845000D092D404E092D504F092D6042CEA35EC04
:1084600047E25EE3A1966CAD7DAD8EAD9FADA19769
:108470000F94922A6093CF047093D0048093D10418
:108480009093D2042CEA35EC47E25EE3A5966CADFE
:108490007DAD8EAD9FADA5970F943C2F6093CB041F
:1084A0007093CC048093CD049093CE04A5C4C09265
:1084B000C704D092C804E092C904F092CA042CEA1E
:1084C00035EC47E25EE3A1966CAD7DAD8EAD9FAD20
:1084D000A1970F94922A6093C3047093C40480936D
:1084E000C5049093C6042CEA35EC47E25EE3A596FA
:1084F0006CAD7DAD8EAD9FADA5970F943C2F609375
:10850000BF047093C0048093C1049093C20474C4E8
:108510000E9403BEF9CC8091800281116DC40F943A
:1085200015046AC40E9430B567C481E00E94ABF8AC
:1085300063C480E00E94ABF85FC486E50F94E7183F
:10854000882321F08FE697E00F94D80483E50F94F9
:10855000E718882321F00E94C955182F01C010E0A8
:1085600083E50F94E718882319F0812F0E94E35DBB
:10857000F090E404111103C0EBE2F0E11AC0F11035
:10858000FBCFE0EFFFE084918F010F5F1F4F882347
:1085900021F00E943954F801F6CFE0E5F7E084912C
:1085A0008F010F5F1F4F882339F30E943954F80160
:1085B000F6CF84918F010F5F1F4F882321F00E9417
:1085C0003954F801F6CFFF2019F060EF72E002C0D5
:1085D00064EF72E082E497E00E9442C98AE00E9460
:1085E00039540AC4F10181911F01882309F4A3C001
:1085F000D5014D905D906D907C90F801E05BFD4F52
:108600002081318142815381F801EF50FB4F60811D
:108610007181828193810F94602E20E030E040E0F0
:108620005FE30F94922A9B01AC01C301B2010F9446
:108630008630181644F4F801E457F84FC590D590E9
:10864000E590F49003C0C12CD12C7601F801EB51D8
:10865000FB4F2081318142815381C301B2010F94CC
:108660005F2E9B01AC01C701B6010F945F2E6B0119
:108670007C0120E030E040EA51EC0F94863087FD29
:108680002BC020E030E040EA51E4C701B6010F946E
:108690002D2A18160CF1F401208131814281538179
:1086A000C701B6010F945F2E9B01AC01C301B2015B
:1086B0000F94602ED5016D937D938D939C931397AA
:1086C000F401C082D182E282F38226968FAD269792
:1086D000820D0F9468182FC0E0EFFFE084918F01A6
:1086E0000F5F1F4F882321F00E943954F801F6CF05
:1086F000E6EBF7E084918F010F5F1F4F882321F095
:108700000E943954F801F6CF61E088EA97E00E94B0
:10871000E7D20E9467D488E290E09A83898388EC4C
:1087200090E09EA38DA3BE016F5F7F4FCE01859623
:108730000E94B97C61C3F4E08F0E911C0C5F1F4F47
:1087400024E0A20EB11C0C30110509F04BCF0E94A1
:1087500063BD0F94170560E088E997E00E94E7D2B7
:1087600083E992E09EA38DA304E610E01A830983B7
:10877000BE016B5D7F4FCE0101960E94B97C8AEBF2
:1087800092E09EA38DA31A830983BE016B5D7F4F88
:10879000CE0101960E94B97C2FC30E9441C22CC316
:1087A0000E9437B829C30E949BB626C30F940804C1
:1087B00023C30F949A0320C30E94B765882319F03E
:1087C00081E00E947DDF85E40F94E718882319F08B
:1087D0000F943C1704C060E070E080E090EC2596B8
:1087E0006CAF7DAF8EAF9FAF25978AE50F941519BB
:1087F000882319F00F943C1704C060E070E080E219
:1088000091E421966CAF7DAF8EAF9FAF219788E545
:108810000F941519882319F00F943C1704C060E0D9
:1088200070E080E291E469AF7AAF8BAF9CAF89E5ED
:108830000F941519882319F00F943C1704C060E0B9
:1088400070E882E993E46DAB7EAB8FAB98AF85E5C2
:108850000F94E718882319F00F943C1704C060E0C8
:1088600070E088EC92EC69AB7AAB8BAB9CAB8CE4A0
:108870000F94E718882319F00F943C1703C060E0A9
:1088800070E0CB016DA37EA38FA398A782E40F9421
:108890001519882321F00F941B17F62E02C045E00E
:1088A000F42ED090D5128091000581112DC0CC24DA
:1088B000C394EF2C8E010F5C1F4F9E012B5C3F4F2A
:1088C000AE01475C5F4FBE01635C7F4FCE018F5BA3
:1088D0009F4F0F94D50D8823B9F08F2D0E94ECF394
:1088E00000E010E028E432E409831A832B833C8300
:1088F00080910005882341F04F2DBE016F5F7F4FAF
:10890000CE0185960F94161F31E0D31275C20E94D6
:10891000826672C20F94D5026FC20F9499076CC21F
:1089200083E50F941519882309F449C00F942B1778
:10893000813039F0823009F042C000E513E0F12CBB
:1089400023C000E513E0F12CD8018D918D010F9427
:108950001519882339F00F942B174FEF682F8F2D9F
:108960000E943151F394B4E0FB12EECF82E40F94F5
:108970001519882321F10F942B174FEF682F1CC076
:10898000F394F4E0FF1679F0F80181918F010F94D0
:1089900015198823A9F30F942B17482F6FEF8F2DEC
:1089A0000E943151EDCF82E40F941519882339F0DC
:1089B0000F942B17482F6FEF84E00E9431510F94D2
:1089C000E3061AC284918F010F5F1F4F882321F0A5
:1089D0000E943954F801F6CFE4EDF7E084918F015D
:1089E0000F5F1F4F882309F407C20E943954F80112
:1089F000F5CFE0902D05F0902E051E2D80912505D8
:108A0000E81631F083E50F94E71881110E94C955EB
:108A100086E40F941519882319F00F943C1703C0AE
:108A200060E070E0CB01123020F08E2D0E94CBDB95
:108A3000E3C120E030E040E752E40F943C2F5B01BB
:108A40006C0120E030E0A9010F94863018168CF0FC
:108A50002090600230906102C0906202D090630268
:108A600050915C0240915D0230915E0220915F0264
:108A700005C015015A2D432D3C2D2D2D852F942FEA
:108A8000A32FB22F8093600290936102A0936202A1
:108A9000B093630200912505101709F470C10F947B
:108AA00054184701992410E0F401EE0FFF1FEE0F58
:108AB000FF1FEB5EFA4FD801AA0FBB1FAA0FBB1F07
:108AC000AB5EBA4F2D913D914D915C91608171816A
:108AD000828193810F945F2E2B013C01F401EE0FF4
:108AE000FF1FEE0FFF1FE35FFA4FD801AA0FBB1F56
:108AF000AA0FBB1FA35FBA4F2D913D914D915C9181
:108B000060817181828193810F945F2E6DA37EA31A
:108B10008FA398A749A65AA66BA67CA61DA61EA63B
:108B20001FA618AA0091711210917212209173124F
:108B300030917412409175125091761260917712B3
:108B40007091781265964CAF5DAF6EAF7FAF659751
:108B50004090791250907A1260907B1270907C1243
:108B600060917D1270917E1280917F12909180129F
:108B70002D966CAF7DAF8EAF9FAF2D9780908112F9
:108B800090908212A0908312B090841280918512EE
:108B900090918612A0918712B091881269968CAF3D
:108BA0009DAFAEAFBFAF69974091891250918A12C5
:108BB00060918B1270918C1229964CAF5DAF6EAFA5
:108BC0007FAF299740918D1250918E1260918F1234
:108BD0007091901280916D1290916E12A0916F120F
:108BE000B091701289839A83AB83BC834D825E827D
:108BF0006F82788669968CAD9DADAEADBFAD69973D
:108C000089879A87AB87BC870D871E872F87388B0C
:108C10002D968CAD9DADAEADBFAD2D97898B9A8B4A
:108C2000AB8BBC8B29968CAD9DADAEADBFAD2997FE
:108C30008D8B9E8BAF8BB88F65968CAD9DADAEAD99
:108C4000BFAD6597898F9A8FAB8FBC8F8D8E9E8EAF
:108C5000AF8EB8A249A35AA36BA37CA3ADB7BEB78E
:108C600094970FB6F894BEBF0FBEADBF119684E2C5
:108C7000FE01319601900D928A95E1F7CE0185961D
:108C80000E94C4CE8DA09EA0AFA0B8A449A45AA4AF
:108C90006BA47CA42DA53EA54FA558A96091ED0617
:108CA0007091EE068091EF069091F0060F94602E81
:108CB0006093ED067093EE068093EF069093F006B6
:108CC000A50194016091E5067091E6068091E706A2
:108CD0009091E8060F94602E6093E5067093E60687
:108CE0008093E7069093E806A30192016091E9065C
:108CF0007091EA068091EB069091EC060F94602E3D
:108D00006093E9067093EA068093EB069093EC0675
:108D1000A501940160910105709102058091030500
:108D2000909104050F94602E6093010570930205E5
:108D300080930305909304050FB6F894DEBF0FBE31
:108D4000CDBF80E00F946818A301920160910505E2
:108D50007091060580910705909108050F94602E8B
:108D600060930505709306058093070590930805A9
:108D700081E00F946818E09225050E9463BD0E946F
:108D800030B5C101D6018093600290936102A09337
:108D90006202B0936302EBE2F0E184918F010F5F16
:108DA0001F4F882321F00E943954F801F6CF6091BB
:108DB000250570E083EE97E00E940CC28AE00E94D5
:108DC00039541AC0EBE2F0E184918F010F5F1F4F1D
:108DD000882321F00E943954F801F6CF60912605CE
:108DE0007091270585EF97E00E9442C982E20E94B8
:108DF00039548AE00E9439540F94FF053DC42091F4
:108E0000AF043091B004232B39F49F012150310974
:108E10003093B0042093AF0420E030E00C940B2D8D
:108E200080E00E94E35D0F94771B83E50F94E718C1
:108E3000882309F449C00E94C95521E0482FBE018A
:108E40006F5F7F4FCE0185960E942FA36B017C013F
:108E50009B01AC010F940C31811131C02CEA35EC2F
:108E600047E257E36DA17EA18FA198A50F94602ED4
:108E7000AB01BC018FE592E00E944BD52CEA35ECAA
:108E800047E257E369817A818B819C810F94602E40
:108E9000AB01BC018AE592E00E944BD52CEA35EC8F
:108EA00047E257E3C701B6010F94602EAB01BC0146
:108EB00085E592E00E944BD58AE00E9439540F94D8
:108EC0005E1B0F94170598CF81E0B7CF80E00F9419
:108ED000DA110C9420370F941B17AB01BC0140939F
:108EE0008715509388156093891570938A1586EDC0
:108EF00094E10E94516380CF802F0E94C4C66E2DE2
:108F0000802F0F94131BF12CB701802F0E94E3C612
:108F10000630110529F4F092D611E092D5116CCFEC
:108F20000830110509F068CFF092D811E092D711FE
:108F300063CF0F943C170F94A42F6739710514F079
:108F400066E970E07093590E6093580E92D40F94B6
:108F50003C1720E030E040EA50E40F9486301816C9
:108F600014F40E9482666091580E7091590E882701
:108F700077FD8095982F0F94332A2091DF0430914C
:108F8000E0044091E1045091E2040F942D2A60E046
:108F900087FF03C083E793E002C086E693E00E9468
:108FA000E7D281E080938002809125058093E304DD
:108FB0002D961CAE1DAE1EAE1FAE2D9761961CAE3B
:108FC0001DAE1EAE1FAE619726961FAE2697669603
:108FD0001FAE6697FCE36A96FFAF6A972CE16E9628
:108FE0002FAF6E9736E4A2963FAFA297C12CD12C3B
:108FF00040E8E42E5FEBF52E812C912C540160911A
:10900000580E7091590E882777FD8095982F0F94F0
:10901000332A162F072F782E692E262F372F482F09
:10902000592FB601C7010F942D2A882331F12091C1
:10903000DF043091E0044091E1045091E204612F9B
:10904000702F872D962D0F942D2A881F8827881F13
:1090500026968FAF269762964FAD6297442389F08C
:10906000882379F080918002882309F4C5CE60E0DE
:1090700088E593E00E94E7D2BFCE1C2D0D2D7E2CFB
:109080006F2C0F94481B6B017C01DC01CB016196B6
:109090002CAD3DAD4EAD5FAD6197821B930BA40B24
:1090A000B50BB7FD3BC0B701A60148515C4F6F4FF0
:1090B0007F4F61964CAF5DAF6EAF7FAF61970E94FF
:1090C000B295E2E6F3E084912F015FEF451A550A6D
:1090D000882321F00E943954F201F5CF81149104C4
:1090E000A104B104A9F0C501B40168517C4F8F4FB0
:1090F0009F4F6C197D098E099F0928EE33E040E0EF
:1091000050E00F94022ECA01B9010E9480C103C031
:109110008FE30E9439548AE00E94395480E00F9412
:10912000DA110F94541B2090DF043090E00440903B
:10913000E1045090E2049101A201612F702F872D6C
:10914000962D0F945F2E9F7720E030E040EA50E4A8
:1091500081149104A104B10429F40F942D2A87FDF0
:1091600005C006C00F948630181614F44601570146
:1091700026966FAD2697662309F448C02D968CADD0
:109180009DADAEADBFAD2D97892B8A2B8B2B71F08A
:10919000D701C6012D962CAD3DAD4EAD5FAD2D97DF
:1091A000821B930BA40BB50BB7FD30C09101A2013C
:1091B00066966FAD66976A967FAD6A976E968FAD2D
:1091C0006E97A2969FADA2970F945F2E20E030E09D
:1091D00040EC5FE30F942D2A87FD44CFB701A60131
:1091E000405A55416F4F7F4F2D964CAF5DAF6EAFDC
:1091F0007FAF2D9766962FAE66976A963FAE6A97B9
:109200006E964FAE6E97A2965FAEA2978091800247
:10921000882309F427CF81149104A104B10429F40F
:10922000C12ED02EE72CF62CEACE58EEC51A53E00C
:10923000D50AE108F108C818D908EA08FB08F7FEC2
:1092400011CFEECF88E50F941519882361F00F94A4
:109250003C1744E0149FF0011124E35FFA4F608350
:1092600071838283938389E50F941519882381F094
:109270000091E30410E00F943C17F801EE0FFF1F7C
:10928000EE0FFF1FEB5EFA4F60837183828393833F
:10929000EBE2F0E184918F010F5F1F4F882321F0F3
:1092A0000E943954F801F6CFE1ECF5E084918F018A
:1092B0000F5F1F4F882321F00E943954F801F6CF29
:1092C0000DE015E080E20E943954D8016D917D9146
:1092D0008D919D918D0142E00F9462048CE20E9479
:1092E0003954F801648175818681978142E00F9439
:1092F0006204F5E005311F0729F70C944D3DC8576E
:10930000DF4F488059806A807B80C858D040480E23
:10931000591E6A1E7B1EC857DF4F288139814A813A
:109320005B81C858D040281B390B4A0B5B0BCA0124
:10933000B90165962CAD3DAD4EAD5FAD65970F940F
:10934000F32DA30192010F94242E820E931EA41ECE
:10935000B51E34E183169104A104B104B4F1CB56D7
:10936000DF4F488159816A817B81C559D04084167D
:109370009506A606B70674F4C356DF4F6881798157
:109380008A819B81CD59D040681579058A059B0556
:1093900064F508C0C756DF4F88809980AA80BB80DB
:1093A000C959D040CF55DF4F88819981AA81BB81AF
:1093B000C15AD04088199909AA09BB0965968CAF92
:1093C0009DAFAEAFBFAF659716C0A4E18A2E912CBA
:1093D000A12CB12C24E130E040E050E065962CAFA8
:1093E0003DAF4EAF5FAF659706C065968CAE9DAE44
:1093F000AEAEBFAE6597EAE3F7E084919F012F5FC1
:109400003F4F8823C1F0CB55DF4F2883C55AD0404A
:10941000CA55DF4F3883C65AD0400E943954CB55C5
:10942000DF4F2881C55AD040CA55DF4F3881C65A10
:10943000D040F901E2CFC501B4010E9480C1E5E34B
:10944000F7E084919F012F5F3F4F8823C1F0CB55F8
:10945000DF4F2883C55AD040CA55DF4F3883C65ADC
:10946000D0400E943954CB55DF4F2881C55AD04097
:10947000CA55DF4F3881C65AD040F901E2CF659610
:109480006CAD7DAD8EAD9FAD65970E9480C1AE96EF
:109490004FADAE97E2965FADE297EE966FADEE9769
:1094A000EF967FADEF978EE297E00E9490D4C1587F
:1094B000DF4F4881CF57D040C058DF4F5881C05848
:1094C000D040CF57DF4F6881C158D040CE57DF4FD3
:1094D0007881C258D04087E297E00E9490D46B9682
:1094E0004EAD5FAD6B974330510514F40C94FA40C8
:1094F00065966CAD7DAD8EAD9FAD65970F94332AAB
:1095000020E030E040E850E40F94922A6B017C01A7
:10951000AE962FADAE97E2963FADE297EE964FAD89
:10952000EE97EF965FADEF97C158DF4F6881CF5749
:10953000D040C058DF4F7881C058D040CF57DF4F60
:109540008881C158D040CE57DF4F9881C258D04053
:109550000F945F2E2BED3FE049E450E40F94922AE4
:1095600020E030E040E05FE30F94922A9B01AC01E1
:10957000C701B6010F943C2F6B017C01C301B201FE
:109580000F94332A2FE632E143E85AE30F94922AEC
:109590002B013C01B701A60181E297E00E9490D423
:1095A000B301A2018BE197E00E9490D42AE939E946
:1095B00049E15FE3C701B6010F94922A6B017C0178
:1095C0009B01AC010F94602EA30192010F943C2FDC
:1095D000A1966CAF7DAF8EAF9FAFA197A301920113
:1095E000C701B6010F94922A20E030E040E05EE32C
:1095F0000F94922AA5966CAF7DAF8EAF9FAFA597C3
:10960000EBE0F7E084913F015FEF651A750A88236C
:1096100021F00E943954F301F5CFB701A60185E08E
:1096200097E00E9490D4A1964CAD5DAD6EAD7FAD3C
:10963000A1978FEF96E00E9490D4A5964CAD5DADBA
:109640006EAD7FADA59789EF96E00E9490D48AE039
:109650000E9439540C94FA40CD56DF4FE881F981CD
:10966000C359D04080830C941041CD57DF4F1882EE
:10967000C358D0400C943E41C555DF4F0FB6F89407
:10968000DEBF0FBECDBFDF91CF911F910F91FF9035
:10969000EF90DF90CF90BF90AF909F908F907F9092
:1096A0006F905F904F903F902F900895CF93DF93EE
:1096B0002FB7F89494E08902E0011124FE01E95EDD
:1096C000F14F60817181828193812FBF0F94332A82
:1096D000C650D94F288139814A815B810F94922AE3
:1096E000DF91CF9108952FB7F894909105019B7F5A
:1096F000909305012FBF87FD96C0A3982FB7F894CC
:10970000909105019460909305012FBF880F2FB7AA
:10971000F894909105019B7F909305012FBF87FDE1
:109720008EC0A3982FB7F894909105019460909300
:1097300005012FBF880F2FB7F894909105019B7FEB
:10974000909305012FBF87FD78C0A3982FB7F89499
:10975000909105019460909305012FBF880F2FB75A
:10976000F894909105019B7F909305012FBF87FD91
:1097700062C0A3982FB7F8949091050194609093DC
:1097800005012FBF880F2FB7F894909105019B7F9B
:10979000909305012FBF87FD4CC0A3982FB7F89475
:1097A000909105019460909305012FBF880F2FB70A
:1097B000F894909105019B7F909305012FBF87FD41
:1097C00036C0A3982FB7F8949091050194609093B8
:1097D00005012FBF982F990F2FB7F894809105019D
:1097E0008B7F809305012FBF97FD1FC0A3982FB7D4
:1097F000F894809105018460809305012FBF2FB7F5
:10980000F894809105018B7F809305012FBF96FD11
:1098100018C0A3989FB7F894809105018460809345
:1098200005019FBF0895A39A69CFA39AE0CFA39A99
:10983000C9CFA39AB3CFA39A9DCFA39A87CFA39A58
:1098400071CFA39AE7CFFC0120E03EE2DB014C910F
:10985000403241F0283011F430833196DB014C91D5
:10986000408331962F5F6F5F7F4F2B3079F71082E7
:109870000895CF92DF92EF92FF92C090DF04D090D4
:10988000E004E090E104F090E2046091580E7091E1
:10989000590E68507109882777FD8095982F0F948D
:1098A000332A9B01AC01C701B6010F942D2A87FF13
:1098B0001DC020E030E040E050E4C701B6010F9445
:1098C000602E0F94A92F7093A9066093A8060F9499
:1098D000481B605A75418F4F9F4F6093AA06709343
:1098E000AB068093AC069093AD0608C01092AA0612
:1098F0001092AB061092AC061092AD06FF90EF905E
:10990000DF90CF900895CF92DF92EF92FF920F9366
:109910001F93CF93DF93082F10E0E801CC0FDD1FDA
:10992000CC0FDD1FFE01E952FB4FC080D180E280E9
:10993000F380000F111FF801E45AF14F608171812B
:1099400065517109882777FD8095982F0F94332AE8
:109950009B01AC01C701B6010F942D2ACE54D94FFB
:1099600087FF1AC00255194F20E030E040E251E471
:10997000C701B6010F94602E0F94A92FF8017183CF
:1099800060830F94481B605C73468F4F9F4F6883C2
:1099900079838A839B8304C0188219821A821B826E
:1099A000DF91CF911F910F91FF90EF90DF90CF90BB
:1099B00008954F925F926F927F928F929F92AF9293
:1099C000BF92CF92DF92EF92FF920F931F93CF93AC
:1099D000DF932C012CEE38E081E090E0F901459115
:1099E0005491441655060CF062C0AC014150510927
:1099F000DA01AA0FBB1FAA0FBB1FA651B74FFD016B
:109A000065917491440F551F440F551F4851574F8E
:109A1000FA0165907490FC01EE0FFF1FEE0FFF1F1F
:109A2000E651F74FA590B490FD0105911491F9010D
:109A3000C591D491FA0185909490882777FD8095FF
:109A4000982F0F94332A6B017C01B20166197709B4
:109A5000882777FD8095982F0F94332A2B013C019E
:109A6000B501601B710B882777FD8095982F0F94A7
:109A7000332A9B01AC01C301B2010F94922A2B013E
:109A80003C01BE0168197909882777FD8095982FD8
:109A90000F94332A9B01AC01C301B2010F943C2FF8
:109AA0009B01AC01C701B6010F94602E11C0019655
:109AB0002C5F3F4F8A33910509F090CFEEECF9E02F
:109AC00065917491882777FD8095982F0F94332A9C
:109AD000DF91CF911F910F91FF90EF90DF90CF908A
:109AE000BF90AF909F908F907F906F905F904F90BE
:109AF00008954F925F926F927F928F929F92AF9252
:109B0000BF92CF92DF92EF92FF92CF93DF93CDB7C8
:109B1000DEB72C970FB6F894DEBF0FBECDBF809195
:109B2000DF049091E004A091E104B091E204898304
:109B30009A83AB83BC836091580E7091590E88272D
:109B400077FD8095982F0F94332A29813A814B8194
:109B50005C810F945F2E6B017C016093790570939B
:109B60007A0580937B0590937C052091D3043091F6
:109B7000D4044091D5045091D6040F94922A6D8359
:109B80007E838F83988760937505709376058093A5
:109B90007705909378052091710530917205409179
:109BA000730550917405C701B6010F94602E4B01E7
:109BB0005C016093710570937205809373059093B7
:109BC00074052091CF043091D0044091D10450917C
:109BD000D2040F94922A69877A878B879C87609337
:109BE0006D0570936E0580936F059093700520ED61
:109BF0003CEC4CE45DE36091CB047091CC0480912B
:109C0000CD049091CE040F94922A2B013C01209117
:109C1000690530916A0540916B0550916C05698129
:109C20007A818B819C810F945F2E9B01AC01C301D3
:109C3000B2010F94922A2B013C0123E333E343E763
:109C40005FE360916505709166058091670590916D
:109C500068050F94922A9B01AC01C301B2010F94D5
:109C6000602E2B013C01609365057093660580931F
:109C700067059093680589819A81AB81BC81809347
:109C8000690590936A05A0936B05B0936C052985CF
:109C90003A854B855C856D817E818F8198850F9497
:109CA000602EA30192010F945F2E2B013C0120E056
:109CB00030E04EE453E40F94863020E030E0A90118
:109CC0001816ACF4C701B6010F94863018166CF55F
:109CD000A7019601C501B4010F945F2E6093710531
:109CE0007093720580937305909374051EC0C30131
:109CF000B2010F942D2A87FF22C020E030E0A90195
:109D0000C701B6010F942D2A87FF16C0A70196013F
:109D1000C501B4010F945F2E6093710570937205B5
:109D2000809373059093740507C0412C512C8EE4E9
:109D3000682E83E4782E03C0412C512C3201C301DC
:109D4000B2012C960FB6F894DEBF0FBECDBFDF91E7
:109D5000CF91FF90EF90DF90CF90BF90AF909F900A
:109D60008F907F906F905F904F9008952F923F92C9
:109D70004F925F926F927F928F929F92AF92BF921B
:109D8000CF92DF92EF92FF920F931F93CF93DF93C7
:109D9000CDB7DEB72A970FB6F894DEBF0FBECDBFA2
:109DA000082F112707FD1095F801EE0FFF1FE45A49
:109DB000F14F20803180C801880F991F880F991FAB
:109DC0009A878987FC01E952FB4F80809180A280AD
:109DD000B380B101882777FD8095982F0F94332A9F
:109DE000A50194010F945F2E6B017C01E985FA8532
:109DF000E35AFA4F608371838283938320ED3CECB6
:109E00004CE45DE36091BF047091C0048091C10493
:109E10009091C2040F94922A2B013C01A985BA8526
:109E2000AB5ABA4FBE83AD832D913D914D915C915C
:109E3000C501B4010F945F2E9B01AC01C301B201B7
:109E40000F94922A2B013C01E985FA85E35BFA4FD6
:109E5000F887EF8323E333E343E75FE360817181B6
:109E6000828193810F94922A9B01AC01C301B201BC
:109E70000F94602E69837A838B839C83AF81B8852E
:109E80006D937D938D939C931397ED81FE818082DA
:109E90009182A282B382F801E750FE4E8081055B79
:109EA0001A4F81111AC020E030E040E251E4C701AE
:109EB000B6010F948630181624F481E0F8018083EF
:109EC000A2C020E030E040E251ECC701B6010F949F
:109ED0002D2A87FD02C0232821F481E0D8018C932C
:109EE00099C0F8018081882351F0E985FA85ED5BFE
:109EF000FA4F1082118212821382D8011C92209193
:109F0000C7043091C8044091C9045091CA04C701E4
:109F1000B6010F94922A2B013C01E985FA85E55C94
:109F2000FA4F608371838283938309851A850D5B61
:109F30001A4FF8012081318142815381C701B60156
:109F40000F94602E4B015C01D8016D937D938D932E
:109F50009C9313972091C3043091C4044091C5048D
:109F60005091C6040F94922A9B01AC01E985FA85B1
:109F7000ED5CFA4F6083718382839383C301B201E6
:109F80000F94602E29813A814B815C810F945F2E62
:109F90002B013C0120E030E04FE753E40F94863082
:109FA00020E030E0A901181694F4C701B6010F941F
:109FB0008630181644F5A7019601C501B4010F9427
:109FC0005F2EF80160837183828393831CC0C30179
:109FD000B2010F942D2A87FF20C020E030E0A901B4
:109FE000C701B6010F942D2A87FF14C0A70196015F
:109FF000C501B4010F945F2ED8016D937D938D93AD
:10A000009C93139707C0412C512C9FE7692E93E432
:10A01000792E03C0412C512C3201C301B2012A9682
:10A020000FB6F894DEBF0FBECDBFDF91CF911F9169
:10A030000F91FF90EF90DF90CF90BF90AF909F90E7
:10A040008F907F906F905F904F903F902F900895EA
:10A050006091DF047091E0048091E1049091E2044A
:10A06000089594E0899FF0011124E952FB4F60812B
:10A0700071818281938108952F923F924F925F92D6
:10A080006F927F928F929F92AF92BF92CF92DF9208
:10A09000EF92FF920F931F93CF93DF9300D01F9205
:10A0A000CDB7DEB72C0170E0FB01EE0FFF1FEA5ABF
:10A0B000FC4F208131813C832B83232B09F4A2C0E8
:10A0C000FB01EC5AFC4F30813A832B813C812C5FA1
:10A0D0003F4F81E090E08983EA818E1708F077C0D6
:10A0E000DC01F901459154910196B9016C5F7F4FF4
:10A0F000441655060CF069C00297AC01440F551F79
:10A10000440F551F4E5F5F4F6B817C81460F571F79
:10A11000FA0165917491880F991F880F991FEB813F
:10A12000FC818E0F9F1FFC0165907490FD01EE0F66
:10A13000FF1FEE0FFF1F3296AB81BC81EA0FFB1FA2
:10A14000A590B490FA0105911491F901859094902D
:10A15000FC0125903490882777FD8095982F0F94E7
:10A16000332A6B017C01B20166197709882777FDD4
:10A170008095982F0F94332A2B013C01B501601B69
:10A18000710B882777FD8095982F0F94332A9B01B8
:10A19000AC01C301B2010F94922A2B013C01B4011E
:10A1A00062197309882777FD8095982F0F94332AB9
:10A1B0009B01AC01C301B2010F943C2F9B01AC0188
:10A1C000C701B6010F94602E06C09B0184CF60E0EA
:10A1D00070E080E090E0F9812A81F2132BC02B819E
:10A1E0003C8144E0F49F200D311D1124225031099F
:10A1F000F90165917491882777FD8095982F0F94C8
:10A20000332A18C0BC01882777FD8095982F0F94BA
:10A21000332A20E030E04AEF5EE30F94922A20E0F8
:10A2200030E040E85DE30F94922A20E030E0A9019D
:10A230000F94602E0F900F900F900F90DF91CF91A1
:10A240001F910F91FF90EF90DF90CF90BF90AF9054
:10A250009F908F907F906F905F904F903F902F9046
:10A26000089567FD5CC0823021F128F4882349F00D
:10A27000813069F054C0833071F1843009F43DC0FD
:10A280004EC0662311F0A19A8FC0A1988DC09FB7D0
:10A29000662329F0F89480910801806804C0F8943E
:10A2A000809108018F77809308019FBF47FF4CC0C2
:10A2B0007FC09FB7662329F0F894809108018064DD
:10A2C00004C0F894809108018F7B809308019FBFA0
:10A2D00047FF40C06FC09FB7662329F0F894809174
:10A2E0000801886004C0F89480910801877F8093FA
:10A2F00008019FBF47FF3EC05AC09FB7662329F0A1
:10A30000F89480910801826004C0F894809108015B
:10A310008D7F809308019FBF47FF39C04AC047FD2A
:10A3200049C08230B9F028F4882341F0813061F0CF
:10A3300008958330F9F0843051F10895442311F0E9
:10A34000A09A0895A0980895442311F0A29A089520
:10A35000A29808959FB7442329F0F89480910801AA
:10A36000806204C0F894809108018F7D8093080179
:10A370009FBF08959FB7442329F0F8948091080166
:10A380008061F4CFF894809108018F7EEFCF9FB762
:10A39000442329F0F894809108018460E7CFF89471
:10A3A000809108018B7FE2CF47FFC8CF08950895C1
:10A3B000089508950895643079F028F4613041F0EB
:10A3C000623041F00895683051F0603141F00895F5
:10A3D00040E003C040E004C041E060E002C041E072
:10A3E00061E03FCF24E08202C0011124FC01E95E5C
:10A3F000F14F4081518162817381FC01E25FF84F2E
:10A400004083518362837383E0914A0EF0914B0E37
:10A4100082899389A489B5898093270E9093280E09
:10A42000A093290EB0932A0E089580E03FD960933F
:10A43000B7107093B8108093B9109093BA1081E060
:10A4400035D96093BB107093BC108093BD1090936E
:10A45000BE1082E02BD96093BF107093C010809320
:10A46000C1109093C21008958091490E9FB780FF4C
:10A4700009C0F89480910B018D7F80930B019FBFE1
:10A480008FEF08C0F89480910B01826080930B01DC
:10A490009FBF81E0809381028091490E9FB781FF29
:10A4A00009C0F89480910B01816080930B019FBFDC
:10A4B0008FEF08C0F89480910B018E7F80930B0181
:10A4C0009FBF81E0809382028091490E9FB782FFF7
:10A4D00009C0F89480910B018B7F80930B019FBF83
:10A4E0008FEF08C0F89480910B01846080930B017A
:10A4F0009FBF81E0809383028091490EE0914A0ED4
:10A50000F0914B0E83FF12C081819FB7811105C06E
:10A51000F89480910B01806404C0F89480910B0141
:10A52000806880930B019FBF8FEF11C081819FB71F
:10A53000811105C0F89480910B018F7B04C0F894C1
:10A5400080910B018F7780930B019FBF81E08093F7
:10A55000840208954F925F926F927F92AF92BF9262
:10A56000CF92DF92EF92FF920F931F93CF93DF93DF
:10A570008C01EB01FC0147A050A461A472A4AFA020
:10A58000B8A4C9A4DAA49501A601C301B2010F942D
:10A590002D2A87FF40C0A3019201C301B2010F948D
:10A5A000922A2B013C01F80183A994A9A5A9B6A977
:10A5B000BC01CD0190589B01AC010F94602EF801B5
:10A5C00027A530A941A952A90F94922A9B01AC0159
:10A5D000C301B2010F945F2E0F94CB307B018C012D
:10A5E0009B01AC01B501C6010F942D2A87FF02C063
:10A5F000750186019701A801B501C6010F942D2AA6
:10A60000882349F0A701B8014FA358A769A77AA7E3
:10A61000888181608883DF91CF911F910F91FF9096
:10A62000EF90DF90CF90BF90AF907F906F905F9052
:10A630004F9008954F925F926F927F928F929F9268
:10A64000AF92BF92CF92DF92EF92FF920F931F9340
:10A65000CF93DF9300D01F92CDB7DEB700912505D1
:10A6600010E00D5F1F4F8BEFE82E81E1F82E9BE984
:10A67000692E94E0792E23E6C22E24E0D22E412CBE
:10A68000512C812C912C54018394F701619171918B
:10A69000819191917F01F3012191319141915191EA
:10A6A0003F0129833A834B835C830F94312A2981AC
:10A6B0003A814B815C810F94922A0F94A92FF60165
:10A6C00061937193819391936F01F2E0F41518F403
:10A6D0004016510639F486169706A806B90610F4F6
:10A6E0004B015C012FEF421A520A85E048165104D3
:10A6F00061F66FEF7FEFCB01A50194010F94022E5D
:10A700002093201130932111409322115093231153
:10A710000F900F900F900F90DF91CF911F910F919D
:10A72000FF90EF90DF90CF90BF90AF909F908F9071
:10A730007F906F905F904F90089561E0FC01808161
:10A740000D94131B8EBD0DB407FEFDCF08958FEF42
:10A750008EBD0DB407FEFDCF8EB508950F931F93E8
:10A76000CF93DF93EB010F94481B8B01F0DF8F3FFA
:10A7700049F00F94481B601B710B6C177D07B0F3F9
:10A7800080E001C081E0DF91CF911F910F9108958A
:10A79000CF92DF92FF920F931F93CF93DF9300D05E
:10A7A0001F92CDB7DEB76C01F62EFC018281982F87
:10A7B000906A96959CBD80FD06C091E0863009F4B4
:10A7C00090E0892F01C080E08DBD60E0F6018081BE
:10A7D00029833A834B835C830F94131B6CE271E0F3
:10A7E000C601BCDF8F2D8064ADDF08E110E05C8125
:10A7F0004B813A812981DA01C901002E04C0B69546
:10A80000A795979587950A94D2F729833A834B8326
:10A810005C8398DF0850110929813A814B815C8162
:10A82000083FFFEF1F0739F7FF2029F088E0F816EF
:10A8300021F08FEF03C085E901C087E883DFECE0FA
:10A84000FE1201C084DF10E082DFF601838387FF00
:10A8500004C01F3F11F01F5FF7CF0F900F900F90B4
:10A860000F90DF91CF911F910F91FF90DF90CF90CC
:10A8700008959091C00095FFFCCF8093C600089585
:10A88000EF92FF921F93CF93DF931F92CDB7DEB766
:10A89000182FE0EEF8E084917F012FEFE21AF20A20
:10A8A000882329F09983E5DFF7019981F4CFE12F1F
:10A8B000F92F84917F019FEFE91AF90A882319F093
:10A8C000D8DFF701F6CFE7ECF8E084917F01AFEF36
:10A8D000EA1AFA0A882319F0CCDFF701F6CF0F90B5
:10A8E000DF91CF911F91FF90EF900895DF92EF924B
:10A8F000FF920F931F93CF93DF9383E50F94151966
:10A90000882319F00F942B1701C080E08093300545
:10A91000EBE2F0E18491EF012196882319F0A9DFA1
:10A92000FE01F8CFE0ECF8E08491EF012196882356
:10A9300019F09FDFFE01F8CF80913005882371F177
:10A9400002EB18E0C0E0D0E020E08091300590E01C
:10A950000C2E02C0959587950A94E2F780FF15C0EA
:10A96000DD24D394D20E222311F08CE282DFF80191
:10A9700025913491F90184917901FFEFEF1AFF0AD3
:10A98000882321F076DF9701F5CFD22E21960E5F36
:10A990001F4FC530D10561F02D2DD7CFECEBF8E07E
:10A9A0008491EF012196882319F063DFFE01F8CF2F
:10A9B0008AE0DF91CF911F910F91FF90EF90DF9090
:10A9C00058CF3FB7F8942091200980911F09821732
:10A9D00059F0E22FF0E0E156F74F808190E02F5FD1
:10A9E0002F772093200902C08FEF9FEF3FBF08957C
:10A9F000CF93FC01C62F80818B33A1F080919C08FE
:10AA0000843080F420912F1130E6239FC00111245F
:10AA1000BF01855E984F0F94A0318C2F0F94D218F0
:10AA200081E001C080E0CF9108958091310590913F
:10AA30003205009731F04AE050E060E070E00D949C
:10AA40006D2860E070E0CB01089583E50F94E7186E
:10AA5000882351F00F943C1760933711709338118D
:10AA60008093391190933A1184E50F94E718882365
:10AA700051F00F943C17609333117093341180930D
:10AA800035119093361182E40F94E718882349F02A
:10AA9000CCDF6093E8107093E9108093EA109093F4
:10AAA000EB1088E50F94E718882351F00F943C17BA
:10AAB00060938B0470938C0480938D0490938E0428
:10AAC00089E50F94E718882351F00F943C176093A1
:10AAD0008F047093900480939104909392048AE57C
:10AAE0000F94E718882351F00F943C176093930458
:10AAF00070939404809395049093960485E40F9446
:10AB0000E718882351F00F943C17609397047093D3
:10AB100098048093990490939A04089580E50F9483
:10AB20001519882331F00F941B176230710550F40A
:10AB300002C060E070E0FB01EE0FFF1FEB52FE4E23
:10AB4000118210820895CF93DF9383E50F94151936
:10AB5000882339F00F941B17EB016F3F710519F033
:10AB600010F0CFEFD0E080E50F941519882329F07D
:10AB70000F942B17823050F401C080E0E82FF0E0F2
:10AB8000EE0FFF1FEB52FE4ED183C083DF91CF91BA
:10AB900008958091310590913205892B41F00F94F1
:10ABA0002B1791E0811101C090E0892F089581E079
:10ABB0000895CF93DF9385E40F94E718882369F015
:10ABC000E8DF882351F0EBE2F0E18491EF01219678
:10ABD000882319F04EDEFE01F8CF81E40F94E718C8
:10ABE000882369F0D6DF882351F0EEEAF8E08491FB
:10ABF000EF012196882319F03CDEFE01F8CFC091C9
:10AC0000AF04D091B0048991882311F032DEFBCFDC
:10AC10008AE0DF91CF912DCE83E50F94E71888234A
:10AC200019F0B7DF8093F9060895CF92DF92EF9283
:10AC3000FF9283E50F9415198823F1F00F942B17D9
:10AC40008D3308F08CE38093BB110F94481B6B018C
:10AC50007C012091BB1130E0A8EEB3E00F94502EA0
:10AC6000C60ED71EE81EF91EC092B711D092B811B9
:10AC7000E092B911F092BA11FF90EF90DF90CF906F
:10AC800008952F923F924F925F926F927F928F9290
:10AC90009F92AF92BF92CF92DF92EF92FF920F936B
:10ACA0001F93CF93DF93CDB7DEB72B970FB6F894F2
:10ACB000DEBF0FBECDBF9E838D83DC0159962D90E4
:10ACC0003C905A97F1014184528463847484FFEF6D
:10ACD0004F1A5F0A6F0A7F0A1496CD90DD90ED90AF
:10ACE000FC901797C114D104E104F10439F02FEF5F
:10ACF000C21AD20AE20AF20A1B8607C0D101CD901D
:10AD0000DD90ED90FC90B1E0BB87460157011F82BA
:10AD1000188619861A86F10181859285A385B485E6
:10AD20002F81388549855A85281739074A075B07D7
:10AD300008F08DC04C145D046E047F0450F482E072
:10AD4000C82ED12CE12CF12C92E0892E912CA12C33
:10AD5000B12C9E012F5F3F4FB701A601C1010E9498
:10AD60005861882309F473C089819A81AB81BC81C1
:10AD7000892B8A2B8B2B41F0460157013FEF831A19
:10AD8000930AA30AB30A05C0C814D904EA04FB0451
:10AD900089F08F819885A985BA850196A11DB11D7D
:10ADA0008F839887A987BA879FEFC91AD90AE90ABA
:10ADB000F90AB1CF0FEF1FEF2FEF3FE0B501A4016C
:10ADC000C1010E94A164F82E882309F440C0ED81DE
:10ADD000FE81448155816681778141155105610568
:10ADE000710539F095018401C1010E94A164882395
:10ADF00071F1AD81BE8114968D929D92AD92BC92FF
:10AE00001797BB85BB2351F0D501C4010196A11D45
:10AE1000B11DF10180839183A283B383ED81FE8113
:10AE200085899689A789B08D892B8A2B8B2B81F4F4
:10AE3000AD81BE8155968D929D92AD92BC925897F0
:10AE400011968C911197806811968C9301C0F12C0A
:10AE50008F2D2B960FB6F894DEBF0FBECDBFDF91BE
:10AE6000CF911F910F91FF90EF90DF90CF90BF9007
:10AE7000AF909F908F907F906F905F904F903F909A
:10AE80002F900895CF93DF93EC018B81882391F16C
:10AE9000898187FF2BC06C857D858E859F8541E0EC
:10AEA0000E94C85F882331F1E88980E2E89FF001C1
:10AEB0001124E356F14F3097E9F08081853ED1F0BF
:10AEC0008B81823040F449895A896B897C89448F0F
:10AED000558F668F778F4D895E896F89788D538FF7
:10AEE000428F758B648B89818F778983DF91CF91B6
:10AEF0000C948A5F81E0888380E0DF91CF91089590
:10AF0000CF93DF93EC018B81813099F4898181FFAC
:10AF100010C049895A896B897C89452B462B472B60
:10AF200059F140E050E0BA01CE010E945163811115
:10AF300002C080E022C04D895E896F89788D898D3D
:10AF40009A8D0E9430658823A1F31D8A1E8A1F8A6C
:10AF5000188E198A1A8A1B8A1C8A898180688983BB
:10AF6000CE0190DF882329F340E050E0BA01CE0102
:10AF7000DF91CF910C94516381E0DF91CF910895DF
:10AF80006F927F928F929F92AF92BF92CF92DF92F9
:10AF9000EF92FF920F931F93CF93DF931F92CDB742
:10AFA000DEB78C015B014A01722EDB0159968D914F
:10AFB0009C915A97F801928F818F40E050E0BA013E
:10AFC000C5010E945163E12CF50180859185A28520
:10AFD000B385418952896389748984179507A607C7
:10AFE000B70708F0CEC035E0B695A7959795879539
:10AFF0003A95D1F7F82FFF70FF2ED50113968C915B
:10B00000823008F497C141E050E0BE016F5F7F4F8E
:10B01000C5010E94D761019719F4898190E002C0AF
:10B020008FEF9FEF019609F485C1F5018085918529
:10B03000A285B3854F96A11DB11D80879187A287F8
:10B04000B387F0E2FF9EB00111246356714F611582
:10B05000710509F46FC1DB018C91882311F0853EE5
:10B06000B9F4E1100EC08091800590918105A09106
:10B070008205B0918305F80184879587A687B787F5
:10B08000F08ADB018C91EE24E39481119DCF79C08D
:10B090004BE050E0C4010F946131892B09F094CF4B
:10B0A00077FC48C120E2F29EF0011124E356F14FF3
:10B0B0008385817121F0872D827109F05EC04091F6
:10B0C0008005509181056091820570918305D801BA
:10B0D0001C964D935D936D937C931F975096FC92B5
:10B0E0004489558960E070E0BA0155274427828D74
:10B0F000938DA0E0B0E0482B592B6A2B7B2BD80115
:10B1000055964D935D936D937C9358978385887185
:10B1100059F4848D958DA68DB78DF801818B928B16
:10B12000A38BB48B81E010C0803139F598012F5E7C
:10B130003F4FD80159968D919C915A970E94EA638E
:10B140008823D9F084E0F8018383872D8F70D8019C
:10B1500011968C931197F80114821582168217822A
:10B1600018961D921D921D921C921B9774FED5C0BD
:10B17000C801C6DE8111D1C0DEC0D80113961C9271
:10B18000D9C0872D8274823409F0D4C0EE20D9F062
:10B19000D8015096FC9050971C966D917D918D91A1
:10B1A0009C911F9741E0F4D6882309F4C3C0F801AD
:10B1B0008089F0E28F9FC00111248356914F009740
:10B1C00009F08CC0B7C0D50113968C9113978230CB
:10B1D00009F4B0C051968D919D910D90BC91A02D18
:10B1E000803E9F4FAF41B10508F0A4C0C50149DDC5
:10B1F000882309F49FC08ED6882309F49BC0D5010B
:10B200005996ED91FC915A971496CD90DD90ED9062
:10B21000FC901797B2E0CB1AD108E108F108058439
:10B2200004C0CC0CDD1CEE1CFF1C0A94D2F78685F2
:10B230009785A089B189C80ED91EEA1EFB1E81E040
:10B2400080937F05C0928005D0928105E0928205AF
:10B25000F092830580E092E0EDE9FEE0DF019C01E1
:10B260001D9221503040E1F766246394D501599630
:10B27000ED91FC915A978481681690F42DE93EE097
:10B28000B701A601460D511D611D711D80917D05FF
:10B2900090917E05D3D5882309F44CC06394E6CF02
:10B2A00040E052E060E070E0058404C0440F551FA8
:10B2B000661F771F0A94D2F751968D919D910D903C
:10B2C000BC91A02D840F951FA61FB71FF501818B80
:10B2D000928BA38BB48B8DE99EE0F12C20E2DC01F4
:10B2E0001D922A95E9F72BE0F401DC0101900D9203
:10B2F0002A95E1F721E238E2FC01318B208B40E016
:10B3000058E057874687338B228B318F208F578B9E
:10B31000468B00D68111C6CE0DC075FE09C0F8015E
:10B320004189528963897489C8010E94516303C0AD
:10B3300081E001C080E00F90DF91CF911F910F91CC
:10B34000FF90EF90DF90CF90BF90AF909F908F9045
:10B350007F906F9008952F923F924F925F926F92DD
:10B360007F928F929F92AF92BF92CF92DF92EF9295
:10B37000FF920F931F93CF93DF9300D01F921F92E2
:10B38000CDB7DEB78C015B014D83252EDC01139612
:10B390008C9113978130C9F411968C9181FF15C05F
:10B3A00082FF19C0F80141895289638974898085B7
:10B3B0009185A285B38584179507A607B70759F02D
:10B3C000C8010E945163811106C081E0F8018083A9
:10B3D0008FEF9FEF29C1ED80F22C7FC0D8015996E5
:10B3E000ED91FC915A9734803A94DB01CA0169E0EF
:10B3F000B695A795979587956A95D1F738224A0112
:10B40000B1E09B22332009F474C080E092E08819F7
:10B41000990967018E159F0508F46C01D8015996AA
:10B42000ED91FC915A9714964D905D906D907C90A3
:10B430001797B2E04B1A510861087108058404C0DF
:10B44000440C551C661C771C0A94D2F78685978598
:10B45000A089B189480E591E6A1E7B1E430C511CDF
:10B46000611C711CC114E2E0DE0609F089C0809104
:10B47000800590918105A0918205B0918305841586
:10B480009505A605B70569F410927F058FEF9FEF2C
:10B49000DC018093800590938105A0938205B09391
:10B4A00083059501B301A20180917D0590917E05F0
:10B4B000C5D4882309F489CFF80180859185A285B8
:10B4C000B3858C0D9D1DA11DB11D80879187A2871D
:10B4D000B387AC0CBD1CEC18FD08D80118964D9133
:10B4E0005D916D917C911B97E114F10409F076CF89
:10B4F0007BC08114910409F088CFD80114964D9136
:10B500005D916D917C91179741155105610571050C
:10B5100059F455968D919D910D90BC91A02D009759
:10B52000A105B10539F521C09E012F5F3F4FCF0125
:10B53000BFD6882309F449CF89819A81AB81BC8128
:10B54000F801218D328DF9012789203139F4883FA6
:10B55000FFEF9F07A105B10540F40CC0883F2FEF16
:10B560009207A2072FE0B20728F0C8018ADB8111F9
:10B570004CCF2BCFF80184839583A683B78345CF27
:10B580008114910411F5D80118964D915D916D913A
:10B590007C911B9751968D919D910D90BC91A02D02
:10B5A000481759076A077B0780F0B4D4882309F449
:10B5B0000CCF81E080937F054092800550928105F9
:10B5C000609282057092830507C041E0C301B20119
:10B5D000DFD4882309F4F9CEA601B501C40183564E
:10B5E000914F0F946E3168CF51968D919D910D9032
:10B5F000BC91A02D84179507A607B70740F4F80162
:10B60000418B528B638B748B818180688183D801DD
:10B6100011968C9183FD03C08D81922D05C0C801C8
:10B6200031DC8111F9CFD1CE0F900F900F900F9098
:10B630000F90DF91CF911F910F91FF90EF90DF90CE
:10B64000CF90BF90AF909F908F907F906F905F90C2
:10B650004F903F902F900895CF93DF931F92CDB7D7
:10B66000DEB7698341E050E0BE016F5F7F4F049613
:10B6700072DE0F90DF91CF910895CF93DF93EC01AD
:10B6800001DC1B82DF91CF9108951092E41280912A
:10B69000D914882319F086ED94E1EFCF0895CF9265
:10B6A000DF92EF92FF921F93CF93DF931092E512F8
:10B6B00080913F13882319F08CE393E1DEDF109231
:10B6C000B3141092B01485E38093AF140F94481B09
:10B6D000EB01A8958091AF140E94C4C68FEA94E153
:10B6E0002CD82398229A219A209A289A85E0809330
:10B6F000B11482E58CBD1DBC1AE08FEF23D8115028
:10B70000E1F720E030E0A90160E08FEA94E140D861
:10B71000182F8093B214813049F00F94481B6C1B92
:10B720007D0B613D774068F381E051C02AEA31E04A
:10B7300040E050E068E08FEA94E12AD882FF03C03D
:10B740001093B3140DC014E002D88093B2141150BA
:10B75000D9F78A3A11F082E03AC082E08093B314BC
:10B760008091B314823031F4C12CD12CE12C70E4DF
:10B77000F72E03C0C12CD12C760120E030E0A901C6
:10B7800067E38FEA94E104D8A701960169E28FEAA2
:10B7900094E10E94C8538093B214882349F00F9417
:10B7A000481B6C1B7D0B613D774038F38AE00FC06E
:10B7B0008091B314823011F520E030E0A9016AE3F2
:10B7C0008FEA94E10E94C853882351F088E0809367
:10B7D000B0148FEA94E10E949D53EBE2F0E119C0AE
:10B7E0000E94A753807C803C19F483E08093B314BB
:10B7F0000E94A7530E94A7530E94A7538FEA94E187
:10B800000E949D531092B11481E0F9D381112DC093
:10B8100013C08491EF012196882319F02AD8FE01E4
:10B82000F8CFE1E0FAE08491EF012196882309F452
:10B8300053C01FD8FE01F7CF80E0E1D3811115C0BE
:10B84000E0EFFFE08491EF012196882319F011D8F1
:10B85000FE01F8CFEDEEF9E08491EF012196882307
:10B8600009F43AC006D8FE01F7CF64EB74E18CE32B
:10B8700093E10E945064811116C0E0EFFFE08491D3
:10B88000EF012196882321F00E943954FE01F7CF61
:10B89000ECEDF9E08491EF0121968823E9F00E9414
:10B8A0003954FE01F7CF81E08093E512EBE2F0E13D
:10B8B0008491EF012196882321F00E943954FE01E2
:10B8C000F7CFE0EDF9E08491EF012196882321F094
:10B8D0000E943954FE01F7CF8BE1ECE3F3E1ADE5D3
:10B8E000B3E101900D928A95E1F780913A1390911E
:10B8F0003B1390935C1380935B1388E393E19093E5
:10B90000581380935713DF91CF911F91FF90EF90C1
:10B91000DF90CF900895FC0123812111AECE0895D0
:10B920002F923F924F925F926F927F928F929F924F
:10B93000AF92BF92CF92DF92EF92FF920F931F933D
:10B94000CF93DF93CDB7DEB7C454D1090FB6F894C7
:10B95000DEBF0FBECDBF4C015B017A01322E1C8EC3
:10B960001F8E19821C826115710511F410E0ABC0A5
:10B97000FC0183818111FACFFA0180818F3261F459
:10B98000CA017C010196F70120812F32D1F3F50124
:10B9900083818250823010F465010AC0618D728DFE
:10B9A000CE0101967DD7882309F3CE0101966C0163
:10B9B0008E01045E1F4F2801E7E36E2E712C6C0E82
:10B9C0007D1E9BE0690E711CFE0131962496FFAF2F
:10B9D000EEAF249725960FAF2597212E35C080E234
:10B9E0008193E615F705D9F7D70120E097E04A2FB4
:10B9F0003B2F8D9181112BC08FA9803209F4B6CFD6
:10BA0000842F932F7C01FC01208101962F32D1F3EA
:10BA1000222309F450C021E0AE01495C5F4FB6011A
:10BA2000C801AEDA882309F4A1CFCA14DB0411F0EF
:10BA3000C60123DE04151505B9F125969FAD25979E
:10BA4000822D6801092F182FFE01F796C8CF8F327B
:10BA500099F28E3219F0EFE0FAE00AC09A3009F458
:10BA600085CF28E09AE0C3CF3196381709F47ECF0E
:10BA700034913111F9CF921708F478CF813208F45C
:10BA800075CF8F3709F472CF31E0320FE7E3F0E082
:10BA9000EC0FFD1FE20FF11D2FE9280F2A3108F4EA
:10BAA00080528083232FA3CF23969FAD2397249684
:10BAB0008FAD2497C6CF232DAE01495C5F4FB601F1
:10BAC000C4015EDA182FCE01019625DFCE014C9617
:10BAD00022DF812FCC5BDF4F0FB6F894DEBF0FBEA5
:10BAE000CDBFDF91CF911F910F91FF90EF90DF902D
:10BAF000CF90BF90AF909F908F907F906F905F900E
:10BB00004F903F902F90089520E733E0FC01318360
:10BB10002083049600CFCF92DF92EF92FF920F9393
:10BB20001F93CF93DF938C01EB016A0179010E948F
:10BB300079D323E020939E0210934811009347117C
:10BB4000D0934611C0934511A601662757FD609515
:10BB5000762F40934111509342116093431170939B
:10BB60004411C701AA2797FDA095BA2F841B950BF6
:10BB7000A60BB70B80933D1190933E11A0933F11FC
:10BB8000B093401188819981AA2797FDA095BA2F7B
:10BB9000841B950BA60BB70B80931F12909320125A
:10BBA000A0932112B09322128AEC95E7909397020A
:10BBB00080939602DF91CF911F910F91FF90EF90AC
:10BBC000DF90CF9008959091E404891781F08093DD
:10BBD000E404811108C00E94155287EB90E10E9495
:10BBE00018D00D94C71985EE96E00C9418D00895DE
:10BBF00080E0E9DF80E090E0A0E8BFE380936D1291
:10BC000090936E12A0936F12B093701210927112F3
:10BC10001092721210927312109274121092751286
:10BC20001092761210927712109278121092791266
:10BC300010927A1210927B1210927C1280937D12D5
:10BC400090937E12A0937F12B09380121092811273
:10BC50001092821210928312109284121092851206
:10BC600010928612109287121092881210928912E6
:10BC700010928A1210928B1210928C1280938D1255
:10BC800090938E12A0938F12B093901208958F927A
:10BC90009F92AF92BF92CF92DF92EF92FF920F935B
:10BCA0001F93CF93DF93882EB62EA42EF22EE80199
:10BCB000242F220F220F220F0F2D462F682F83E3F0
:10BCC00092E10F942A1A882351F10B2D0F0DCA2CE3
:10BCD000D12CB01621F17E019A2C182D9920D9F083
:10BCE000F7018491609135127091361210934F12C2
:10BCF000B092501210925212809351122FE432E1FE
:10BD00004BE383E392E10F944C1AFFEFEF1AFF0A23
:10BD10009A94185FE3CFCC0DDD1DB394DACFDF9199
:10BD2000CF911F910F91FF90EF90DF90CF90BF9038
:10BD3000AF909F908F900895FB014081FC0120817E
:10BD40003181342768E0A901440F551F37FD07C032
:10BD50009A016150C1F7FC013183208308959A0153
:10BD6000F1E22F27F0E13F27F4CFEF92FF920F93FC
:10BD70001F93CF93DF93EC0189018C81833039F0DD
:10BD8000E9E0440F551F661F771FEA95D1F79A0126
:10BD9000AB0161E1CE010E94C853882331F084E0F9
:10BDA0008983CE010E949D5341C00F94481B7B01A3
:10BDB0000E94A7538B838F3F49F40F94481B6E1941
:10BDC0007F096D327140A0F381E103C08E3F49F0DD
:10BDD0008FE08983CE010E949D538FEF0E94A25372
:10BDE00025C08FEF8EBDF80180E090E02FEF0DB4FD
:10BDF00007FEFDCF3EB531932EBD01968F3F31E05A
:10BE00009307A9F70DB407FEFDCF8EB5F801E150F9
:10BE1000FE4F80830E94A7530E94A753CE010E9429
:10BE20009D538FEF0E94A25381E001C080E0DF911B
:10BE3000CF911F910F91FF90EF9008950F931F9353
:10BE4000CF93DF93EC0189018C81833039F0F9E0E5
:10BE5000440F551F661F771FFA95D1F79A01AB0162
:10BE600068E1CE010E94C853882311F086E034C0F7
:10BE70008EEF8EBD80E090E00DB407FEFDCFF8019F
:10BE8000E80FF91F20812EBD0DB407FEFDCF2181E3
:10BE90002EBD0296811522E0920771F70DB407FEC0
:10BEA000FDCF8FEF0E94A2538FEF0E94A2530E94FA
:10BEB000A7538B838F71853031F083E18983CE0165
:10BEC0000E949D530AC068E572E0CE010E94AE5305
:10BED000182F811107C087E18983CE010E949D53ED
:10BEE00010E012C020E030E0A9016DE0CE010E9418
:10BEF000C853811104C00E94A753882311F086E122
:10BF0000EBCFCE010E949D53812FDF91CF911F91E6
:10BF10000F910895CF9380917F058823A9F14091D7
:10BF200080055091810560918205709183052DE90E
:10BF30003EE080917D0590917E0580DFC82F8823AB
:10BF400021F140918405509185056091860570919D
:10BF50008705411551056105710589F02DE93EE020
:10BF600080917D0590917E0569DF882359F01092BC
:10BF7000840510928505109286051092870510920F
:10BF80007F058C2FC82F01C0C1E08C2FCF91089561
:10BF9000CF92DF92EF92FF92CF936B017C01C42F7F
:10BFA0008091800590918105A0918205B0918305D3
:10BFB0008C159D05AE05BF05C1F0ACDF811102C037
:10BFC00080E017C02DE93EE0B701A60180917D0514
:10BFD00090917E05CADE882399F3C0928005D092A5
:10BFE0008105E0928205F092830581E0C111809382
:10BFF0007F05CF91FF90EF90DF90CF9008958F92C3
:10C000009F92AF92BF92CF92DF92EF92FF921F93D7
:10C01000CF93DF93C82F2FEA34E130937E0520932E
:10C020007D051092CB1442E050E060E070E0409358
:10C03000B4145093B5146093B6147093B71410925F
:10C040007F05109284051092850510928605109246
:10C0500087054FEF5FEFBA0140938005509381054C
:10C060006093820570938305882349F1853008F039
:10C07000F6C040E060E070E0CB018ADF882309F47D
:10C08000EEC020E1C29FF0011124E55BFF4E8081EC
:10C090008F7709F0E4C044855585668577854436F9
:10C0A00051056105710508F4DAC0C084D184E284C9
:10C0B000F384C114D104E104F10421F4D0C0C12CF3
:10C0C000D12C760140E0C701B60162DF182F88232A
:10C0D00009F4C5C08091A80E9091A90E81159240D7
:10C0E00009F0BDC0A091AD0EAA2309F4B8C080919B
:10C0F000AB0E9091AC0E009709F4B1C04091AA0E1E
:10C10000442309F4ACC0A093C6144093B814E0E0F3
:10C1100050E061E070E0CE2F9B010E2E02C0220F96
:10C12000331F0A94E2F74217530749F021E02E0F1C
:10C13000E83018F02093C11492C0E22FECCFE093C6
:10C14000C1142091B30E3091B40E2115310519F0B0
:10C1500040E050E008C02091C10E3091C20E4091E5
:10C16000C30E5091C40E2093B9143093BA14409367
:10C17000BB145093BC1446015701880E991EA11C94
:10C18000B11C8092C7149092C814A092C914B092A6
:10C19000CA14E091AE0EF091AF0EF093CD14E0937F
:10C1A000CC14B0E00F94402E680D791D8A1D9B1DA4
:10C1B0006093CE147093CF148093D0149093D114C5
:10C1C000A5E0EE0FFF1FAA95E1F7E150FE4FEF2F1C
:10C1D000FF27E695DC01CB018E0F9F1FA11DB11D2E
:10C1E0008093C2149093C314A093C414B093C51445
:10C1F0008090B00E9090B10E8114910419F0A12C92
:10C20000B12C08C08090BD0E9090BE0EA090BF0EC5
:10C21000B090C00EA7019601281B390B4A0B5B0B8F
:10C22000DA01C901880D991DAA1DBB1D0C2E04C081
:10C23000B695A795979587950A94D2F78093BD14E4
:10C240009093BE14A093BF14B093C014853F4FE0E9
:10C250009407A105B10528F48CE08093CB1410E07D
:10C260001AC0853F9F4FA105B10510F480E111C0B0
:10C270008091C90E9091CA0EA091CB0EB091CC0EB8
:10C280008093CE149093CF14A093D014B093D11474
:10C2900080E28093CB14812FDF91CF911F91FF908B
:10C2A000EF90DF90CF90BF90AF909F908F900895C8
:10C2B0008F929F92AF92BF92CF92DF92EF92FF92B6
:10C2C0000F931F93CF93DF93EC016A017B018901E8
:10C2D00089859A85AB85BC850196A11DB11D841702
:10C2E0009507A607B70710F480E054C08F89803106
:10C2F00029F49927872F762F652F0BC08032A1F75D
:10C30000CB01BA0127E096958795779567952A9591
:10C31000D1F78B889C88AD88BE88680D791D8A1DF1
:10C320009B1D8090800590908105A0908205B09023
:10C330008305681579058A059B0581F48F8980310D
:10C3400091F4DD24EE24FF24F601EE0FFF1FE356E7
:10C35000F14F80819181A0E0B0E016C040E018DE8E
:10C360008111ECCFC1CFE894C7F8DD24EE24FF247F
:10C37000F601EE0FFF1FEE0FFF1FE356F14F808116
:10C380009181A281B381BF70F80180839183A283E0
:10C39000B38381E0DF91CF911F910F91FF90EF90D8
:10C3A000DF90CF90BF90AF909F908F9008952F9285
:10C3B0003F924F925F926F927F928F929F92AF9235
:10C3C000BF92CF92DF92EF92FF920F931F93CF9382
:10C3D000DF93EC015B016A018B81811103C08FEF58
:10C3E0009FEFC6C0898180FFFACF49895A896B893E
:10C3F0007C8988859985AA85BB852601612C712C4D
:10C400008A019B01081B190B2A0B3B0B0415150510
:10C410002605370518F46A01C81AD90A76013E01C3
:10C4200024E0620E711CE114F10409F476C0488521
:10C4300059856A857B854A0181E098222B811A0102
:10C440002B01E9E05694479437942794EA95D1F765
:10C45000898D9A8DFC01223049F4628D738D848D13
:10C46000958D620D731D841D951D3CC01481115066
:10C47000122181149104C1F4111116C0452B462BD1
:10C48000472B49F48D899E89AF89B88D8C839D8314
:10C49000AE83BF8309C04C815D816E817F81930132
:10C4A00007DF882309F49BCFE98DFA8D6C817D81AC
:10C4B0008E819F816250710981099109058404C0B0
:10C4C000660F771F881F991F0A94D2F72685378534
:10C4D00040895189620F731F841F951F610F711D61
:10C4E000811D911D20E032E02819390987012E15A0
:10C4F0003F0508F489010115F2E01F0761F520915D
:10C500008005309181054091820550918305621725
:10C5100073078407950719F41EC0C60129C0950149
:10C52000AB01BC0180917D0590917E051EDC8823C6
:10C5300009F455CFA00EB11E88859985AA85BB85C3
:10C54000800F911FA11DB11D88879987AA87BB877E
:10C55000E01AF10A68CF40E01BDD882309F43FCFE1
:10C56000B4016356714FA801C5010F946E31E2CF3B
:10C57000DF91CF911F910F91FF90EF90DF90CF90BF
:10C58000BF90AF909F908F907F906F905F904F90F3
:10C590003F902F900895AF92BF92CF92DF92EF928B
:10C5A000FF920F931F93CF93DF936C01EB017A01FE
:10C5B000DC0113968C911397823070F018960D91D0
:10C5C0001D912D913C911B970F7111272227332725
:10C5D000012B022B032B11F08FEF58C04115510591
:10C5E00011F0F70110821DE040E250E0BE01C601EB
:10C5F000DEDE9C018032910531F081E0232B09F4CD
:10C6000080E0819543C088818823C1F1853E61F334
:10C610008E3251F3E114F10461F19B859F739F30D9
:10C6200041F54A8D5B8D452B21F58F719FEF980F5A
:10C630009530F8F490E00197189F9001199F300D04
:10C640001124FE0180E090E05701A20EB31E853058
:10C65000B8F46181A501480F591FDA016C93019666
:10C6600032968D30910599F7888186FF02C0F501D9
:10C6700015868B8583FDB8CF822F08C080E006C069
:10C680008B3010F46481E6CF6681E4CFDF91CF91E7
:10C690001F910F91FF90EF90DF90CF90BF90AF90E0
:10C6A00008954F925F926F927F92AF92BF92CF9216
:10C6B000DF92EF92FF920F931F93CF93DF93EC01E2
:10C6C0006A017B012B81222349F089899A89AB89F0
:10C6D000BC8984179507A607B70710F480E06BC0E4
:10C6E000223009F463C0C114D104E104F10449F417
:10C6F0001C821D821E821F82188619861A861B863E
:10C7000059C088859985AA85BB85E98DFA8DE5850F
:10C71000F0E03996AC01BD01415051096109710940
:10C720000E2E04C076956795579547950A94D2F7D3
:10C7300097018601015011092109310904C036957C
:10C74000279517950795EA95D2F704171507260739
:10C75000370720F0892B8A2B8B2B49F48D899E89F2
:10C76000AF89B88D8C839D83AE83BF8304C0041BC7
:10C77000150B260B370B280139015E0184E0A80E4A
:10C78000B11C411451046104710481F04C815D813C
:10C790006E817F819501898D9A8D8ADD91E0491A9C
:10C7A0005108610871088111ECCF05C0C886D9868F
:10C7B000EA86FB8681E0DF91CF911F910F91FF9078
:10C7C000EF90DF90CF90BF90AF907F906F905F9091
:10C7D0004F9008954F925F926F927F92AF92BF9267
:10C7E000CF92DF92EF92FF920F931F93CF93DF933D
:10C7F00000D01F92CDB7DEB78C0149835A836B837B
:10C800007C835901C12CD12C7601412CF2E05F2EA2
:10C81000612C712C49815A816B817C819E012F5F33
:10C820003F4FC80145DD882341F1D301C201F80122
:10C83000058404C0880F991FAA1FBB1F0A94D2F752
:10C84000C80ED91EEA1EFB1E49815A816B817C816C
:10C850008789803139F481E0483F5F4F6105710578
:10C8600038F4D8CF81E0483F5F4F6F4F7F4090F260
:10C87000F501C082D182E282F3820F900F900F9077
:10C880000F90DF91CF911F910F91FF90EF90DF906C
:10C89000CF90BF90AF907F906F905F904F90089532
:10C8A0000F931F93CF93DF93EC018B018B81882330
:10C8B00011F080E041C0FB018789803131F1803285
:10C8C000C1F783E08B83F801428D538D648D758DA4
:10C8D0004D8B5E8B6F8B788F9E012F5E3F4FC80113
:10C8E00079DF882331F31A8F098F81E089831C82D5
:10C8F0001D821E821F82188619861A861B861C8638
:10C900001D861E861F86188A17C082E08B831D8AAB
:10C910001E8A1F8A188EFB01408D518D60E070E0E9
:10C92000A5E0440F551F661F771FAA95D1F7498BC5
:10C930005A8B6B8B7C8BD7CFDF91CF911F910F914F
:10C9400008954F925F926F927F928F929F92AF92D3
:10C95000BF92CF92DF92EF92FF920F931F93CF93EC
:10C96000DF93EC014A015B01280139014230510596
:10C970006105710508F462C049855A856B857C851F
:10C980004F5F5F4F6F4F7F4F481559056A057B0515
:10C9900008F454C08F89803129F4FF24EB2CDA2C61
:10C9A000C92C0CC0803209F049C07501640107E050
:10C9B000F694E794D794C7940A95D1F74B895C898C
:10C9C0006D897E89C40ED51EE61EF71E41E0C701A3
:10C9D000B601DEDA882391F19F89903159F49924C8
:10C9E000AA24BB24F401EE0FFF1FE356F14F51823E
:10C9F000408210C0E89487F89924AA24BB24F4014B
:10CA0000EE0FFF1FEE0FFF1FE356F14F40825182E2
:10CA1000628273829A89923090F04D815E816F813B
:10CA200078854C0D5D1D6E1D7F1D409384055093D0
:10CA30008505609386057093870501C080E0DF91CE
:10CA4000CF911F910F91FF90EF90DF90CF90BF900B
:10CA5000AF909F908F907F906F905F904F900895D0
:10CA6000AF92BF92CF92DF92EF92FF920F931F93FC
:10CA7000CF93DF9300D01F92CDB7DEB75C016A0180
:10CA80007B0182E090E0A0E0B0E0F501808391833B
:10CA9000A283B3839E012F5F3F4FB701A601C5015B
:10CAA00007DC811102C080E023C000E010E09801A3
:10CAB000B701A601C50145DF8823A9F3C980DA8043
:10CAC000EB80FC80F5018789803149F481E0F8EF43
:10CAD000CF16FFEFDF06E104F10450F4DBCF81E075
:10CAE00098EFC9169FEFD906E9069FE0F90690F284
:10CAF0000F900F900F900F90DF91CF911F910F919A
:10CB0000FF90EF90DF90CF90BF90AF90089580910D
:10CB1000D5128150823010F080E008951092D51225
:10CB20000F94481B6093DE127093DF128093E01223
:10CB30009093E11281E00895CF93DF93CDB7DEB7F4
:10CB400080915A04811110C09E01275F3F4F4F8191
:10CB5000588562E470E08AE092E00F94F5290E9423
:10CB6000B8D283E080939E02DF91CF910895FF9227
:10CB70000F931F93CF93DF93C091FD0481E0C827EB
:10CB8000D091FE04D827F090FF04F826C11102C00E
:10CB9000DD2319F0EBE2F0E104C0F110FBCF80E0FF
:10CBA00077C084918F010F5F1F4F882321F00E946F
:10CBB0003954F801F6CFE6E6FAE084918F010F5F71
:10CBC0001F4F882321F00E943954F801F6CFCC235F
:10CBD00061F0E4E6FAE084918F010F5F1F4F882334
:10CBE00021F00E943954F801F6CFDD2361F0E2E62E
:10CBF000FAE084918F010F5F1F4F882321F00E947C
:10CC00003954F801F6CFF11003C0E8E5FAE00CC0A2
:10CC1000E0E6FAE084918F010F5F1F4F8823A9F3AC
:10CC20000E943954F801F6CF84918F010F5F1F4F96
:10CC3000882321F00E943954F801F6CFFF2019F023
:10CC40004AE553E002C04FEA53E0DD2319F02CE53A
:10CC500033E002C02FEA33E0CC2319F08EE593E0F5
:10CC600002C08FEA93E05F934F933F932F939F937C
:10CC70008F9386E49AE09F938F931F925DDF8DB729
:10CC80009EB709960FB6F8949EBF0FBE8DBF81E088
:10CC9000DF91CF911F910F91FF9008950F931F93F4
:10CCA0008091D512813019F40F94481B08C060910F
:10CCB000DE127091DF128091E0129091E1120091EA
:10CCC000DA121091DB122091DC123091DD12601B20
:10CCD000710B820B930B28EE33E040E050E00F9491
:10CCE000022E8091D6129091D712A091D812B091B5
:10CCF000D912280F391F4A1F5B1FCA01B9011F91A2
:10CD00000F9108958091D512813099F1823051F4BC
:10CD1000C5DF6093D6127093D7128093D812909388
:10CD2000D91218C01092DA121092DB121092DC1293
:10CD30001092DD121092DE121092DF121092E012A9
:10CD40001092E1121092D6121092D7121092D812AD
:10CD50001092D91281E08093D5120F94481B6093F2
:10CD6000DA127093DB128093DC129093DD1281E073
:10CD7000089580E00895CF92DF92EF92FF92E091C4
:10CD80002505E093DD10C090F106D090F206E0900A
:10CD9000F306F090F406ED5F84E0E89FF0011124C3
:10CDA000E556FB4F2081318142815381C701B60195
:10CDB0000F94922A0F9491306093B1127093B21233
:10CDC0008093B3129093B412C701B6010F94A42FAD
:10CDD0002FB7F8946093230E7093240E8093250E42
:10CDE0009093260E2FBF1092A1121092A2121092B1
:10CDF000A3121092A412FF90EF90DF90CF900895AD
:10CE00008091D512813079F482E08093D5120F940D
:10CE1000481B6093DE127093DF128093E0129093B0
:10CE2000E11281E0089580E00895E82FF0E0EB53EF
:10CE3000F54B849190E0FC013797EC30F105F8F464
:10CE4000EE58FF4F0D944F318091B100887F846080
:10CE50008093B100089580919100887F84608093D1
:10CE6000910008958091A100887F84608093A10043
:10CE7000089580912101887F846080932101089525
:10CE80008F929F92AF92BF92CF92DF92EF92FF92DA
:10CE90000F931F93CF93DF931F921F92CDB7DEB7EF
:10CEA0007C0149018091DE10811148C08B015B013A
:10CEB000A40EB51E0A151B0509F440C0F701C08079
:10CEC000D180F80161918F016983C6016A830F9453
:10CED000E32C6A81681729F1C6010F94EB2CC60177
:10CEE0000F94E32C99818917E1F0EBE2F0E1849152
:10CEF0008F010F5F1F4F882321F00E943954F801E2
:10CF0000F6CFECE2FAE084918F010F5F1F4F882388
:10CF100021F00E943954F801F6CF81E08093DE10B1
:10CF20000DC0BE016F5F7F4FC4010E949C5EF70180
:10CF300080819181019691838083BCCF0F900F9067
:10CF4000DF91CF911F910F91FF90EF90DF90CF90E5
:10CF5000BF90AF909F908F900895AF92BF92CF9265
:10CF6000DF92EF92FF920F931F93CF93DF931F9265
:10CF7000CDB7DEB78C016B017A0159018091DE10CB
:10CF800081111CC0F801808191810F94E32C898369
:10CF9000F60181936F01BE016F5F7F4FC5010E9453
:10CFA0009C5EF801408151814F5F5F4F5183408308
:10CFB000F1E0EF1AF108E114F10421F70F90DF918D
:10CFC000CF911F910F91FF90EF90DF90CF90BF9086
:10CFD000AF900895CF92DF92EF92FF920F931F933D
:10CFE000CF93DF937C018B016A01E9010E9479D321
:10CFF00083E080939E02F0924811E09247111093D3
:10D000004611009345111092411110924211109255
:10D01000431110924411A601662757FD6095762FA3
:10D0200040933D1150933E1160933F117093401116
:10D03000F80180819181AA2797FDA095BA2F80934E
:10D040001F1290932012A0932112B093221281EC10
:10D0500095E79093970280939602D0939506C0939C
:10D06000940610929306DF91CF911F910F91FF903C
:10D07000EF90DF90CF900895CF92DF92EF92FF92E2
:10D080000F931F93CF93DF9300D01F92CDB7DEB7DE
:10D090007C018B01CA01B90129837A838B839C832C
:10D0A0000E9479D323E020939E02F0924811E092EF
:10D0B000471110934611009345112AE037ED43E2E2
:10D0C0005CE369817A818B819C810F94922A0F9411
:10D0D000A42F609341117093421180934311909358
:10D0E00044110F94332A6B017C019B01AC0160E079
:10D0F00070E887E794E40F945F2E0F94A42F609359
:10D100003D1170933E1180933F11909340112AE09E
:10D1100037ED43E25CE3F8016081718182819381A4
:10D120000F94922AA70196010F945F2E0F94A92FB6
:10D1300060931F12709320128093211290932212F9
:10D1400084E992E790939702809396020F900F9054
:10D150000F900F90DF91CF911F910F91FF90EF9063
:10D16000DF90CF900895EF92FF920F931F93CF938C
:10D17000DF937C018B01EA010E9479D383E08093E5
:10D180009E02F0924811E0924711109346110093CD
:10D19000451184EF91E0A0E0B0E0809341119093BD
:10D1A0004211A0934311B093441188EE9FE3AFE086
:10D1B000B0E080933D1190933E11A0933F11B09346
:10D1C000401120E030E048EC52E4F80160817181C8
:10D1D000828193810F94922A20E030E04AEF53E459
:10D1E0000F945F2E0F94A92F60931F12709320123B
:10D1F000809321129093221287E493E790939702F1
:10D2000080939602D0939506C0939406109293064D
:10D21000DF91CF911F910F91FF90EF900895AF9202
:10D22000BF92CF92DF92EF92FF920F931F93CF9313
:10D23000DF9300D01F92CDB7DEB77C015B0129835D
:10D240003A834B835C830E9479D383E080939E0270
:10D25000F0924811E0924711B0924611A092451108
:10D2600029813A814B815C81CA01B9010F94312A2D
:10D270002AE037ED43E25CE30F94922A0F94A42F47
:10D280006093411170934211809343119093441124
:10D290000F94332A6B017C019B01AC0160E070E8C4
:10D2A00087E794E40F945F2E0F94A42F60933D11B1
:10D2B00070933E1180933F1190934011F50160816E
:10D2C0007181828193810F94312A2AE037ED43E204
:10D2D0005CE30F94922AA70196010F945F2E0F949E
:10D2E000A92F60931F1270932012809321129093A4
:10D2F000221286ED91E79093970280939602109305
:10D30000950600939406109293060F900F900F903D
:10D310000F90DF91CF911F910F91FF90EF90DF90D1
:10D32000CF90BF90AF9008958F929F92AF92BF928F
:10D33000CF92DF92EF92FF92CF9320E030E04AE766
:10D3400054E4FC0160817181828193810F94922A5F
:10D350000F94A42F6B017C01611571058105910566
:10D3600061F097FF0AC0F094E094D094C094C11C7F
:10D37000D11CE11CF11C8DE201C080E28093840E7F
:10D38000C701B60128EE33E040E050E00F94242EB0
:10D390009AE0892E912CA12CB12CCA01B901A501CA
:10D3A00094010F94242E605D6093850E8EE280932D
:10D3B000860EC701B60124E630E040E050E00F944D
:10D3C000242ECA01B901A50194010F94242E605D99
:10D3D0006093870EC701B601A50194010F94242E16
:10D3E000C62FCA01B901A50194010F94242E605DD6
:10D3F0006093880EC05DC093890E84E89EE0CF9153
:10D40000FF90EF90DF90CF90BF90AF909F908F9064
:10D4100008950F931F93CF93DF938C01EBE2F0E11C
:10D420008491EF012196882321F00E943954FE0156
:10D43000F7CFB8018FE19AE00E9442C982E20E94D0
:10D4400039548AE00E94395481E0DF91CF911F91D5
:10D450000F910895CF92DF92FF920F931F93CF9376
:10D46000DF931F921F92CDB7DEB76901DB011296E1
:10D470000D911C911397423309F471C0B8F44531F2
:10D4800009F47AC0473109F48BC0443109F0A1C0D6
:10D49000D80115962C9115971696ED91FC9117973A
:10D4A000CF01820F911D820F911D5EC0463409F499
:10D4B00087C0473409F488C04B3309F08AC0F901AA
:10D4C00081819381913029F0933031F4282F885055
:10D4D00004C028E0280F01C0282F31E0D80113969E
:10D4E0004C91481708F430E051E0F80142812417CC
:10D4F00008F450E041E0281708F040E0832F842B27
:10D5000085233423832B09F464C0D6011296FC9042
:10D51000913039F070F0923039F0933041F020E0E2
:10D5200001C021E030E007C020E03FEF04C02FEF52
:10D53000F9CF20E031E0F7FE08C0B601C8012A8328
:10D5400039830F94E91939812A81F6018081830F8B
:10D5500080838181820F8183FF0C69F73AC0B90112
:10D56000C8010F94E91935C01192E817F907E1F7DE
:10D57000C8010F94141A2DC0C8010F94FE198823F6
:10D5800051F1F80125810680F781E02DCF01820F4E
:10D59000911D820F911D1192E817F907E1F719C04B
:10D5A000D9011C92F801828111968C931197858183
:10D5B000815012968C931297838113968C9309C095
:10D5C000D80115968C9103C0D80111968C91F60163
:10D5D000808381E001C080E00F900F90DF91CF91B8
:10D5E0001F910F91FF90DF90CF9008956F927F92DF
:10D5F0008F929F92AF92BF92CF92DF92EF92FF9263
:10D600000F931F93CF93DF935C017B01942E6901ED
:10D610008AE0481709F471C0A5E14A134AC0DB014A
:10D620001296ED91FC9113978280C681D781A49ABE
:10D630000F941B1A80EE782E780C90E1692E680CFE
:10D6400088EF0E94734B0F941B1ABFE1B81508F4C2
:10D6500043C0882D807780680E94734B882D829507
:10D66000807F0E94734B0F941B1A80E80E94734BBB
:10D6700080E00E94734B0F941B1A8AEF0E94734B39
:10D680000F941B1A8E01005F1F4F8881807F0E94BC
:10D69000734B89918295807F0E94734B0C171D07F5
:10D6A000A1F7E8010F941B1A839473948610C8CFD6
:10D6B000A4989601492DB701C501DF91CF911F9123
:10D6C0000F91FF90EF90DF90CF90BF90AF909F9021
:10D6D0008F907F906F90BECE872D807780680E945C
:10D6E000734B872D8295807F0E94734B0F941B1A7A
:10D6F00080E80E94734B80E8BCCF9C9AA4989B9AC8
:10D70000A398809104018460809304019FB7F894EA
:10D71000809105018460809305019FBFA49A0F94B6
:10D720001B1A88E790E00F94201A88EF0E94734B31
:10D730000F941B1A80E00E94734B80E80E94734B89
:10D740000F941B1A80E00E94734B80E10E94734B80
:10D750000F941B1A8FE090E00F94201A80E30E9430
:10D76000734B80EE0E94734B0F941B1AD0E08D2FE9
:10D77000807780680E94734B8D2F8295807F0E94F6
:10D78000734B0F941B1A80E80E94734B80E00E9439
:10D79000734B0F941B1A8AEF0E94734B0F941B1A42
:10D7A000C0E280E00E94734B80E00E94734B0F94B4
:10D7B0001B1AC150B1F788EF0E94734B0F941B1ACC
:10D7C000DF5FD032A1F680E00E94734B80EC0E94B4
:10D7D000734B0F941B1AA4986CCFDF92EF92FF92B9
:10D7E0000F931F93CF93DF93CDB7DEB76E970FB62E
:10D7F000F894DEBF0FBECDBF609121097091220960
:10D800006115710509F14DE150E08E010F5F1F4F69
:10D81000C8010F949E291E8EF8017F01E01AF10ABB
:10D82000D190DD2019F08AE0D812F7CFF801EE0D83
:10D83000FF1D108260E0C8010E94F854882321F087
:10D84000C801E7DD811109C081E0209121093091F3
:10D850002209232BA9F480E013C0DD2051F08FEFC3
:10D86000E81AF80A80912109909122098E0D9F1DD6
:10D8700002C080E090E09093220980932109E4CFD8
:10D880006E960FB6F894DEBF0FBECDBFDF91CF917D
:10D890001F910F91FF90EF90DF900895CF92DF924C
:10D8A000EF92FF920F931F93CF93DF93CDB7DEB725
:10D8B000CDB6DEB6FC0101900020E9F7E81BF90BBC
:10D8C00034962DB73EB72E1B3F0B0FB6F8943EBFD4
:10D8D0000FBE2DBF0DB71EB70F5F1F4F9F938F93C6
:10D8E00083E79BE09F938F931F930F930F94C72918
:10D8F000780134E0E30EF11C0F900F900F900F9021
:10D900000F900F90F7018081882339F090E00F94F9
:10D910005931F70181937F01F5CF60E0C8010E9482
:10D92000F854882311F0C80174DD8FE69BE09093D2
:10D9300022098093210951DF0FB6F894DEBE0FBE95
:10D94000CDBEDF91CF911F910F91FF90EF90DF90AF
:10D95000CF900895AF92BF92CF92DF92EF92FF9255
:10D960000F931F93CF93DF93CDB7DEB76F970FB6AB
:10D97000F894DEBF0FBECDBF80919E02811105C01D
:10D9800080911B12882309F4ABC189E593E1909340
:10D9900058138093571381E080939015109292153D
:10D9A0001092911540E050E0BA018DE593E10E949C
:10D9B000516380915713909158132BE1FC013496D9
:10D9C000DE01159601900D922A95E1F7FC01828106
:10D9D00093819C838B8380E793E09A83898340E0E3
:10D9E00050E0BE016F5F7F4F8FEA93E00E94C298C4
:10D9F000CE0101960E94845DE0909115F090921501
:10DA00001092231280911F1290912012A091211246
:10DA1000B091221281309048A105B10540F01092DA
:10DA20001F12109220121092211210922212D090E6
:10DA30001F12409188061416DCF4842F992787FD65
:10DA4000909501972D2D332727FD309528173907FD
:10DA50007CF0DD24DA94D40E8D2D90E0A0E0B0E0CF
:10DA600080931F1290932012A0932112B093221240
:10DA700010921D1280911C12D81614F4D0921C1210
:10DA800080911C12992787FD909504962D2D3327A0
:10DA900027FD30958217930724F48CEF8D0D80932A
:10DAA0001C12C0901C12B12C21E0E21AF108C11026
:10DAB0001BC080911B12811105C080919E0288239A
:10DAC00099F009C0D110F9CF0E946DD480911D1238
:10DAD000882399F305C181E0D11080E024E04DE96D
:10DAE0005BE06B2D0E9493FE67EE72E18DE593E1A2
:10DAF0000E94EAFF8091E7128F3209F181E0C8129B
:10DB00001CC080911B12811105C080919E02882348
:10DB1000A1F00AC091E0D912F8CF0E94B3FC809125
:10DB20001D12882391F3DCC081E0D81280E020E24E
:10DB300049E95BE06B2D0E9493FE82E001C081E029
:10DB40008701AA24A394AC0C0F3FFFEF1F0709F431
:10DB5000C0C0C812BAC060E070E0C8010E94DA9A82
:10DB60009091E61280911B12992309F492C08823A8
:10DB700009F486C0DC1084C01D8218861C821B82BA
:10DB800080E793E09A83898380916013811103C0B9
:10DB900008E313E102C009E513E17801E4E0EE0EC9
:10DBA000F11C21E047EE52E1B701CE0105960E943B
:10DBB000905C811127C0EBE2F0E184918F010F5F4F
:10DBC0001F4F882321F00E943954F801F6CFE3E873
:10DBD000FBE084918F010F5F1F4F811103C007EE9F
:10DBE00012E104C00E943954F801F3CFF801819189
:10DBF0008F01882319F00E943954F8CF8AE00E94DF
:10DC000039542BC08091AE148A30C0F491E0980F43
:10DC10009093AE14FFE18F9FC001112488589C4E51
:10DC20002BE1F701DC01149601900D922A95E1F7A2
:10DC3000F80122813381FC01338322838BE1FE01D1
:10DC40003596ADE5B3E101900D928A95E1F78B81B0
:10DC50009C8190935C1380935B13CE0101960E948C
:10DC6000845D10921F1210922012109221121092B5
:10DC7000221281E080931D1283E080939E0230C0C7
:10DC800080919E028823F9F081E0DC1080E041E081
:10DC900017C0811105C080919E028823A1F00CC09D
:10DCA000DC10F9CF87EE92E1F9DD0E9467D4809114
:10DCB0001D12882381F314C081E0DC1080E040E075
:10DCC0006B2D0E941AFE8A2D01C08F5F0150110931
:10DCD0003BCFB394C39425E0B212E9CE809388067B
:10DCE0006F960FB6F894DEBF0FBECDBFDF91CF9118
:10DCF0001F910F91FF90EF90DF90CF90BF90AF906A
:10DD000008957F928F929F92AF92BF92CF92DF92AF
:10DD1000EF92FF920F931F93CF93DF93CDB7DEB7B0
:10DD2000AA970FB6F894DEBF0FBECDBF8091371310
:10DD30008F93809136138F938AE79BE09F938F9305
:10DD40008E010F5D1F4F1F930F930F94C7290F90E4
:10DD50000F900F900F900F900F90D12CF801019021
:10DD60000020E9F73197E01BF10BDE1674F478011F
:10DD7000ED0CF11CD7FCFA94F701808190E00F9430
:10DD80005931F7018083D394E9CF40E050E0BA01E4
:10DD90008CE393E10E945163912CCE0101967C01AA
:10DDA00040E050E0B7018CE393E10E94CB6218168B
:10DDB0008CF5F70101900020E9F73197EE19FF0982
:10DDC000C12CD12C8E2E77247A947E0E872D8C191F
:10DDD0008C1481F05701A80EB11C87FDBA94F5018F
:10DDE000808190E00F945931F5018083FFEFCF1AC5
:10DDF000DF0AECCF8A858E3799F245E050E0B80112
:10DE0000C7010F94A731892B59F6C80147DD992422
:10DE10009394C6CF911003C08FEF9FEF05C0809100
:10DE200036139091371301969093371380933613DE
:10DE3000AA960FB6F894DEBF0FBECDBFDF91CF918B
:10DE40001F910F91FF90EF90DF90CF90BF90AF9018
:10DE50009F908F907F9008958091300583FD1DC025
:10DE60008091BE04811119C0E0912505F0E0EE0F0C
:10DE7000FF1FE45AF14F2081318180914E02909131
:10DE80004F02281739074CF40E9479D340E050E044
:10DE9000BA0182E99BE90C940FD481E08093DE11F2
:10DEA00040E050E0BA018FE79CE90E940FD487E67A
:10DEB0009BE090932209809321098FCC83E69BE01D
:10DEC000909322098093210988DC6FEF82E69BE022
:10DED0000C94E7D26F927F928F929F92AF92BF92F3
:10DEE000DF92EF92FF920F931F93CF93DF93CDB703
:10DEF000DEB7AD970FB6F894DEBF0FBECDBF7C0185
:10DF0000D62E8091E512882309F4F8C18091D914A6
:10DF1000882309F49EC0442309F4C5C18091F114FB
:10DF2000882329F1E0EFFFE084918F010F5F1F4FFD
:10DF3000882321F00E943954F801F6CFEFE1FBE08D
:10DF400084918F010F5F1F4F882321F00E94395465
:10DF5000F801F6CF61E070E080E090E00E9480C1BF
:10DF60008AE00E94395486E19BE00E94BA788FE2F1
:10DF70008093F614B12C21E007EF14E14FE1A42EB9
:10DF80008091AE14B816B8F4AB9CC0011124B8014E
:10DF900084589C4E2DA70E94EAFFC8012DA58C0134
:10DFA0000196F8013081332321F02D3810F42F5FD2
:10DFB000F6CFB394E5CF27FD06C0B80186ED94E116
:10DFC0000E94EAFF02C0F8011082EBE2F0E18491C6
:10DFD0008F010F5F1F4F882321F00E943954F801F1
:10DFE000F6CFB7018DEF9AE00E9442C96091F1141B
:10DFF000FDE86F9FB00111246A507B4E82EF9AE0DA
:10E000000E9442C9409187155091881560918915E9
:10E0100070918A158CEE9AE00E9425C28AE00E94D7
:10E0200039548091F11494E0899FF0011124EE504D
:10E03000FB4E40918715509188156091891570911C
:10E040008A1540835183628373838F5F8093F114B9
:10E050000DC01092F11432E0B32E27C1B7018FED3D
:10E060009AE00E9442C98AE00E9439540E94455BAE
:10E070001D8218861C821B8280E793E09A83898325
:10E0800088E393E19093581380935713F7018081AD
:10E090008F3209F06DC087010F5F1F4FCE010196CF
:10E0A0003C010115110509F469C06FE270E0C80177
:10E0B0000F9495315C01009709F461C008171907A6
:10E0C00008F05DC04C01801A910AA401B801CE018C
:10E0D00080960F94B531E0E2F0E0EC0FFD1FE80D03
:10E0E000F91D10828E01005E1F4FF80181918F0192
:10E0F000882319F00E943954F8CF8AE00E943954DD
:10E1000060915713709158136115710519F06C5F88
:10E110007F4F02C060E070E021E0AE01405E5F4FE3
:10E12000CE0105960E94905C81111AC0EBECFAE0DA
:10E1300084918F010F5F1F4F811104C08E01005E1B
:10E140001F4F04C00E943954F801F2CFF8018191A9
:10E150008F01882319F00E943954F8CF8EE28CC0C9
:10E16000709258136092571385010F5F1F4F99CF1C
:10E1700089E593E190935813809357138701609139
:10E18000571370915813DD2009F45DC061157105B6
:10E1900019F06C5F7F4F02C060E070E021E0A801E1
:10E1A00086ED94E10E94905C882309F448C0809138
:10E1B000E7149091E814A091E914B091EA148093C7
:10E1C000831590938415A0938515B0938615B80197
:10E1D0008DEB9AE00E9442C94091831550918415BD
:10E1E000609185157091861585EB9AE00E9425C295
:10E1F0008AE00E9439541092871510928815109267
:10E20000891510928A15E6EAFAE084917F019FEF62
:10E21000E91AF90A882321F00E943954F701F5CF51
:10E22000B80180E090E00E94DA9A8091F4128111A6
:10E2300002C0C80102C084EF92E160E02DC0B801C5
:10E2400082E99AE013C06115710519F06C5F7F4F88
:10E2500002C060E070E026E5A80186ED94E10E942E
:10E26000905C81110CC0B8018EE79AE00E9442C90F
:10E270008EE20E9439548AE00E9439540FC081E036
:10E280008093E212B7018CE69AE00E9442C98AE0CC
:10E290000E94395460E0C8010E94D7D2CE01019695
:10E2A0000E94845D2BC0BB24B394EBE2F0E1849127
:10E2B0008F010F5F1F4F882321F00E943954F8010E
:10E2C000F6CFE7EEFAE084918F010F5F1F4F8823AE
:10E2D00021F00E943954F801F6CFE1E0BE1203C0EC
:10E2E00006E613E002C000E613E0F80181918F0119
:10E2F000882309F4B3CE0E943954F7CFAD960FB6F8
:10E30000F894DEBF0FBECDBFDF91CF911F910F916B
:10E31000FF90EF90DF90BF90AF909F908F907F9095
:10E320006F9008950F931F93CF93DF93CDB7DEB710
:10E3300028970FB6F894DEBF0FBECDBF8823C9F073
:10E3400083E992E098878F8304E610E01A830983BB
:10E35000BE01695F7F4FCE0101960E94B97C8AEBB6
:10E3600092E09E838D831A830983BE016B5F7F4F8A
:10E370000BC088EB91E09C838B8384E190E09A83CF
:10E380008983BE016D5F7F4FCE0101960E94B97CEB
:10E3900028960FB6F894DEBF0FBECDBFDF91CF91A8
:10E3A0001F910F9108950E9441C2BCCFCF92DF927E
:10E3B000EF92FF921F93CF93DF9300D01F92CDB7C0
:10E3C000DEB780911F1290912012A0912112B0917E
:10E3D0002212B7FF08C010921F1210922012109242
:10E3E00021121092221280913D1190913E11A09124
:10E3F0003F11B091401140911F1250912012609135
:10E4000021127091221284179507A607B70744F4CA
:10E4100080931F1290932012A0932112B093221286
:10E4200080919E02882359F160911F1270912012F1
:10E430008091211290912212C0904111D0904211EE
:10E44000E0904311F09044116C0D7D1D8E1D9F1DB9
:10E450000F94312A20E030E048EC52E40F94922AE5
:10E4600069837A838B839C83CE0101960E94A0CA24
:10E47000BC0180914711909148110E94279580918D
:10E480001B1210919306811106C01123C1F18091D6
:10E490009E028823A1F160911F1270912012809139
:10E4A000211290912212C0904111D0904211E0901F
:10E4B0004311F09044116C0D7D1D8E1D9F1D0F9416
:10E4C000312A20E030E048EC52E40F94922A0F9475
:10E4D000A92FE0914511F0914611309721F060830A
:10E4E000718382839383112329F0E0919406F09144
:10E4F0009506199580911B1281110E946DD480910F
:10E500001B12882329F0E0919406F0919506199545
:10E510000F900F900F900F90DF91CF911F91FF9070
:10E52000EF90DF90CF900895CF92DF92EF92FF921D
:10E530001F93CF93DF9300D01F92CDB7DEB78091AA
:10E540001F1290912012A0912112B0912212B7FFB8
:10E5500008C010921F1210922012109221121092D5
:10E56000221280913D1190913E11A0913F11B091E6
:10E57000401140911F125091201260912112709110
:10E58000221284179507A607B70744F480931F1239
:10E5900090932012A0932112B093221280919E0298
:10E5A000882359F160911F127091201280912112DD
:10E5B00090912212C0904111D0904211E0904311ED
:10E5C000F09044116C0D7D1D8E1D9F1D0F94332AFC
:10E5D00020E030E048EC52E40F94922A69837A8379
:10E5E0008B839C83CE0101960E94A0CABC018091BE
:10E5F0004711909148110E94279580911B1210910C
:10E600009306811106C01123B1F180919E028823E7
:10E6100091F160911F1270912012809121129091BE
:10E620002212C0904111D0904211E0904311F0901D
:10E6300044116C0D7D1D8E1D9F1D0F94332A20E00B
:10E6400030E048EC52E40F94922AE0914511F091A9
:10E650004611309721F06083718382839383112365
:10E6600029F0E0919406F0919506199580911B127E
:10E6700081110E946DD40F900F900F900F90DF9139
:10E68000CF911F91FF90EF90DF90CF900895CF92A0
:10E69000DF92EF92FF921F93CF93DF9300D01F92F0
:10E6A000CDB7DEB780911F1290912012A091211258
:10E6B000B0912212B7FF08C010921F1210922012C0
:10E6C000109221121092221280913D1190913E11D0
:10E6D000A0913F11B091401140911F125091201212
:10E6E000609121127091221284179507A607B7072F
:10E6F00044F480931F1290932012A0932112B093A0
:10E70000221280919E02882359F160911F1270910C
:10E7100020128091211290912212C0904111D0902C
:10E720004211E0904311F09044116C0D7D1D8E1D3F
:10E730009F1D0F94332A2AE037ED43E25CE30F94E8
:10E74000922A69837A838B839C83CE0101960E94EF
:10E750006AC9BC0180914711909148110E94279588
:10E7600080911B1210919306811106C01123B1F103
:10E7700080919E02882391F160911F127091201266
:10E780008091211290912212C0904111D09042119B
:10E79000E0904311F09044116C0D7D1D8E1D9F1D66
:10E7A0000F94332A2AE037ED43E25CE30F94922A78
:10E7B000E0914511F0914611309721F0608371830B
:10E7C00082839383112329F0E0919406F0919506BA
:10E7D000199580911B1281110E946DD480911B129A
:10E7E000882329F0E0919406F091950619950F90F1
:10E7F0000F900F900F90DF91CF911F91FF90EF90AE
:10E80000DF90CF900895CF92DF92EF92FF921F9307
:10E81000CF93DF9300D01F92CDB7DEB780911F1248
:10E8200090912012A0912112B0912212B7FF08C03E
:10E8300010921F1210922012109221121092221286
:10E8400080913D1190913E11A0913F11B0914011E6
:10E8500040911F125091201260912112709122124A
:10E8600084179507A607B70744F480931F12909367
:10E870002012A0932112B093221280919E0288232D
:10E8800059F160911F127091201280912112909184
:10E890002212C0904111D0904211E0904311F090AB
:10E8A00044116C0D7D1D8E1D9F1D0F94332A2AE08F
:10E8B00037ED43E25CE30F94922A69837A838B837A
:10E8C0009C83CE0101960E941FCABC018091471112
:10E8D000909148110E94279580911B1210919306E8
:10E8E000811106C01123B1F180919E02882391F11C
:10E8F00060911F127091201280912112909122122A
:10E90000C0904111D0904211E0904311F090441119
:10E910006C0D7D1D8E1D9F1D0F94332A2AE037ED4F
:10E9200043E25CE30F94922AE0914511F091461185
:10E93000309721F06083718382839383112329F0C0
:10E94000E0919406F0919506199580911B12811122
:10E950000E946DD40F900F900F900F90DF91CF9188
:10E960001F91FF90EF90DF90CF9008950F931F932A
:10E97000CF9380911F1290912012A0912112B091FB
:10E980002212B7FF08C010921F121092201210928C
:10E9900021121092221280913D1190913E11A0916E
:10E9A0003F11B091401140911F125091201260917F
:10E9B00021127091221284179507A607B70744F415
:10E9C00080931F1290932012A0932112B0932212D1
:10E9D00080919E02882311F160911F127091201284
:10E9E00080912112909122120091411110914211B7
:10E9F0002091431130914411600F711F821F931FAA
:10EA00000F94332A0F94A42FCB010E94F3CBBC01A7
:10EA100080914711909148110E94279580911B1277
:10EA2000C0919306811106C0CC23A1F180919E0272
:10EA3000882381F160911F12709120128091211220
:10EA40009091221200914111109142112091431195
:10EA500030914411600F711F821F931F0F94332A4E
:10EA6000E0914511F0914611309721F06083718358
:10EA700082839383CC2329F0E0919406F09195064C
:10EA8000199580911B12882329F0CF911F910F9126
:10EA90000C946DD4CF911F910F91089580911F1206
:10EAA00090912012A0912112B0912212B7FF08C0BC
:10EAB00010921F1210922012109221121092221204
:10EAC00080913D1190913E11A0913F11B091401164
:10EAD00040911F12509120126091211270912212C8
:10EAE00084179507A607B70744F480931F129093E5
:10EAF0002012A0932112B093221280919E028823AB
:10EB000099F0209141113091421180911F12909102
:10EB10002012820F931F0E94F3CBBC0180914711FA
:10EB2000909148110E94279580911B124091930665
:10EB3000811106C0442311F180919E028823F1F0D7
:10EB4000809141119091421120911F123091201219
:10EB5000820F931FE0914511F0914611309711F00B
:10EB600091838083442329F0E0919406F0919506E7
:10EB7000199580911B1281110E946DD480911B12F6
:10EB800008958CDF882329F0E0919406F091950692
:10EB90001994089583CFCF93DF93C82F80911B12D0
:10EBA000882321F0DF91CF910C946DD460911F12D6
:10EBB000709120128091211290912212611571059D
:10EBC0008105910579F10F94332A20918F063091B8
:10EBD000900640919106509192060F94922A9B01C3
:10EBE000AC016091F1067091F2068091F30690916C
:10EBF000F4060F94602E6093F1067093F2068093F2
:10EC0000F3069093F40610921F12109220121092A5
:10EC10002112109222126C2F83E00E943CD381E0DB
:10EC200080939E0280919E02882389F0C13019F062
:10EC3000C9EADCE002C0CFE9DCE081EF96E00E94A7
:10EC400042CBBC01CE01DF91CF910C942795DF918F
:10EC5000CF91089581E09FCF8FEF9DCF3F924F924C
:10EC60005F926F927F928F929F92AF92BF92CF925C
:10EC7000DF92EF92FF920F931F93CF93DF9300D019
:10EC800000D0CDB7DEB78C01362E80911B128823C1
:10EC9000C9F026960FB6F894DEBF0FBECDBFDF9148
:10ECA000CF911F910F91FF90EF90DF90CF90BF9089
:10ECB000AF909F908F907F906F905F904F903F901C
:10ECC0000C946DD480911F1290912012A09121126A
:10ECD000B0912212892B8A2B8B2B09F493C00F94AD
:10ECE000541B932DA4E09A02C00111249E838D83AE
:10ECF000FC01EB51F94F408051806280738080911C
:10ED00004D0281110BC020E030E04AE754E4C3011A
:10ED1000B2010F94602E6B017C0108C0ED81FE8171
:10ED2000E05BFD4FC080D180E280F38080911F12B4
:10ED300090912012A0912112B091221289839A837E
:10ED4000AB83BC83BC01CD010F94332A20918F0685
:10ED50003091900640919106509192060F94922A1C
:10ED60009B01AC01C301B2010F94602E4B015C0109
:10ED7000AD81BE81AB51B94FBE83AD83FD016083D0
:10ED800071838283938389819A81AB81BC81B7FF30
:10ED900013C020E030E04AE754E4C301B2010F940D
:10EDA0005F2E6B017C019B01AC01C501B4010F9486
:10EDB0002D2A87FF18C010C089819A81AB81BC8140
:10EDC000892B8A2B8B2B79F0A7019601C501B40101
:10EDD0000F94863018163CF4AD81BE81CD92DD9241
:10EDE000ED92FC9213976FEF832D0E943CD310920B
:10EDF0001F1210922012109221121092221281E002
:10EE000080939E0280919E02882309F442C02DECDB
:10EE10003CEC4CEC5DE360918F0670919006809124
:10EE20009106909192060F948630232D332727FD6B
:10EE3000309587FD0AC0C901880F991F880F991F57
:10EE40008B51994F0E9442CB09C0C901880F991F6D
:10EE5000880F991F8B51994F0E949469BC01C8017A
:10EE600026960FB6F894DEBF0FBECDBFDF91CF91CF
:10EE70001F910F91FF90EF90DF90CF90BF90AF90D8
:10EE80009F908F907F906F905F904F903F900C94E9
:10EE9000279526960FB6F894DEBF0FBECDBFDF9143
:10EEA000CF911F910F91FF90EF90DF90CF90BF9087
:10EEB000AF909F908F907F906F905F904F903F901A
:10EEC000089562E088E99CE0C9CE61E081E99CE0B8
:10EED000C5CE60E08AE89CE0C1CE8F929F92AF924F
:10EEE000BF92CF92DF92EF92FF920F931F93CF9337
:10EEF000DF9300D01F92CDB7DEB780911B1288231D
:10EF000009F448C080918C0290918D021816190660
:10EF10000CF03BC09A8389839E012D5F3F4F44E0F4
:10EF200050E06AEA70E1CE0101960E944067EBE290
:10EF3000F0E184917F019FEFE91AF90A882321F01B
:10EF40000E943954F701F5CF4091AA105091AB10AF
:10EF50006091AC107091AD1085EB9BE00E9490D455
:10EF600060918C0270918D0284EA9BE00E940CC239
:10EF7000E2EAFBE084917F019FEFE91AF90A882316
:10EF800021F00E943954F701F5CF1092DE110E9452
:10EF90006DD4DFC081E08093DE1180901F129090CD
:10EFA0002012A0902112B090221281149104A10489
:10EFB000B10409F457C010921F121092201210923F
:10EFC000211210922212B401882777FD8095982F84
:10EFD0000F94332A209102073091030740910407D0
:10EFE000509105070F94922A2091AA103091AB10EE
:10EFF0004091AC105091AD100F94602E6B017C01CC
:10F0000020E030E040E050EC0F94863087FD2AC0CD
:10F0100020E030E040EA50E4C701B6010F942D2A09
:10F02000181604F18091E404882371F08091D706CA
:10F03000882351F08091560E9091570E880D991D9E
:10F040009093570E8093560EC092AA10D092AB1098
:10F05000E092AC10F092AD1081E00F943D0382E09D
:10F0600080939E0280919E02882349F08AEA90E173
:10F070000E949469BC0181E89CE00E942795C090A1
:10F08000AA10D090AB10E090AC10F090AD10809032
:10F090008B0690908C06A0908D06B0908E06A501F0
:10F0A0009401C701B6010F942D2A8823C9F0A50148
:10F0B0009401C701B6010F94863018161CF481E044
:10F0C00090E002C08FEF9FEF90938A0680938906AD
:10F0D000C0928B06D0928C06E0928D06F0928E063E
:10F0E00064E080918906681B09E61CE02CE042E0A0
:10F0F00082E40E94475E06E61CE021E043E064E112
:10F100008CE30E94475E06E31CE020E143E06FE2EF
:10F1100085E00E94475E06E01CE020E143E06FE2EC
:10F120008AE50E94475E60E380918906681B0CEEC9
:10F130001BE02DE042E08EE60E94475E61E3809195
:10F140008906681B02ED1BE02DE042E089E10E9488
:10F15000475E0F900F900F900F90DF91CF911F910E
:10F160000F91FF90EF90DF90CF90BF90AF909F9066
:10F170008F900895EC01E0EFFFE084918F010F5F25
:10F180001F4F882321F00E943954F801F6CFEFEC8D
:10F19000FCE084918F010F5F1F4F882321F00E94B4
:10F1A0003954F801F6CF0F9415040F9474170E9488
:10F1B0005B9761E0CE010E94E7D20E9467D40F9472
:10F1C000330084E00E9435C880913412869586957C
:10F1D00010926A1280936B120E94EAC880913412D6
:10F1E00086958695880F10926A1280936B1280EC38
:10F1F0009CE00E947EC88091341286958695982F57
:10F20000990F980F10926A1290936B1283EB9CE007
:10F210000E947EC80E94A7C78111D3CF2FEF8BE435
:10F220009DE1215080409040E1F700C00000F8943B
:10F230002FEF84E39CE0215080409040E1F700C034
:10F2400000000F941504A895FECF60E08091600E39
:10F250009091610E0E943C506093D7047093D80443
:10F260008093D9049093DA0461E08091620E9091CA
:10F27000630E0E943C506093DB047093DC04809327
:10F28000DD049093DE0480915A0E90915B0E0E94F3
:10F29000D94C6093DF047093E0048093E104909371
:10F2A000E204A8958FB7F8941092640E8FBF08956A
:10F2B000CF92DF92FF920F931F93CF93DF931F9212
:10F2C0001F92CDB7DEB7F82E6A01809164028823C1
:10F2D00009F441C0E0EFFFE084918F010F5F1F4F01
:10F2E000882341F069837A830E943954F801698147
:10F2F0007A81F2CFFB0184918F010F5F1F4F88232A
:10F3000021F00E943954F801F6CFE4EFFCE084913B
:10F310008F010F5F1F4F882321F00E943954F8019D
:10F32000F6CFF7FC0CC06F2D772767FD7095872F00
:10F33000972F0E9480C18AE00E9439540CC0EFEEE2
:10F34000FCE084918F010F5F1F4F882321F00E9402
:10F350003954F801F6CF80919606811107C01092BA
:10F36000640281E080939606C60104DF0F900F903F
:10F37000DF91CF911F910F91FF90DF90CF900D946F
:10F3800015042F923F924F925F926F927F928F92CD
:10F390009F92AF92BF92CF92DF92EF92FF920F9324
:10F3A0001F93CF93DF9300D01F92CDB7DEB74C01F0
:10F3B0001B0129833A834B835C8327013801D7FEE5
:10F3C00012C08091820E882309F4A7C0F401108234
:10F3D00010929F061092A0061092A1061092A2060B
:10F3E00002E010E015C0F601E750FE4E8081882350
:10F3F00009F4BEC0F4011082F601EE0FFF1FEE0FFC
:10F40000FF1FE956F94F1082118212821382860182
:10F41000F40180818230E1F0833009F455C08130FD
:10F4200009F0A8C0F801EE0FFF1FEE0FFF1FE9560D
:10F43000F94F208131814281538169817A818B81A9
:10F440009C810F942D2A87FD95C082E0F401808372
:10F45000000F111F000F111F0956194FB501882702
:10F4600077FD8095982F0F94332A9B01AC01F8010A
:10F4700060817181828193810F945F2E9B01AC0129
:10F4800069817A818B819C810F94863087FD0CC0C5
:10F490000F94481B6856754C8F4F9F4FF101608346
:10F4A00071838283938366C00F94481BF1010081AE
:10F4B000118122813381601B710B820B930B97FDAD
:10F4C00059C083E0F4018083FFEFCF16DF0631F0EF
:10F4D000C114D10431F449E45DE005C042E15DE0CE
:10F4E00002C046E35DE066E27DE08C2D0F900F9058
:10F4F0000F900F90DF91CF911F910F91FF90EF90A0
:10F50000DF90CF90BF90AF909F908F907F906F9043
:10F510005F904F903F902F90CBCE02E010E07801AB
:10F52000EE0CFF1CEE0CFF1CC7018956994F7C01A5
:10F53000A3019201FC0160817181828193810F940A
:10F540002D2A882309F464CFF70140825182628218
:10F550007382FF24F39420E030E0A901C301B201DB
:10F560000F94863018160CF0F12CF401F08250CF75
:10F570008601D5CF0F900F900F900F90DF91CF9114
:10F580001F910F91FF90EF90DF90CF90BF90AF90C1
:10F590009F908F907F906F905F904F903F902F90B3
:10F5A00008958F3F29F0811106C040E958E105C058
:10F5B0004DE558E102C040E858E16EE678E178CECA
:10F5C0008F3F29F0811106C043ED58E105C040EAA4
:10F5D00058E102C043EC58E161EB78E169CE2F922B
:10F5E0003F924F925F926F927F928F929F92AF92D3
:10F5F000BF92CF92DF92EF92FF920F931F93CF9320
:10F60000DF93CDB7DEB728970FB6F894DEBF0FBEF5
:10F61000CDBF8091640E811119C028960FB6F89461
:10F62000DEBF0FBECDBFDF91CF911F910F91FF9035
:10F63000EF90DF90CF90BF90AF909F908F907F9092
:10F640006F905F904F903F902F900895FEDD0F9444
:10F65000481B6B837C838D839E83312C22242394CF
:10F660008091730290917402181619060CF02BC148
:10F6700001979093740280937302232D30E03887B2
:10F680002F834901880C991C880C991CF401E952BC
:10F69000FB4F4080518062807380EF81F885E75096
:10F6A000FE4E8081811116C0D401A152BE4ECD9074
:10F6B000DD90ED90FC90C114D104E104F10451F00F
:10F6C0002B813C814D815E812C193D094E095F09DA
:10F6D00057FF20824F815885440F551F5A83498315
:10F6E000FA01E45AF14F60817181882777FD809596
:10F6F000982F0F94332A0EE1A02EB12CCF80D884FE
:10F700007B018C01A3019201B4016454794FC601BD
:10F710008654994F36DEF401E952FB4F4080518008
:10F7200062807380E981FA81E153F94F60817181D0
:10F73000882777FD8095982F0F94332A9B01AC0181
:10F74000C301B2010F9486301816A4F4E981FA813E
:10F75000E558FD4F60817181882777FD8095982F4E
:10F760000F94332A9B01AC01C301B2010F942D2ADF
:10F7700087FDE2C060E0EF81F885E958F14F6083D2
:10F78000F401EE54F94F80819181A281B3810097F9
:10F79000A105B10551F12B813C814D815E81281B72
:10F7A000390B4A0B5B0B57FD20C0832D0E94315053
:10F7B0002B013C01E981FA81E255F94F60817181A9
:10F7C00080E090E00F94312A9B01AC01C301B201AB
:10F7D0000F942D2A87FFC3C0332009F4C7C04DE81A
:10F7E0005DE06EE77DE0832D63DD832D3394813012
:10F7F00009F036CF8091AA069091AB06A091AC0695
:10F80000B091AD060097A105B10521F12B813C8196
:10F810004D815E81281B390B4A0B5B0B57FD1AC0CB
:10F820000E9428502B013C016091A8067091A90606
:10F8300080E090E00F94312A9B01AC01C301B2013A
:10F840000F942D2A87FF8FC04CE55DE06FE67DE0C9
:10F850008FEF2EDD6091580E7091590E882777FD3D
:10F860008095982F0F94332A2091DF043091E00483
:10F870004091E1045091E204FAE0AF2EB12CCC2487
:10F88000CA94DC2C7B018C0163EA76E087EA96E07F
:10F8900078DD8091820E81115FC04090DF0450902E
:10F8A000E0046090E1047090E20420E030E040EA7F
:10F8B00050E4C301B2010F94863087FF2CC060E092
:10F8C0006093740EAACE432D50E058874F834A01AF
:10F8D000880C991C880C991C840109521B4FD80173
:10F8E0004D905D906D907C9020E030E848E953E4C5
:10F8F000C301B2010F948630181634F120E030E0D5
:10F9000040EA50E4C301B2010F942D2A87FFC5CE0F
:10F9100080E047DEBBCE20E030E046E153E4C301A7
:10F92000B2010F942D2A181654F20E94794D0F94AB
:10F93000A42F75956795C4CF832D0E94B64E0F9462
:10F94000A42F7595679517CF80E03ADEF8014080C7
:10F95000518062807380D2CF1092740E5ECE832D60
:10F960000E94834C42CF0E94394C74CF4FE95DE036
:10F9700038CF0F931F93CF93DF93EC018B016091EE
:10F98000C3124091C412641306C087EB92E10E9437
:10F99000F2FC25DEF4CF28813981F8018081918144
:10F9A0005091C21274E0579FF0011124E554FD4EAE
:10F9B00033872287958784876F5F6093C31281E0C6
:10F9C000850F841719F08093C21202C01092C212E0
:10F9D000DF91CF911F910F910895AF92BF92CF9277
:10F9E000DF92FF920F931F93CF93DF9300D01F926C
:10F9F000CDB7DEB7F82E662351F01092C8061092EC
:10FA0000C4061092C5061092C6061092C7060F943F
:10FA1000481B0091C4061091C5062091C60630917E
:10FA2000C7065B016C01A01AB10AC20AD30AD7FC4F
:10FA30003DC0F7FE05C004EC19E020E030E015C041
:10FA4000E091C8062F2D332727FD30952C5F3F4FBF
:10FA50004E2F552747FD5095241735073CF1EF15DC
:10FA600054F300E911E020E030E0DC01CB01800F2D
:10FA7000911FA21FB31F8093C4069093C506A09345
:10FA8000C606B093C70680ED97E09C838B838CE21B
:10FA900091E09A838983BE016D5F7F4FCE0101960D
:10FAA00068DF8091C8068F5F8093C8060F900F9023
:10FAB0000F900F90DF91CF911F910F91FF90DF90EA
:10FAC000CF90BF90AF900895CF93DF9300D01F9257
:10FAD000CDB7DEB783E50F941519882319F00F947D
:10FAE0001B1702C064E071E07C836B8380E50F9498
:10FAF0001519882339F00F941B17693823E1720711
:10FB000030F402C068EE73E07A83698304C088E849
:10FB100093E19A838983BE016D5F7F4FCE01019689
:10FB200028DF0F900F900F900F90DF91CF910895E5
:10FB3000CF92DF92EF92FF926B017C0183E3C816B4
:10FB4000D104E104F10468F082E3C81AD108E108A5
:10FB5000F10862E370E080E090E00F94B51A3FDDB9
:10FB6000EDCFC701B6010F94B51AFF90EF90DF906B
:10FB7000CF9035CDCF93DF931F921F92CDB7DEB7D5
:10FB8000789484B5826084BD84B5816084BD85B578
:10FB9000826085BD85B5816085BD80916E00816084
:10FBA00080936E001092810080918100826080932A
:10FBB000810080918100816080938100809180002C
:10FBC0008160809380008091B10084608093B10057
:10FBD0008091B00081608093B0008091910082603C
:10FBE0008093910080919100816080939100809139
:10FBF00090008160809390008091A100826080934A
:10FC0000A1008091A10081608093A1008091A0005B
:10FC100081608093A0008091210182608093210106
:10FC20008091210181608093210180912001816078
:10FC30008093200180917A00846080937A00809183
:10FC40007A00826080937A0080917A00816080934C
:10FC50007A0080917A00806880937A001092C100C7
:10FC60006F98779A82E08093C0001092C50087E079
:10FC70008093C4008091C10080618093C100809115
:10FC8000C10088608093C1008091C100806880932A
:10FC9000C10002ED1FE0F8018491882329F00F5F75
:10FCA0001F4F0E943954F7CF0BE210E1F801849105
:10FCB000882329F00F5F1F4F0E943954F7CFF4B605
:10FCC000F0FE0CC0E9ECFFE084918F010F5F1F4F45
:10FCD000882321F00E943954F801F6CFF1FE0CC0C0
:10FCE000E8EBFFE084918F010F5F1F4F882321F025
:10FCF0000E943954F801F6CFF2FE0CC0E6EAFFE0AC
:10FD000084918F010F5F1F4F882321F00E94395487
:10FD1000F801F6CFF3FE0CC0E5E9FFE084918F0116
:10FD20000F5F1F4F882321F00E943954F801F6CF4E
:10FD3000F5FE0CC0E4E8FFE084918F010F5F1F4FD8
:10FD4000882321F00E943954F801F6CF14BE0DE744
:10FD50001FE0F8018491882329F00F5F1F4F0E9454
:10FD60003954F7CF80E20E94395406E71FE0F801CA
:10FD70008491882329F00F5F1F4F0E943954F7CFD9
:10FD80008AE00E9439540BE210E1F8018491882343
:10FD900029F00F5F1F4F0E943954F7CF06E61FE08E
:10FDA000F8018491882329F00F5F1F4F0E94395476
:10FDB000F7CF02E51FE0F8018491882329F00F5F57
:10FDC0001F4F0E943954F7CF09E11FE0F8018491D9
:10FDD000882329F00F5F1F4F0E943954F7CF0BE2A1
:10FDE00010E1F8018491882329F00F5F1F4F0E94D2
:10FDF0003954F7CF02E01FE0F8018491882329F0FD
:10FE00000F5F1F4F0E943954F7CF0BE210E1F8014A
:10FE10008491882329F00F5F1F4F0E943954F7CF38
:10FE20008091951590919615BE016F5F7F4F009759
:10FE300019F0681B790B02C06B59754183EF9EE086
:10FE40000E940CC260EF74E08CED9EE00E940CC238
:10FE50008AE00E94395481E08093F5068093F6068B
:10FE60008093F7068093F8060E9437B88CE0E9ED9E
:10FE7000F6E0A5EEB6E001900D928A95E1F70E94BA
:10FE800063BD80917B0290917C0290937E0280936F
:10FE90007D028091010180648093010180910101C4
:10FEA000806180930101809101018860809301014C
:10FEB0006D9A8091010188608093010186E00E9423
:10FEC00015678091010180628093010188E00E94A2
:10FED00015676C9A82E00E94156787ED80937A001F
:10FEE00010927E0010927D0080917E008160809350
:10FEF0007E0080917E00826080937E0080917E00F3
:10FF0000846080937E0080E888BD80916E0084606C
:10FF100080936E006AEF70E080E090E00F94B51A75
:10FF200085E090E09093D0068093CF0660E08091CA
:10FF30007702909178020E943C5020E030E040EA45
:10FF400050E40F942D2A87FF0AC080917702909188
:10FF5000780240979093780280937702E7CF81E30D
:10FF600091E090937C0280937B0260E08091CB06CD
:10FF70009091CC060E943C5020E030E848E953E4E0
:10FF80000F948630181654F48091CB069091CC06CD
:10FF900040969093CC068093CB06E7CF85E090E027
:10FFA0009093D2068093D10661E08091790290917E
:10FFB0007A020E943C5020E030E040EA50E40F9486
:10FFC0002D2A87FF0AC08091790290917A0240978A
:10FFD00090937A0280937902E7CF81E391E0909346
:10FFE0007E0280937D0261E08091CD069091CE06E5
:10FFF0000E943C5020E030E848E953E40F948630FA
:020000021000EC
:10000000181654F48091CD069091CE0640969093A8
:10001000CE068093CD06E7CF80917502909176024F
:100020000E94D94C20E030E040EA50E40F942D2AA1
:1000300087FF0AC080917502909176024097909355
:10004000760280937502E8CF8091C9069091CA0626
:100050000E94D94C20E030E046E153E40F94863012
:10006000181654F48091C9069091CA064096909350
:10007000CA068093C906E8CF28E288E190E00FB66F
:10008000F894A895809360000FBE209360001FB77E
:10009000F8948091D306811124C0E6E4FEE08491B7
:1000A000E0E0FEE09491E82FF0E0EE0FFF1FEF5448
:1000B000F24FA591B4918C91892321F461E085E3FD
:1000C0000F94131B85E30E94C4C68CB580618CBD60
:1000D0008CB580648CBD84E30E94C4C683E30E9417
:1000E000C4C68091D3068F5F8093D3061FBF579AF3
:1000F00002E913E0F12CF80161918F0170E08F2D7E
:100100000F94F102F394F5E0FF12F5CF999A989AC3
:10011000809107018068809307019A9A8091070176
:1001200080648093070180910701806280930701BA
:1001300080910701886080930701809107018061A9
:10014000809307018091070182608093070180916D
:10015000070184608093070107E913E0F12CF8019F
:1001600061918F018F2D0E94DB51F394F5E0FF1216
:10017000F6CF80910A01826080930A0180910A0182
:10018000816080930A0180910A01846080930A0152
:1001900080910A01806480930A0180910A0180683D
:1001A00080930A010F9A179A0E9A169A0D9A159A29
:1001B0000C9A149A0B9A139A26982E9A25982D9A8F
:1001C00024982C9A0A98129A0998119A3F98479A5B
:1001D0000898109A389A4098179A1092D506399A2A
:1001E0004198169A1092D6063A9A4298159A109209
:1001F000D7063B9A4398149A3C9A4498139A809154
:1002000080008C7F8093800080918100877E886051
:1002100080938100809180008F7380938000809113
:100220008100887F82608093810080E090E49093D9
:10023000890080938800109285001092840080913C
:100240006F00826080936F0081E08093D406789481
:100250000E9434521092D8066C9A0E945B9764EC0C
:1002600079E080E090E064DC80917F02811110C031
:1002700064EC79E080E090E05BDCA0E6CA2EBDE0B3
:10028000BB2E07EF1FE080E0E82E80E0F82EAEC026
:1002900010927F022091331230E0C901C89797FD78
:1002A000019695958795E82E2E513109369527951B
:1002B000F22E0F94330007E51EE023E147E06CE0E7
:1002C0008E2D0E94475E84E00E9435C80091331253
:1002D00010E002571109169507956091341262518A
:1002E00048E753E08F2D0E94C0966091341266500B
:1002F0004EE753E0802F0E94C0960E94A7C781114D
:10030000DACFB6CF80911A0780FD5EC180911A07BF
:1003100084FD5AC150E2A52E80911A0781FD71C15A
:1003200080911A0785FD6DC140E2942E80911A07D5
:1003300082FD84C180911A0786FD80C130E2832E40
:1003400080911A0783FF3BC16091160770911707D0
:1003500080911807909119070F94332A2091020772
:100360003091030740910407509105070F94922A9A
:10037000AB01BC018CE090E10E9490D490E58AE052
:100380009A830E9439541F929A819F931F928F9251
:100390001F929F921F92AF921F930F931F920E94E2
:1003A0009C6510921A070FB6F894DEBF0FBECDBF42
:1003B0008091F906882391F01092E41286ED94E181
:1003C0000E94425786ED94E10E943D5B1092E31239
:1003D0001092E2120E940DFA0F94150480E00F941F
:1003E000DA11E114F10421F00E9400006AE0D62E37
:1003F00080919C08843010F40F94530F80918F15D6
:100400008823E1F00F94481B40908B1550908C1579
:1004100060908D1570908E1564197509860997097D
:1004200097FD0CC010928F158091E5128111C9C003
:100430000E944F5B8091E5128111C3C080919C089E
:10044000882309F49CC08091E212882309F485C0B6
:1004500080909B08C89C40011124C401855E984F80
:100460004C0164E470E10F94AD29892B01F186ED14
:1004700094E10E94425786ED94E10E943D5B109208
:10048000E3121092E212E1E3F0E184914F019FEF59
:10049000891A990A882341F00E943954F401F5CF52
:1004A0008091E312811159C00F94FF0558C0F401E7
:1004B00001900020E9F7CF0101973C016818790805
:1004C0001092D6146EE470E0C4010F9495312C01A3
:1004D000009729F4F3013197E80DF91D0DC060E292
:1004E00070E00F94953101964C016AE270E0C20110
:1004F0000F949531FC013197B182D2821382F401BD
:1005000001900020E9F7AF014150510948195909FC
:10051000B40186ED94E10E94AB598091D6148823F2
:1005200009F4BECFE0EFFFE084914F019FEF891AFD
:10053000990A882321F00E943954F401F5CFE9ED9E
:10054000FFE084914F019FEF891A990A882309F4EB
:10055000A7CF0E943954F401F4CF0E94EF2B809171
:100560009C08882361F0815080939C0880919B08AF
:100570008F5F80939B08843010F010929B088091CD
:100580001A07882309F42ACFEBE2F0E184914F01A6
:100590009FEF891A990A882321F00E943954F401A7
:1005A000F5CFECE1F0E184914F019FEF891A990AB0
:1005B000882309F4A7CE0E943954F401F4CF90E2C5
:1005C000DECE0E94816E3ACF60910E0770910F07C8
:1005D00080911007909111070F94332A2091FA0609
:1005E0003091FB064091FC065091FD060F94922A33
:1005F000AB01BC0188E190E10E9490D428E5A22ED5
:100600008BCE60911207709113078091140790911F
:1006100015070F94332A2091FE063091FF06409172
:100620000007509101070F94922AAB01BC0184E1AD
:1006300090E10E9490D499E5992E78CE60911607AA
:100640007091170780911807909119070F94332A1A
:10065000209102073091030740910407509105074C
:100660000F94922AAB01BC0180E190E10E9490D4EA
:100670008AE5882E65CE1F920F920FB60F92112435
:100680000BB60F922F933F934F935F936F937F938C
:100690008F939F93AF93BF93EF93FF9380917D0EC2
:1006A00090917E0EA0917F0EB091800E892B8A2BA7
:1006B0008B2B59F190917C0EE0917A0EF0917B0E8C
:1006C00080818927808380917D0E90917E0EA091FC
:1006D0007F0EB091800E181619061A061B060CF034
:1006E00056C080917D0E90917E0EA0917F0EB091AC
:1006F000800E0197A109B10980937D0E90937E0E23
:10070000A0937F0EB093800E42C080918902E3EEE9
:10071000F8E1E4919FEF90938902E230C9F050F440
:10072000EE2399F0E13081F590916F009D7F9093D9
:100730006F002AC0E43019F1E0F0E53029F590911E
:1007400073009D7F909373001FC010926E001CC0B9
:10075000909170009D7F9093700091E09093B00015
:100760009091B100987F94609093B1001092B30083
:100770000BC0909171009D7F9093710005C0909186
:1007800072009D7F9093720060E00F94131BFF91A5
:10079000EF91BF91AF919F918F917F916F915F91F9
:1007A0004F913F912F910F900BBE0F900FBE0F9066
:1007B0001F9018951F920F920FB60F9211240BB62F
:1007C0000F920F931F932F933F934F935F936F93CA
:1007D0007F938F939F93AF93BF93CF93DF93EF93C9
:1007E000FF938091790E8111DFC181E08093790EB2
:1007F00080916E008B7F80936E0078948091880248
:100800008F3778F18F579091770E9093760E2FB7A0
:10081000992329F0F89490910201906404C0F8940F
:10082000909102019F7B909302012FBF9091780ECF
:100830009093750E2FB7992329F0F89490910201A7
:10084000906104C0F894909102019F7E9093020100
:100850002FBF9091740E9093730E9923F1F0759AB7
:100860001DC09091760E891740F02FB7F8949091A3
:1008700002019F7B909302012FBF9091750E891703
:1008800040F02FB7F894909102019F7E909302015F
:100890002FBF9091730E891708F075988F5F809322
:1008A00088028091720E91E089278093720E8111E7
:1008B0000E9463D28091870290E08730910508F012
:1008C00057C0FC01E258FF4F0D944F318091710EDB
:1008D000811103C084E08093710E8091710E81506C
:1008E0008093710E882309F443C085E080938702CA
:1008F0003FC010927B0080E412C0209178003091BC
:1009000079008091670E9091680E820F931F9093EB
:10091000680E8093670E2CC010927B0082E4809357
:100920007C0080917A00806480937A0021C02091BD
:100930007800309179008091650E9091660E820F5B
:10094000931F9093660E8093650E12C010927B00E9
:1009500081E4E5CF20917800309179008091690E93
:1009600090916A0E820F931F90936A0E8093690E86
:1009700010918702111182C0809186028F5F80934F
:10098000860280310CF47AC0109286028091640E47
:1009900081111BC08091670E9091680E9093610E3B
:1009A0008093600E8091690E90916A0E9093630E11
:1009B0008093620E8091650E9091660E90935B0E0F
:1009C00080935A0E81E08093640E8AE0E7E6FEE0B1
:1009D000DF011D928A95E9F71092660E1092650E5E
:1009E000C091600ED091610ED195C195D1098091D1
:1009F000CB069091CC069195819591098C179D0716
:100A00000CF472C080917702909178029195819553
:100A10009109C817D9070CF477C0C091620ED09124
:100A2000630ED195C195D1098091CD069091CE06E6
:100A30009195819591098C179D070CF475C0809153
:100A4000790290917A02919581959109C817D907F9
:100A50000CF47AC0C0915A0ED0915B0E2091C90659
:100A60003091CA062C173D070CF07EC0209175020C
:100A700030917602C217D3070CF086C0812F90E028
:100A8000019667E070E00F943C318093870200E0AC
:100A900010E0E801CC0FDD1FCE5AD14F888199813B
:100AA0001816190644F461E0802F0F94D20588814E
:100AB0009981019709C0892B49F060E0802F0F943C
:100AC000D205888199810196998388830F5F1F4F92
:100AD00003301105F1F6F8941092790E80916E00B2
:100AE000846080936E0060C080915C0E90915D0E7A
:100AF000181619060CF086CF43ED58E161EB78E14A
:100B000080E00E9458797ECF80915C0E90915D0EBE
:100B1000181619060CF081CF40E958E16EE678E12D
:100B200080E00E94587979CF80915E0E90915F0E9F
:100B3000181619060CF083CF43EC58E161EB78E10D
:100B400081E00E9458797BCF20915E0E30915F0E3C
:100B5000121613060CF07ECF40E858E16EE678E1FD
:100B600081E00E94587976CF2091580E3091590E2D
:100B7000121613060CF07ACF40EA58E161EB78E1E7
:100B80008FEF0E94587972CF2091580E3091590EF4
:100B9000121613060CF072CF4DE558E16EE678E1BF
:100BA0008FEF0E9458796ACFFF91EF91DF91CF913B
:100BB000BF91AF919F918F917F916F915F914F9175
:100BC0003F912F911F910F910F900BBE0F900FBE71
:100BD0000F901F9018951F920F920FB60F9211242D
:100BE0000BB60F92BF92CF92DF92EF92FF920F93CC
:100BF0001F932F933F934F935F936F937F938F93A5
:100C00009F93AF93BF93EF93FF93CF93DF9300D066
:100C10001F92CDB7DEB780916E008B7F80936E0000
:100C200080916F008D7F80936F007894C0904E0EFE
:100C3000D0904F0EE090500EF090510EC114D104A0
:100C4000E104F10409F442C08091D406811104C08A
:100C50008091D8068823D1F10E9429CCF9EBCF16D8
:100C6000FBE0DF06E104F10488F008EBC01A0BE0BA
:100C7000D00AE108F108C0924E0ED0924F0EE092D9
:100C8000500EF092510E88EB9BE009C0C601109205
:100C90004E0E10924F0E1092500E1092510E9093D5
:100CA000890080938800209188003091890080918C
:100CB00084009091850040962817390708F070C08D
:100CC0008091840090918500409620C080914C0EC8
:100CD00090914D0E009709F496C08C0101501109B6
:100CE00010934D0E00934C0E10924B0E10924A0E24
:100CF0000F946800012B41F481E598E1909322095B
:100D0000809321090E94ED6B88EC90E0909389001C
:100D10008093880045C0C8010E94BFDB24E630E014
:100D20008091D406882309F4B5C4C901293BBBE0EE
:100D30003B0708F0E8C590938900809388004091B4
:100D40003B0E50913C0E60913D0E70913E0E420F55
:100D5000531F611D711D40933B0E50933C0E6093D9
:100D60003D0E70933E0E2091880030918900809155
:100D700084009091850040962817390748F48091A7
:100D8000840090918500409690938900809388001C
:100D9000BB2031F010924B0E10924A0E0F94680057
:100DA000F8948091790E882321F080916E008B7FDA
:100DB00003C080916E00846080936E0080916F000C
:100DC000826080936F000F900F900F900F90DF91D3
:100DD000CF91FF91EF91BF91AF919F918F917F91B3
:100DE0006F915F914F913F912F911F910F91FF90C4
:100DF000EF90DF90CF90BF900F900BBE0F900FBE83
:100E00000F901F90189580914A0E90914B0E892B50
:100E100009F0B1C19091B5128091B612981749F1BD
:100E20009091B6121FE4919F90011124295D364FD5
:100E30008091230990912409A0912509B091260958
:100E4000F901E55BFF4F4081518162817381841B11
:100E5000950BA60BB70B8093230990932409A093BD
:100E60002509B0932609D9018C9188608C9369017A
:100E70000DC08FB7F8941092230910922409109294
:100E80002509109226098FBFC12CD12CD0924B0E70
:100E9000C0924A0EC114D10409F46AC1F60152A1EC
:100EA0008091490E418158130AC0242F30E080916F
:100EB0008502992787FD90952817390731F05093BF
:100EC000490E409385020E9434521092450E1092B2
:100ED000460E1092470E1092480ED601D7968D916D
:100EE0009C91D8978134BCE99B0728F48132EEE4C9
:100EF0009E0748F002C080E49CE9969587959695F8
:100F0000879524E007C08131F7E29F0730F096957E
:100F1000879522E02093440E08C021E02093440EE0
:100F20008032910510F480E290E08C0100521109AA
:100F3000011528E01207D0F0812F9927880F991FFB
:100F4000880F991F8F5A9B4EFC0132964591549100
:100F5000AA27059F9001049F210D3A1F06942A1F7E
:100F60003A1F1124FC01859194911DC0C8019695EA
:100F700087958C7F8F5A9F4EFC0145915491029624
:100F8000FC0185919491B80167707727869F900145
:100F9000879F300D969F300D112463E0369527957D
:100FA0006A95E1F7CA01821B930B8436910588F498
:100FB0008CE9E82E83E0F82ED7018D917D018823FE
:100FC00019F00E943954F8CFC8010E94BFDB84E6B3
:100FD00090E09093430E8093420E8091440E809354
:100FE000410EF60183AD94AD9093400E80933F0E79
:100FF0008134FCE99F0728F481320EE4900748F021
:1010000002C080E49CE9969587959695879524E0A3
:1010100007C0813117E2910730F09695879522E05D
:101020002093440E08C021E02093440E80329105A5
:1010300010F480E290E08C0100521109011528E0C3
:101040001207E0F0812F9927880F991F880F991FA9
:101050008F5A9B4EFC01329625913491AA27039F0B
:10106000A001029F410D5A1F06944A1F5A1F1124C6
:10107000FC0125913491241B350B1EC0C8019695A7
:1010800087958C7F8F5A9F4EFC0125913491029653
:10109000FC0145915491B80167707727469FC001C4
:1010A000479F900D569F900D1124E3E096958795EC
:1010B000EA95E1F7281B390B2436310588F46CE9F1
:1010C000E62E63E0F62ED7018D917D01882319F07D
:1010D0000E943954F8CFC8010E94BFDB24E630E0FB
:1010E000C901A0E0B0E080933B0E90933C0EA0932A
:1010F0003D0EB0933E0E3093890020938800F60198
:1011000082899389A489B589B695A795979587957E
:10111000B095A095909581959F4FAF4FBF4F80930D
:10112000370E9093380EA093390EB0933A0E8093F9
:10113000330E9093340EA093350EB093360E8093F9
:101140002F0E9093300EA093310EB093320E8093F9
:101150002B0E90932C0EA0932D0EB0932E0E10926A
:10116000270E1092280E1092290E10922A0E03C0FC
:1011700080ED97E0CBCD8091D4068111C1C38091E1
:10118000D8068111BDC32091440E222309F4ABC1BE
:10119000E0914A0EF0914B0E80912B0E90912C0E07
:1011A000A0912D0EB0912E0E4281538164817581E4
:1011B000840F951FA61FB71F80932B0E90932C0EA4
:1011C000A0932D0EB0932E0E181619061A061B06A4
:1011D0000CF4409AE0914A0EF0914B0E80912F0E44
:1011E0009091300EA091310EB091320E4681578110
:1011F00060857185840F951FA61FB71F80932F0EE2
:101200009093300EA093310EB093320E181619063B
:101210001A061B060CF4419AE0914A0EF0914B0E0F
:101220008091330E9091340EA091350EB091360E10
:101230004285538564857585840F951FA61FB71F4A
:101240008093330E9093340EA093350EB093360EE8
:10125000181619061A061B060CF4429AE0914A0E5B
:10126000F0914B0E8091370E9091380EA091390E6F
:10127000B0913A0E4685578560897189840F951F14
:10128000A61FB71F8093370E9093380EA093390E88
:10129000B0933A0E181619061A061B0634F481810B
:1012A000811102C0439A01C0449A80912B0E909103
:1012B0002C0EA0912D0EB0912E0E181619061A069E
:1012C0001B0684F5E0914A0EF0914B0E428953893A
:1012D00064897589841B950BA60BB70B80932B0E25
:1012E00090932C0EA0932D0EB0932E0E4091810260
:1012F0008091170E9091180EA091190EB0911A0EB0
:10130000552747FD5095652F752F840F951FA61FF4
:10131000B71F8093170E9093180EA093190EB093D9
:101320001A0E409880912F0E9091300EA091310EA0
:10133000B091320E181619061A061B0684F5E091B4
:101340004A0EF0914B0E4289538964897589841B3A
:10135000950BA60BB70B80932F0E9093300EA09396
:10136000310EB093320E4091820280911B0E90910B
:101370001C0EA0911D0EB0911E0E552747FD5095D5
:10138000652F752F840F951FA61FB71F80931B0E07
:1013900090931C0EA0931D0EB0931E0E4198809149
:1013A000330E9091340EA091350EB091360E181672
:1013B00019061A061B0684F5E0914A0EF0914B0EB1
:1013C0004289538964897589841B950BA60BB70BD9
:1013D0008093330E9093340EA093350EB093360E57
:1013E0004091830280911F0E9091200EA091210EBA
:1013F000B091220E552747FD5095652F752F840F0C
:10140000951FA61FB71F80931F0E9093200EA093C9
:10141000210EB093220E42988091370E9091380E93
:10142000A091390EB0913A0E181619061A061B062D
:10143000ACF5E0914A0EF0914B0E428953896489D4
:101440007589841B950BA60BB70B8093370E909371
:10145000380EA093390EB0933A0E409184028091D9
:10146000230E9091240EA091250EB091260E5527A3
:1014700047FD5095652F752F840F951FA61FB71F29
:101480008093230E9093240EA093250EB093260EE6
:101490008181811102C0439801C044988091270E38
:1014A0009091280EA091290EB0912A0E0196A11DAF
:1014B000B11D8093270E9093280EA093290EB09310
:1014C0002A0E2150E0914A0EF0914B0E4289538929
:1014D0006489758984179507A607B70708F455CE60
:1014E000BB24B39401C0B12C4091270E5091280E1B
:1014F0006091290E70912A0EE0904A0EF0904B0EEA
:10150000F70186899789A08DB18D84179507A60765
:10151000B70708F4C5C040913B0E50913C0E609156
:101520003D0E70913E0E068D178D20A131A1AA2788
:10153000419FB12D529FC001629F900D619F800D10
:10154000911D429FB00D811D9A1F519FB00D811DAD
:101550009A1F609FB00D811D9A1F509FB10D8A1F69
:101560009A1FB6958A1F9A1F349F800D911D359F33
:10157000900D112443AD54AD480F591F5093400EA8
:1015800040933F0E87A990ADA1ADB2AD60E070E091
:1015900084179507A607B70720F49093400E809311
:1015A0003F0E80913F0E9091400E8134BCE99B0725
:1015B00028F48132EEE49E0748F002C080E49CE902
:1015C000969587959695879524E007C08131F7E237
:1015D0009F0730F09695879522E02093440E08C02F
:1015E00021E02093440E8032910510F480E290E0D7
:1015F0008C0100521109011528E01207E0F0812F3B
:101600009927880F991F880F991F8F5A9B4EFC01AD
:10161000329625913491AA27039FA001029F410D84
:101620005A1F06944A1F5A1F1124FC012591349118
:10163000241B350B1EC0C801969587958C7F8F5A49
:101640009F4EFC01259134910296FC0145915491E5
:10165000B80167707727469FC001479F900D569F3E
:10166000900D1124B3E096958795BA95E1F7281B64
:10167000390B2436310508F053CBFCE9EF2EF3E0AB
:10168000FF2ED7018D917D01882309F444CB0E9460
:101690003954F7CF8091D806811147CBC9014BCB84
:1016A0004091270E5091280E6091290E70912A0EBC
:1016B000F701828D938DA48DB58D84179507A607AC
:1016C000B70708F0EAC00091450E1091460E209130
:1016D000470E3091480E09831A832B833C83468D35
:1016E000578D60A171A1AA27059FB12D169F60019A
:1016F000269FD00C259FC00CD11C069FB00DC11C8D
:10170000DA1E159FB00DC11CDA1E249FB00DC11C3E
:10171000DA1E149FB10DCA1EDA1EB695CA1EDA1E55
:10172000709FC00CD11C719FD00C112480913F0E72
:101730009091400EFF96C816D90680F48C199D0929
:1017400040815181628173818C0120E030E0041777
:1017500015072607370720F4CA0102C0808191814E
:1017600081341CE9910728F481322EE4920748F075
:1017700002C080E49CE9969587959695879524E02C
:1017800007C0813137E2930730F09695879522E0C4
:101790002093440E08C021E02093440E803291052E
:1017A00010F480E290E08C0100521109011548E02C
:1017B0001407E0F0812F9927880F991F880F991F30
:1017C0008F5A9B4EFC01329625913491AA27039F94
:1017D000A001029F410D5A1F06944A1F5A1F11244F
:1017E000FC0125913491241B350B1EC0C801969530
:1017F00087958C7F8F5A9F4EFC01259134910296DC
:10180000FC0145915491B80167707727469FC0014C
:10181000479F900D569F900D112443E09695879514
:101820004A95E1F7281B390B2436310588F49CE9E9
:10183000E92E93E0F92ED7018D917D01882319F0CF
:101840000E943954F8CFC8010E94BFDB24E630E083
:101850008091D406811104C08091D806882339F084
:10186000C901293BBBE03B0708F068C001C0C901C2
:10187000909389008093880089819A81AB81BC8193
:10188000820F931FA11DB11D8093450E9093460EAC
:10189000A093470EB093480E66CA2091420E309135
:1018A000430E8091D406811104C08091D80688230C
:1018B000F1F0293BEBE03E07D0F0C90168EB7BE09B
:1018C0000F942831883E43E0940708F052C08854B2
:1018D000944FA901481B590B60E070E040934E0EF5
:1018E00050934F0E6093500E7093510E9C013093A5
:1018F0008900209388008091410E8093440E33CA62
:101900000E9429CC40CC68EB7BE00F942831883EC4
:1019100003E0900780F48854944FA901481B590BA9
:1019200060E070E040934E0E50934F0E6093500E67
:101930007093510E00CA88EB9BE0EFCF68EB7BE021
:101940000F942831883E13E0910780F48854944F17
:10195000A901481B590B60E070E040934E0E509374
:101960004F0E6093500E7093510E82CF88EB9BE028
:10197000EFCF88EB9BE0ADCF1F920F920FB60F9287
:1019800011240BB60F922F933F934F935F936F9356
:101990007F938F939F93AF93BF93EF93FF93209188
:1019A000C6009FB7F894E0911F0981E08E0F8F77F2
:1019B00030912009831731F0F0E0E156F74F208392
:1019C00080931F099FBF30919E08832F90E08C3039
:1019D000910508F044C0FC01EB57FF4F0D944F31C7
:1019E0002D3441F02E34B9F481E005C02A3330F0B3
:1019F0002D3481F582E080939E0846C0203308F0A4
:101A000043C0203209F440C02D3221F53DC02133BE
:101A100029F0243329F02032E9F436C083E0EBCFFB
:101A200088E0E9CF203321F02133A1F486E0E3CF31
:101A300084E0E1CF283371F485E0DDCF223351F427
:101A400087E0D9CF213331F489E0D5CF203311F4A9
:101A50008AE0D1CF8BE0CFCF2A30B1F413C02A3047
:101A600099F4373049F03A3059F0353059F4109242
:101A7000800210929D0806C088E490E10E94BA7826
:101A80000E940DFA10929E08FF91EF91BF91AF91C5
:101A90009F918F917F916F915F914F913F912F9186
:101AA0000F900BBE0F900FBE0F901F901895609176
:101AB00035127091361280934F1281E38093501249
:101AC00081E08093521280EF809351122FE432E133
:101AD0004BE383E392E10D944C1A0F93CF93DF9382
:101AE000C82FD62F04E0262F41E3682F83E392E12D
:101AF0000F942A1A8823B9F02D2F41E36C2F83E32A
:101B000092E10E9447FD8C2FD2DF8FEF8D0F8C0F5B
:101B1000CEDF2D2F44E36C2F83E392E1DF91CF9151
:101B20000F910C9447FDDF91CF910F9108954F9243
:101B30005F926F927F928F929F92AF92BF92CF925D
:101B4000DF92EF92FF920F931F93CF93DF93CDB766
:101B5000DEB72A970FB6F894DEBF0FBECDBF109246
:101B6000231280911B12882351F00E94399740E084
:101B700050E0BA018EE59AEF0E940FD4DFC4409185
:101B80009C0250919D0280911F1290912012A09171
:101B90002112B09122129A01280F391F44365105A3
:101BA00024F4253631053CF41CC04436510551F06F
:101BB00024363105B4F484E690E090939D0280933E
:101BC0009C0213C08B309105A105B1051CF02A5071
:101BD000310907C0863F9F4FAF4FBF4F74F4265F58
:101BE0003F4F30939D0220939C0210921F1210923F
:101BF0002012109221121092221280919C02909138
:101C00009D028A3091053CF0883E53E095072CF008
